:020000040800F2
:100000000020001025CD020825850208C9530008EC
:10001000218502081D8502081985020800000000DC
:10002000000000000000000000000000158502082C
:1000300011850208000000000D850208D96600083D
:100040008DCD02088DCD02088DCD02088DCD020820
:100050008DCD02088DCD0208C5270008F1280008C3
:10006000B5280008792800083D280008B13E00089E
:10007000A13E0008913E0008813E0008713E000844
:100080005D3E0008493E00088DCD02088DCD020876
:1000900081D501088DCD02088DCD02080128000808
:1000A000C95F0008196000088DCD020829600008AA
:1000B00009600008F95F00088DCD02088DCD0208A7
:1000C0008DCD02088DCD02088DCD02088DCD0208A0
:1000D0008DCD02088DCD02088DCD02080D67000878
:1000E000892700088DCD020871D501088DCD020841
:1000F000D95F00088DCD0208E95F00088DCD0208A8
:100100000000000000000000000000008DCD02088B
:100110008DCD02088DCD0208891A01086D1A0108DB
:10012000353E0008213E00080D3E0008F93D00085C
:10013000E53D00088DCD0208000000000000000031
:100140008DCD02088DCD02088DCD02080000000083
:10015000000000000000000000000000000000009F
:1001600000000000000000008DCD02088DCD0208C7
:100170008DCD02080000000000000000000000001B
:08018000000000008DCD020813
:100188002B2303732A238370002383757047036826
:100198002DE9F041DF691FB13B46BDE8F041184742
:1001A800002A164611DD04460D460E4400E0236879
:1001B8009B68204698470028F9D0236815F8011B4A
:1001C8001B6820469847AE42F1D1BDE8F081002374
:1001D8003F22027043708370C37070471523037009
:1001E8001623C370172383712D2343702E230371A5
:1001F8002F23C3717047002870B51EDB09280446F9
:1002080020DD012303EB83035B00B0FBF3F2092A33
:10021800F8D87BB10D4EB4FBF3F00928CCBF5722B8
:100228003022A6FB03E5024403FB1044EB0801F867
:10023800012BF0D100230B7070BD2D230B704042B1
:100248000131DBE7303001F8010BF3E7CDCCCCCC42
:10025800884230B44FF001042ED301FB04F4B0FB04
:10026800F4F58D42F9D284B1AAB901E0B0FBF4F5F6
:10027800092DCCBF572230222A4404FB150003F86D
:10028800012BB4FBF1F4002CF0D100221A7030BC21
:100298007047B0FBF4F5092DCCBF372230222A4431
:1002A80004FB150003F8012BB4FBF1F4002CF0D18A
:1002B80000221A7030BC70470546002AEBD1D7E7F8
:1002C80003685A1C0260197070472DE9F047089CB2
:1002D8002578002B804689460CBF4FF0200A4FF046
:1002E800300A661C35B3002A29DD334601E0024690
:1002F80098B113F8011B501E0029F8D1971E60B160
:100308003D46013D51464046C8476B1C002BF8DC72
:10031800257827EAE770013055B1041B2946404685
:10032800C847301916F8015B002DF7D1BDE8F087F2
:10033800BDE8F087002A04DC2846BDE8F0870020E5
:10034800EBE7571EDCE783684268D0ED037A00EBE1
:1003580083010133934281ED040A836004BF0023C3
:10036800836000EB830393ED047A036870EE277AC9
:100378009A42C0ED037A77EEC77AC0ED037A0CDAB9
:10038800013307EE103AF8EEC76AB7EE007A87EE47
:10039800A60A036030EE070A704707EE102AB8EE87
:1003A800C77A87EE870A704790ED057A90ED004A84
:1003B800D0ED066AD0ED014AD0ED047A90ED035AEB
:1003C800D0ED025AA4EE007AB0EE406AB0EE470AC9
:1003D800B0EE667AA6EE247A67EEC07AA0EE457A89
:1003E800E6EE257A80ED057AC0ED067A7047D0ED05
:1003F800057A90ED013AD0ED003AD0ED064A90ED3D
:10040800024A90ED077A90ED035A90ED086AD0ED14
:10041800045AC0ED067AF0EE406A27EE830AC0ED72
:10042800056AA3EEA60A80ED087AA4EE240AA5EED2
:10043800470AA5EEC60A80ED070A7047D0ED007A94
:1004480090ED017A30EE670AE7EE007AB0EE670ABF
:10045800C0ED007A704770470A44914214D030B416
:100468000139551E41F2210211F8014F082380EA93
:10047800042004044CBF82EA40004000013B80B2E3
:10048800F7D18D42F0D130BC7047024B00221A7070
:100498005A7070477C230020044A13783F2B03D8F6
:1004A800D118013308711370704700BF7C230020F6
:1004B800F0B58F7A8D79CC7ACE790A7C4B7C9FED1A
:1004C8005C4A4FEA072C0CF4706C45EA0C053F01B6
:1004D80007F4706E03EE905A4FEA042C0D7A24014B
:1004E80004F470670CF4706C46EA0E0404EE904A4B
:1004F80045EA0C0405EE104A4C7A16023C431201F8
:1005080002F4706505EE904A4A7B0C7B06F470662F
:1005180034432A431D021B0106EE104A06EE902AB8
:1005280003F470648A7BCB7B05F470652A4323430C
:1005380007EE102A07EE903AB8EEC55AF8EEE33AFD
:10054800F8EEE55A25EE045AF8EEE44AB8EEC66A23
:10055800F8EEE66AB8EEC77AF8EEE77A65EE845AFE
:1005680063EE843A64EE844A26EE046A66EE846A90
:1005780027EE047A67EE847ABCEEC55ABCEEE34AED
:10058800FCEEE55A87B015EE102AFCEEE44ABCEE04
:10059800C66AFCEEE66ABCEEC77AFCEEE77A15EEB0
:1005A800907A8DED014ABDF80410ADF80C2017EED5
:1005B800104A17EE902A14EE90EA16EE106A16EE1C
:1005C800905AADF80E700DF10A07ADF81440ADF869
:1005D8001620ADF808100B46ADF80AE0ADF810602B
:1005E800ADF812503A4606AC01E032F8023BA3F5EA
:1005F8004873B3F5AF6F0CD8A242F6D1831E0E3004
:1006080001E037F8021B23F8021F9842F9D107B01E
:10061800F0BD084B1B78162BF9D1074A0749B2F8E9
:10062800443001339BB2A2F844300B8007B0F0BDD0
:10063800ABAA2A3F385600207C2300203C560020D5
:100648002DE9F04FDFF81CB2DFF81CE2BBF8002000
:10065800DEF84860BBF90430BBF90250BBF90A80E8
:10066800C2EB261404FB04F424135200C2EBE60286
:1006780003FB04F305FB02F29B1303EBE223B3F540
:10068800FA364FEAE37589B045F1FF373246A6FBE3
:100698000645CDE9024502FB07F205EB4202CDE92A
:1006A8000467029EBBF90840039208FB02FC4FEA6C
:1006B800E87906FB09CC3A46A8FB0689049ECBF8E4
:1006C8001830E51704FB02F206FB0522A4FB0667B7
:1006D800E14417444FEA182242EA096200924FEABD
:1006E800292201923D03DDE90078340345EA1655D5
:1006F8003F19BBF80660069048EB05083C1C48F516
:10070800004503EB8302A4FB068906FB05998032AA
:1007180013124FEA69064FEAE977079356EA070387
:100728008A4600F09280DDE90489BBF90E20DEF8E4
:100738004C40BBF910004946C4F5801ED317DDE9CB
:10074800024502FB01F108FB0311A2FB08230B443D
:100758004FEA43492B46C11700FB03F304FB01335F
:10076800A0FB0401BBF90C401944E3000193734654
:10077800DC170023009349EAD2394FEA4248DDE901
:10078800002310EB080041EB0901E50712184FEAB6
:10079800CE744B4145EA5E05A41A65EB03052219A0
:1007A80045EB050312196B4199019001801841EA44
:1007B800926159418B00820043EA9073101943EB10
:1007C80005018B00820043EA907310460019194610
:1007D80032463B4669412CF0CDF8BBF916204C1344
:1007E800450B45EAC14502FB04F6D31705FB036632
:1007F800A2FB05233344BBF9146002FB04F405FB98
:10080800034406FB01FEA2FB0523F717234400FB64
:1008180007EE540EA6FB0067774444EAC3144FEA78
:10082800D64800194FEA636548EA473869414FEAF4
:10083800E74918EB0008BBF9124049EB01094FEAF8
:10084800182646EA096620013618069B0BB1360AB7
:100858001E60BAF1000F02D0079BCAF8003009B039
:10086800BDE8F08FD05D00207C23002070477047E2
:1008780050F8043C012280F84520103803B118478D
:10088800704790F8203033B1012B03D14FF4006347
:100898008382704770474FF480638382704770B5D6
:1008A800044682B01430E56D06236A464321A84702
:1008B800B0B19DF804009DF800609DF801109DF806
:1008C80002509DF803209DF8053041EA062143EACD
:1008D800002342EA0522A187E287A4F840300120DC
:1008E80002B070BD70B5044682B00830656A062350
:1008F8006A463B21A847A8B19DF804009DF800600E
:100908009DF801109DF802509DF803209DF80530D0
:1009180041EA062143EA002342EA0522E1822283D2
:100928006383012002B070BD70B40468037B226841
:10093800022101FA03F31A4213D042690A495820E6
:1009480000FB02124FF6FE7650685289C5680068AF
:10095800296831402960C168D24392B20A40C26016
:10096800636070BC704700BF584C002030B4094B1E
:100978001C7864B1084B002503EBC4041A689988F5
:100988005562D06808330143A342D160F6D130BC28
:10099800704700BF184F00201C4F002010B4026899
:1009A800047B11680223A340194209D00649406814
:1009B80000240C7001684FF6FE74214001605360FA
:1009C8005DF8044B704700BF095F0020F0B4334C5A
:1009D80000EB800004EB80046468002C5BD0304E90
:1009E80049004FF42040CDB23065A169090444D4D0
:1009F80060682C4F45F08071384041F490310143D4
:100A08004FF420406160306503E0411E002838D073
:100A18000846A1698F07F8D54FF42040A2623065D7
:100A280002E0421E68B31046A2691106F9D5626851
:100A38001C4945F0007545F480350A4015434FF4CC
:100A480020406560306502E0421ED0B11046A269C0
:100A58009207F9D5A362A3694FF420409B0630653D
:100A680005D4431E68B11846A3699B06F9D520230F
:100A78003065E3610120F0BC7047411E08B10846AB
:100A8800B3E7094A138801339BB24FF0FF31316550
:100A98001380F0BC70472046F0BC7047E43000205B
:100AA8007C230020009800FC984100201346002079
:100AB8000A4668218AE730B50446C06C617103684C
:100AC800A26823F00103036087B0A379009213F0B2
:100AD80004023DD04FF4805213F00203019244D136
:100AE80002934FF480630022039311F001030592EF
:100AF80037D1049308238D07694648BF049328F02B
:100B080021F96079E36CA17900F00202002A15BF8F
:100B18004FF440324FF480324FF40034002410F088
:100B2800010F586808BF2246CC074CBF024320EA91
:100B380002025A609A6809074CBF42F0080222F084
:100B480008029A601A6842F001021A6007B030BDC4
:100B580013F0020301920BD04FF40055134602958F
:100B6800C1E7042304930C23C5E74FF40053B7E708
:100B78000293B8E710B50446C06CA160036823F07F
:100B880001030360A37986B013F00402009141D0F9
:100B98004FF4805213F00203019244D102934FF4B0
:100BA800806362790393D1074FF0000304930593A0
:100BB80045BF0423049308230C236946920748BFC2
:100BC800049328F0BFF86079E36CA17900F0020281
:100BD800002A15BF4FF440324FF480324FF40034EE
:100BE800002410F0010F586808BF2246CC074CBFFC
:100BF800024320EA02025A609A6809074CBF42F091
:100C0800080222F008029A601A6842F001021A608B
:100C180006B010BD13F00203019207D04FF4005143
:100C280013460291BDE74FF40053B7E70293B8E7C4
:100C38002622192102702722002382704170012286
:100C48001A2102718371C1704271C37170472DE915
:100C5800F341056906460F467DBBD0F80080C8F30E
:100C68000A0323B30023D6F8008001932AF00EF973
:100C7800042819D1214C236943F001032361BBB235
:100C8800A8F800302AF002F904282ED108F102034E
:100C98000193019B3F0C1F802AF0F8F82369042870
:100CA80023F00103236125D06FF0010505E02AF048
:100CB800EDF8042805D04FF0FF35284602B0BDE80E
:100CC800F0810E4C236943F002032361C4F81480B9
:100CD800236943F0400323612AF0D8F823690428E4
:100CE80023F002032361BDD0E5E7236923F0010364
:100CF8002361D9E7336804333360DEE7002002401C
:100D0800F8B504460D468E180027B54201D1206972
:100D1800F8BDE368591CE160234415F8012B1A72E9
:100D28000429F2D1A1682046FFF791FFE76020610E
:100D3800EBE7F8B50D4E336AB28C1A850446FF20EE
:100D48000D462AF033F8074655B1013D54FA85F5AA
:100D5800013CFF202AF02AF804F8010FAC42F8D130
:100D6800336AB28C9A613846F8BD00BF3C6E0020E9
:100D780010F0AEBD38B51F4C94F8543094F8552097
:100D88001844C0B2904284F8540005D3801AC0B207
:100D98009042FBD284F85400362010F0ADFD94F850
:100DA80054502544232095F85C3303EB4303234434
:100DB80093F85810FFF7DCFF95F85C3303EB430317
:100DC8002344242093F85910FFF7D2FF95F85C3399
:100DD80003EB43031C44252094F85A10FFF7C8FF7F
:100DE80095F85C130A20FFF7C3FF3A20BDE83840A6
:100DF80010F082BD7C23002038B5104C054694F8CD
:100E08005B130C20FFF7B4FF08211820FFF7B0FF91
:100E18008DB994F859130920FFF7AAFF0D2107206F
:100E2800FFF7A6FF16211920FFF7A2FF0A20BDE849
:100E3800384005F0AFBB0321EDE700BF7C2300205D
:100E480010B490E80600047B40690223A3404B607D
:100E580013685DF8044B4FF6FE710B40136005F004
:100E68008FBC03682DE9F041DF691FB13B46BDE83F
:100E7800F0411847002A164611DD04460D460E4477
:100E880000E023689B68204698470028F9D023682B
:100E980015F8011B1B6820469847AE42F1D1BDE802
:100EA800F08103689B69184703685B691847036802
:100EB800DB68184703685B68184703681B681847AE
:100EC800014B1868F9E700BF34660020054B53F85A
:100ED800203033B11A689B88918A0B4218BF1B04D3
:100EE80093617047AC61002003682DE9F04F03F16E
:100EF8003845644EAD0A0124755D05F01F066D097D
:100F0800022D04FA06F400F0A280032D00F0A4805C
:100F1800012D52D08088B0FA80F4C4F11F04A4B225
:100F2800E50803EB850504F007042E6AA4000F27E3
:100F3800A74026EA07062E622E6A01F0030702FA86
:100F480004F47A1E3443012AC1F3810CC1F300185A
:100F58002C62C1F3411135D9C60700F19780850786
:100F680000F1A380440700F1B180020700F1BF80BF
:100F7800C60600F1CD80850600F1DB80440600F14D
:100F8800E980020600F1F780C60500F105818505B4
:100F980000F11381440500F12181020500F12F8140
:100FA800C60400F13D81850400F14B81440400F141
:100FB8005981020455D4BDE8F08F334D6E6934432E
:100FC8006C61A7E7002422464FF0010E4FF0030999
:100FD80004E00132102A04F10204ECD00EFA02F601
:100FE80036EA0005F5D1D3F808A009FA04F5ED436F
:100FF8000AEA050AC3F808A0D3F808B00CFA04FAFC
:101008004AEA0B0AC3F808A0B3F804A01FFA8AFA40
:101018002AEA06069E80B3F804A008FA02F646EA11
:101028000A06B6B29E801E682E401E60D3F800A045
:1010380007FA04F646EA0A061E60D3F80CA001FA7D
:1010480004F605EA0A0A46EA0A05DD60C1E70E4D1C
:10105800AE693443AC615DE70B4DEE693443EC6136
:1010680058E71A6822F040421A601A6842EA8777FD
:101078001F60DA6822F0404242EA8171D960BDE817
:10108800F08F00BFC41C0308001002401A6822F049
:1010980003021A601A683A431A60DA6822F00302F7
:1010A8000A438507DA607FF55DAF1A6822F00C0203
:1010B8001A601A6842EA87021A60DA6822F00C029B
:1010C80042EA81024407DA607FF54FAF1A6822F0DE
:1010D80030021A601A6842EA07121A60DA6822F0C7
:1010E800300242EA0112DA6002077FF541AF1A685E
:1010F80022F0C0021A601A6842EA87121A60DA6897
:1011080022F0C00242EA8112C606DA607FF533AFE8
:101118001A6822F440721A601A6842EA07221A60B2
:10112800DA6822F4407242EA01228506DA607FF525
:1011380025AF1A6822F440621A601A6842EA8722C8
:101148001A60DA6822F4406242EA81224406DA60D0
:101158007FF517AF1A6822F440521A601A6842EAFB
:1011680007321A60DA6822F4405242EA0132DA6041
:1011780002067FF509AF1A6822F440421A601A681D
:1011880042EA87321A60DA6822F4404242EA81323F
:10119800C605DA607FF5FBAE1A6822F440321A60A1
:1011A8001A6842EA07421A60DA6822F4403242EAD0
:1011B80001428505DA607FF5EDAE1A6822F4402217
:1011C8001A601A6842EA87421A60DA6822F44022F2
:1011D80042EA81424405DA607FF5DFAE1A6822F4FC
:1011E80040121A601A6842EA07521A60DA6822F452
:1011F800401242EA0152DA6002057FF5D1AE1A6860
:1012080022F440021A601A6842EA87521A60DA68C1
:1012180022F4400242EA8152C604DA607FF5C3AE86
:101228001A6822F040721A601A6842EA07621A6065
:10123800DA6822F0407242EA01628504DA607FF5DA
:10124800B5AE1A6822F040621A601A6842EA8762EC
:101258001A60DA6822F0406242EA81624404DA6085
:101268007FF5A7AE1A6822F040521A601A6842EA5F
:1012780007721A60DA6822F0405242EA0172DA60B4
:1012880097E6036803F138422DE9F04F920A584D6A
:10129800AA5C02F01F0552090124022A04FA05F487
:1012A80000F08C80032A00F08E80012A3CD001F0E7
:1012B80003077A1E012AC1F3810CC1F30018808844
:1012C800C1F3411135D9C60700F19680850700F1B1
:1012D800A280440700F1B080020700F1BE80C60674
:1012E80000F1CC80850600F1DA80440600F1E88040
:1012F800020600F1F680C60500F10481850500F1BB
:101308001281440500F12081020500F12E81C604F6
:1013180000F13C81850400F14A81440400F15881C0
:10132800020455D4BDE8F08F324A55692C43546104
:10133800BDE7002422464FF0010E4FF0030904E0F8
:101348000132102A04F10204ECD00EFA02F636EA51
:101358000005F5D1D3F808A009FA04F5ED430AEA27
:10136800050AC3F808A0D3F808B00CFA04FA4AEA48
:101378000B0AC3F808A0B3F804A01FFA8AFA2AEAED
:1013880006069E80B3F804A008FA02F646EA0A06A2
:10139800B6B29E801E682E401E60D3F800A007FAE1
:1013A80004F646EA0A061E60D3F80CA001FA04F611
:1013B80005EA0A0A46EA0A05DD60C1E70D4A9569A9
:1013C8002C43946173E70B4AD5692C43D4616EE7CB
:1013D8001A6822F040421A601A6842EA87771F604A
:1013E800DA6822F0404242EA8171D960BDE8F08FA4
:1013F800C41C0308001002401A6822F003021A6095
:101408001A683A431A60DA6822F003020A43850729
:10141800DA607FF55EAF1A6822F00C021A601A686B
:1014280042EA87021A60DA6822F00C0242EA810274
:101438004407DA607FF550AF1A6822F030021A606C
:101448001A6842EA07121A60DA6822F0300242EAA1
:101458000112DA6002077FF542AF1A6822F0C00273
:101468001A601A6842EA87121A60DA6822F0C00223
:1014780042EA8112C606DA607FF534AF1A6822F4B0
:1014880040721A601A6842EA07221A60DA6822F47F
:10149800407242EA01228506DA607FF526AF1A68B3
:1014A80022F440621A601A6842EA87221A60DA68EF
:1014B80022F4406242EA81224406DA607FF518AFDE
:1014C8001A6822F440521A601A6842EA07321A600F
:1014D800DA6822F4405242EA0132DA6002067FF505
:1014E8000AAF1A6822F440421A601A6842EA873240
:1014F8001A60DA6822F4404242EA8132C605DA60AC
:101508007FF5FCAE1A6822F440321A601A6842EA83
:1015180007421A60DA6822F4403242EA014285053D
:10152800DA607FF5EEAE1A6822F440221A601A6873
:1015380042EA87421A60DA6822F4402242EA81428B
:101548004405DA607FF5E0AE1A6822F440121A60AA
:101558001A6842EA07521A60DA6822F4401242EA2C
:101568000152DA6002057FF5D2AE1A6822F4400211
:101578001A601A6842EA87521A60DA6822F440024E
:1015880042EA8152C604DA607FF5C4AE1A6822F0D6
:1015980040721A601A6842EA07621A60DA6822F032
:1015A800407242EA01628504DA607FF5B6AE1A68D5
:1015B80022F040621A601A6842EA87621A60DA68A2
:1015C80022F0406242EA81624404DA607FF5A8AE04
:1015D8001A6822F040521A601A6842EA07721A60C2
:1015E800DA6822F0405242EA0172DA6098E610B5F1
:1015F8000409013C052C17D80C4B33F8142000F0D3
:101608000F0042FA00F313F001030DD0012303FA8F
:1016180000F0013810402BF0FDF9054A054B125D2A
:10162800104403EBC00010BD002010BDB420030817
:10163800C02003083C6E00202DE9F04F4A484B4B70
:101648004B4C4FF090414FF0010A4FF002094FF018
:1016580004084FF0080C4FF0100E20274026802574
:1016680030F8022B12F0010F03D01960A3F804A080
:10167800083312F0020F03D01960A3F8049008335E
:1016880012F0040F03D01960A3F80480083312F095
:10169800080F03D01960A3F804C0083312F0100F24
:1016A80003D01960A3F804E0083312F0200F02D029
:1016B80019609F80083312F0400F02D019609E8095
:1016C800083312F0800F02D019609D80083312F49D
:1016D800807F05D04FF4807B1960A3F804B00833ED
:1016E80012F4007F05D04FF4007B1960A3F804B012
:1016F800083312F4806F05D04FF4806B1960A3F89B
:1017080004B0083312F4006F05D04FF4006B196071
:10171800A3F804B0083312F4805F05D04FF4805B5F
:101728001960A3F804B0083312F4005F05D04FF431
:10173800005B1960A3F804B0083312F4804F05D099
:101748004FF4804B1960A3F804B00833D20B04D0CF
:101758004FF4004219609A80083301F58061A14274
:101768007FF47EAFBDE8F08FB42003083C6E002004
:1017780000180048002867D003682DE9F04F03F1EE
:1017880038445C4EA40A0125345D04F01F06640940
:10179800022C05FA06F558D0032C00F0A580012C80
:1017A80058D08088B0FA80F4C4F11F04A4B2E508C8
:1017B80003EB850504F007042E6AA4000F27A74051
:1017C80026EA07062E622E6A01F00307A2407C1E55
:1017D8003243012CC1F3810CC1F300182A62C1F312
:1017E80041113CD9C60700F18980850700F1958031
:1017F800440700F1A380020700F1B180C60600F19A
:10180800BF80850600F1CD80440600F1DB8002062A
:1018180000F1E980C60500F1F780850500F1058132
:10182800440500F11381020500F12181C60400F18D
:101838002F81850400F13D81440400F14B810204AD
:1018480000F15981BDE8F08F70472B4CA6693543EC
:10185800A561A6E7284C666935436561A1E70024C0
:1018680022464FF0010E4FF0030904E00132102A1E
:1018780004F10204E6D00EFA02F636EA0005F5D1C4
:10188800D3F808A009FA04F5ED430AEA050AC3F8F3
:1018980008A0D3F808B00CFA04FA4AEA0B0AC3F80D
:1018A80008A0B3F804A01FFA8AFA2AEA06069E805E
:1018B800B3F804A008FA02F646EA0A06B6B29E8011
:1018C8001E682E401E60D3F800A007FA04F646EA08
:1018D8000A061E60D3F80CA001FA04F605EA0A0A03
:1018E80046EA0A05DD60C1E7034CE6693543E56170
:1018F80057E700BFC41C0308001002401A6822F012
:1019080003021A601A683A431A60DA6822F003027E
:101918000A438507DA607FF56BAF1A6822F00C027C
:101928001A601A6842EA87021A60DA6822F00C0222
:1019380042EA81024407DA607FF55DAF1A6822F057
:1019480030021A601A6842EA07121A60DA6822F04E
:10195800300242EA0112DA6002077FF54FAF1A68D7
:1019680022F0C0021A601A6842EA87121A60DA681E
:1019780022F0C00242EA8112C606DA607FF541AF62
:101988001A6822F440721A601A6842EA07221A603A
:10199800DA6822F4407242EA01228506DA607FF5AD
:1019A80033AF1A6822F440621A601A6842EA872242
:1019B8001A60DA6822F4406242EA81224406DA6058
:1019C8007FF525AF1A6822F440521A601A6842EA75
:1019D80007321A60DA6822F4405242EA0132DA60C9
:1019E80002067FF517AF1A6822F440421A601A6897
:1019F80042EA87321A60DA6822F4404242EA8132C7
:101A0800C605DA607FF509AF1A6822F440321A6019
:101A18001A6842EA07421A60DA6822F4403242EA57
:101A280001428505DA607FF5FBAE1A6822F4402290
:101A38001A601A6842EA87421A60DA6822F4402279
:101A480042EA81424405DA607FF5EDAE1A6822F475
:101A580040121A601A6842EA07521A60DA6822F4D9
:101A6800401242EA0152DA6002057FF5DFAE1A68D9
:101A780022F440021A601A6842EA87521A60DA6849
:101A880022F4400242EA8152C604DA607FF5D1AE00
:101A98001A6822F040721A601A6842EA07621A60ED
:101AA800DA6822F0407242EA01628504DA607FF562
:101AB800C3AE1A6822F040621A601A6842EA876266
:101AC8001A60DA6822F0406242EA81624404DA600D
:101AD8007FF5B5AE1A6822F040521A601A6842EAD9
:101AE80007721A60DA6822F0405242EA0172DA603C
:101AF80002047FF5A7AE1A6822F040421A601A68FD
:101B080042EA87771F60DA6822F0404242EA817130
:101B1800D960BDE8F08F002852D0036803F138423D
:101B28002DE9F04F920A514DAA5C02F01F055209A7
:101B38000124022A04FA05F443D0032A00F0908015
:101B4800012A43D001F003077A1E012AC1F3810C50
:101B5800C1F300188088C1F341113CD9C60700F1D0
:101B68008980850700F19580440700F1A38002076A
:101B780000F1B180C60600F1BF80850600F1CD8076
:101B8800440600F1DB80020600F1E980C60500F199
:101B9800F780850500F10581440500F113810205F0
:101BA80000F12181C60400F12F81850400F13D81F7
:101BB800440400F14B81020400F15981BDE8F08F23
:101BC80070472B4A95692C439461BBE7284A5569AD
:101BD8002C435461B6E7002422464FF0010E4FF023
:101BE800030904E00132102A04F10204E6D00EFAD7
:101BF80002F636EA0005F5D1D3F808A009FA04F58B
:101C0800ED430AEA050AC3F808A0D3F808B00CFAAD
:101C180004FA4AEA0B0AC3F808A0B3F804A01FFAAA
:101C28008AFA2AEA06069E80B3F804A008FA02F6A1
:101C380046EA0A06B6B29E801E682E401E60D3F899
:101C480000A007FA04F646EA0A061E60D3F80CA0BC
:101C580001FA04F605EA0A0A46EA0A05DD60C1E760
:101C6800034AD5692C43D4616CE700BFC41C030840
:101C7800001002401A6822F003021A601A683A43F8
:101C88001A60DA6822F003020A438507DA607FF5F2
:101C98006BAF1A6822F00C021A601A6842EA8702CF
:101CA8001A60DA6822F00C0242EA81024407DA601C
:101CB8007FF55DAF1A6822F030021A601A6842EAAE
:101CC80007121A60DA6822F0300242EA0112DA607A
:101CD80002077FF54FAF1A6822F0C0021A601A682F
:101CE80042EA87121A60DA6822F0C00242EA8112D8
:101CF800C606DA607FF541AF1A6822F440721A60AE
:101D08001A6842EA07221A60DA6822F4407242EA44
:101D180001228506DA607FF533AF1A6822F4406243
:101D28001A601A6842EA87221A60DA6822F4406266
:101D380042EA81224406DA607FF525AF1A6822F468
:101D480040521A601A6842EA07321A60DA6822F4C6
:101D5800405242EA0132DA6002067FF517AF1A688C
:101D680022F440421A601A6842EA87321A60DA6836
:101D780022F4404242EA8132C605DA607FF509AFB3
:101D88001A6822F440321A601A6842EA07421A6056
:101D9800DA6822F4403242EA01428505DA607FF5CA
:101DA800FBAE1A6822F440221A601A6842EA874297
:101DB8001A60DA6822F4402242EA81424405DA6075
:101DC8007FF5EDAE1A6822F440121A601A6842EAEA
:101DD80007521A60DA6822F4401242EA0152DA60C5
:101DE80002057FF5DFAE1A6822F440021A601A680D
:101DF80042EA87521A60DA6822F4400242EA8152C3
:101E0800C604DA607FF5D1AE1A6822F040721A6013
:101E18001A6842EA07621A60DA6822F0407242EAF7
:101E280001628504DA607FF5C3AE1A6822F0406269
:101E38001A601A6842EA87621A60DA6822F0406219
:101E480042EA81624404DA607FF5B5AE1A6822F08E
:101E580040521A601A6842EA07721A60DA6822F079
:101E6800405242EA0172DA6002047FF5A7AE1A68AE
:101E780022F040421A601A6842EA87771F60DA68DF
:101E880022F0404242EA8171D960BDE8F08F70B516
:101E9800044690F85900002833D104F11405236E44
:101EA80080226B2128469847642004F073FB236E38
:101EB800284603226B219847236E94F85420192151
:101EC800284698470F2004F065FB236E94F85220AB
:101ED80028461A219847236E284618221B2198471E
:101EE800236E284618221C219847236E2846022272
:101EF800372198472846236E01223821BDE87040D3
:101F08001847FFF774FB0546D0B1202300218371E1
:101F1800C171FFF700FE21460F4B41F8103F2846DC
:101F280028F0BEFEAB88B3FA83F3C3F11F035A1C33
:101F3800B3D001229A4009490B6813430B60ACE700
:101F48000146FFF7E8FD2146034B41F8103F2846BC
:101F580028F0A6FE0122EEE77908000800040140F7
:101F680010B1036882881A85704710B103688288A7
:101F78009A61704738B100298388026814BF00212C
:101F880010218B409361704710B40A4B0A4A1C78A1
:101F980001238340234052F8200029B9B3FA83F182
:101FA80049095DF8044BE5E7191C18BF01215DF8E4
:101FB800044BDFE7A8610020AC61002030B1036862
:101FC80082881B8A1A4214BF0120002070470F49DB
:101FD80038B5D1F890330446ABB11846FFF7EEFF99
:101FE800024691F894030A4B40B9187881F8942373
:101FF80018B114B1002220461A7038BD002AF4D155
:1020080001251D70F2E7024B1878F1E77C230020C8
:10201800843100202DE9F041C44E044604F014FA3E
:1020280096F895330546092B3ED8DFE813F0B7003C
:102038008901CE010A002E023A02590241004C00E1
:102048007800D6F8A803FFF7B9FF68B3FB2028F09B
:1020580009FF10F07F0527D0294625442046FEF7C2
:1020680068FE15F9013C002B1EDAA378012B1BD161
:102078006079C8B9E278237986F859236FF00401AA
:1020880086F85A33091B621D04F10A0500E06079DD
:102098008B18034412F8010F3344954283F85C030C
:1020A800F5D1042386F8953300242046BDE8F08155
:1020B80008230020C6F8B05386F89533FFF787FF4A
:1020C800002840F01E82D6F8A803FFF777FF002803
:1020D80040F025820024D6F8B413D6F8B02342F293
:1020E800283303FB01F3AD1A9D42DEDD012900F020
:1020F8009D8296F8DA33D6F89C035A1CDB0786F8DB
:10210800DA2340F10982FFF72BFF0D20FEF732FE9C
:1021180034200FF0F1FB072386F89533C5E704F068
:1021280093F9D6F8BC3340F26352C01A9042BBD937
:1021380036200FF0E1FBFE213E200FF0C9FB3A20CC
:102148000FF0DAFBDFF8F48136200FF0D5FB3B20E7
:1021580096F8C4730FF0D0FBD8F82030B8F82420D4
:102168001A857F2028F022FEFF2F08D0704C0137F7
:10217800274414F8010B28F019FEBC42F9D1D8F80D
:102188002030B8F824209A6135200FF0B5FB0823D9
:10219800C6F8B05386F89533022486E7654BD6F81F
:1021A80098231B689B1A0A2B7FF67EAF30200FF00E
:1021B800A3FB22F02BFA8E2028F054FE01210220E6
:1021C800FEF7D6FD0C211720FEF7D2FD1821084690
:1021D800FEF7CEFD19210620FEF7CAFD05210820CD
:1021E800FEF7C6FDFF213E20FEF7C2FD08210B20A9
:1021F800FEF7BEFD00210C20FEF7BAFD5C210D2084
:10220800FEF7B6FD76210E20FEF7B2FD27210F203E
:10221800FEF7AEFDAA211020FEF7AAFD39211120F4
:10222800FEF7A6FD11211220FEF7A2FD232113209F
:10223800FEF79EFD7A211420FEF79AFD4221152013
:10224800FEF796FD16211920FEF792FD6C211A2043
:10225800FEF78EFD03211B20FEF78AFD40211C207E
:10226800FEF786FD91211D20FEF782FD56212120D3
:10227800FEF77EFD10212220FEF77AFDA9212320FA
:10228800FEF776FD0A212420FEF772FD00212520A5
:10229800FEF76EFD11212620FEF76AFD592129203F
:1022A800FEF766FD88212C20FEF762FD31212D20E6
:1022B800FEF75EFD0B212E20FEF75AFD07210320B5
:1022C800FEF756FD00210920FEF752FD36200FF0DB
:1022D80013FB04210720FEF74BFD00210C20FEF71D
:1022E80047FD154C002536200FF006FBE9B20A2001
:1022F800FEF73EFD33200FF0FFFA22F039F9A32054
:1023080028F0B0FD2070A42028F0ACFD6070A52056
:1023180028F0A8FD0135FF2DA07004F10304E2D1D7
:10232800012386F895330024BFE600BF7C230020F4
:10233800402700207C610020D42300203C6E002030
:102348000120FFF744FE20B996F85833002B00F01F
:10235800C080D6F89C03FFF708FE14211920FEF769
:1023680007FDCA4A82231946126886F8A4330C204E
:10237800C6F8A023FEF7FCFC0C210720FEF7F8FCAA
:1023880008211820FEF7F4FC36200FF0B5FA96F86D
:1023980058102320FEF7ECFC96F859102420FEF77D
:1023A800E7FC96F85A102520FEF7E2FC00210A20E7
:1023B800FEF7DEFC3A200FF09FFA34200FF09CFA6B
:1023C800022386F8953300246FE696F9A433AF4AC2
:1023D800D6F8A0137D2BC4BF822386F8A4331368D4
:1023E8005B1A322B00F21181D6F8A803FFF7E6FD3D
:1023F80000283FF459AEFB2028F034FD10F07F058B
:102408003FF452AE294625442046FEF792FC15F8C3
:10241800013C1A067FF548AEA578012D7FF444AE3D
:1024280003F07F03312B3FF63FAE96F8A43386F8CE
:102438005B3336200FF060FA96F858102320FEF729
:1024480097FC96F859102420FEF792FC96F85A103B
:102458002520FEF78DFC00210A20FEF789FC3A2092
:102468000FF04AFA142004F03BF834200FF044FA35
:1024780000240523284686F8AC3386F85540FEF735
:10248800BBFC032386F895330FE696F8AC33782B1C
:102498006FD936200FF030FA052386F895330024DB
:1024A80003E696F85833002B00F0BD802824D6F8B0
:1024B8009C03FFF75AFD322004F06CF8D6F89C0311
:1024C800FFF74EFD322004F065F8631E13F0FF0499
:1024D800EDD10623002486F895332046BDE8F08127
:1024E8002F23002086F85530FEF786FC07230120AD
:1024F80086F89533FEF73EFC34200FF0FDF90124F1
:10250800D3E500243223C6F8B043C6F8B84386F8AA
:102518009543C6F8B433C8E5FFF727FDF5E5FB207A
:1025280028F0A0FC00F07F0013287FF6D3AD14211B
:102538002046FEF7FEFB94F91330002BBFF6CAAD18
:10254800237800220121112BC6F8B823C6F8B4134A
:1025580076D0D6F8B02342F22833AD1A9D427FF7E1
:10256800A3AD012200240120C6F8B823FEF702FC1F
:10257800CEE5D6F8A803FFF721FD00283FF494AD77
:10258800FB2028F06FFC10F07F053FF48DAD294645
:1025980025442046FEF7CDFB15F9013C002BBFF67C
:1025A80083ADA378012B7FF47FADE27896F8593399
:1025B8009A427FF479AD227996F85A339A427FF499
:1025C80073AD637996F8AC239A4219467FF46CADE3
:1025D80004F1050C002204E0052A87F85CE350D0DA
:1025E80063791CF801EF15F8038CB718F045D0B2E1
:1025F8001F4402F1010202D0BEF1000FECD12C29D8
:10260800EAD9034486F8553043E796F8A4331268AC
:10261800C6F8A0230533DBB219460C2086F8A4338C
:10262800FEF7A6FBE0E602F0FDFE52E7D6F8B83367
:10263800642B03F1010296D93223C6F8B43392E72A
:10264800627896F859339A4283D1A27896F85A3329
:102658009A427FF47EAFD6F89C03FFF786FC0846C3
:10266800FEF788FBE37803F00303022B10D0342035
:102678000FF042F9072386F89533C6F8B0530224C1
:1026880029E5053186F8AC1300240EE57C610020AD
:1026980003F0DAFEA37CC6F8BC0313F0800F03EB4B
:1026A800C3034FEA231314BF523B41331BB2D80074
:1026B8000A2290FBF2F06428A8BF642020EAE070A8
:1026C800C0B2A6F8C0332AF065FB2A4A2A4B517CCF
:1026D800107B96F8597333F8102033F8113096F8B8
:1026E800D803217996F85A4386F8C573C3F30B13B8
:1026F800884286F8C833B6F8C03386F8C933C2F3BF
:102708000B120EBF737896F8D933737086F8C72307
:1027180008BF86F8D93311224B1C03F01F0386F833
:10272800C42386F8C64372783478144F86F8D833B1
:1027380086F8C213002302F10108944206EB020C4A
:1027480007EB030ED8B208F03F0203F1010308D0EB
:102758009CF804008EF808000A2BECD17270184619
:1027680000E07470092386F8CA0386F8CB1386F84C
:10277800953382E784610020A06100204027002073
:102788002DE9F0410B4E346873691C400FD0DFF817
:1027980028800127B4FA84F3C3F11F0307FA03F56D
:1027A80058F8230003689847AC437561F2D1BDE837
:1027B800F08100BF00040140C46D00202DE9F04104
:1027C8000B4E346873691C400FD0DFF8288001274E
:1027D800B4FA84F3C3F11F0307FA03F558F823008A
:1027E80003689847AC437561F2D1BDE8F08100BF3A
:1027F80000040140C46D00202DE9F0410B4E3468FF
:1028080073691C400FD0DFF828800127B4FA84F3DD
:10281800C3F11F0307FA03F558F823000368984724
:10282800AC437561F2D1BDE8F08100BF00040140FE
:10283800C46D00202DE9F0410B4E346873691C40CB
:102848000FD0DFF828800127B4FA84F3C3F11F03FF
:1028580007FA03F558F8230003689847AC437561F5
:10286800F2D1BDE8F08100BF00040140C46D002032
:102878002DE9F0410B4E346873691C400FD0DFF826
:1028880028800127B4FA84F3C3F11F0307FA03F57C
:1028980058F8230003689847AC437561F2D1BDE846
:1028A800F08100BF00040140C46D00202DE9F04113
:1028B8000B4E346873691C400FD0DFF8288001275D
:1028C800B4FA84F3C3F11F0307FA03F558F8230099
:1028D80003689847AC437561F2D1BDE8F08100BF49
:1028E80000040140C46D00202DE9F0410B4E34680E
:1028F80073691C400FD0DFF828800127B4FA84F3ED
:10290800C3F11F0307FA03F558F823000368984733
:10291800AC437561F2D1BDE8F08100BF000401400D
:10292800C46D0020084A094808B5936943F00103BB
:102938009361002140222CF014FE054B4FF0FF322A
:102948001A60C3F8032008BD00100240C46D0020BF
:10295800046E00202DE9F041044618460D4616463F
:10296800984629F03DFB2768E6722844A07229465C
:102978007D69434632462046AC46BDE8F041604793
:10298800036810B504461B689847236820469B686F
:102998009847A37B0133A37310BD10B503680446A1
:1029A8009B689847FF2301226373227310BDF8B513
:1029B80005015B4C5B4B625961199A4204EB0507B0
:1029C80004BF01230B730646387A21F06DFE3B7A6B
:1029D80003F01F015B090122022B02FA01F278D0F1
:1029E800032B71D0012B67D0631901361879FEF7D4
:1029F800FEFDF6B2074610B11223C6718371631942
:102A08005879FEF7F4FD10B11323C6718371631969
:102A18009879FEF7ECFD10B11423C671837166191D
:102A28000E21F2793846FEF7A5FE7079FEF7DFFD34
:102A3800F2790E21FEF79EFEB079FEF7D8FDF27905
:102A48000E21FEF797FE6359364A934251D0364A13
:102A5800934259D0354A934240D02C44227B002AD5
:102A68002FD1012002249A8822F480521204120CD9
:102A78009A80998889B241F4805199801A8802F421
:102A8800415242F44572024322431A809A8822F442
:102A980070621204120C42F4E0629A809A8B22F45B
:102AA80000621204120C07219A8319821A8892B2C2
:102AB80042F040021A80F8BD1D4B996A0A439A6297
:102AC80092E700200446CEE7194B19690A431A61B8
:102AD8008AE7174BD9680A43DA6085E702F5EA32D4
:102AE800116941F400411161116921F4004111613A
:102AF800B3E702F56042D16841F48051D160D168F2
:102B080021F48051D160A8E702F5EC32116941F453
:102B180080411161116921F4804111619DE700BF75
:102B28000C6E00200030014000380040003C00409E
:102B380000100240427A02B9704710B50446036893
:102B4800406804F10A0198470023637210BD437A74
:102B58005A1C0344D2B242729972037A934200D843
:102B680002B9704710B504460368406804F10A01C9
:102B780098470023637210BD10B40B49002301E08D
:102B8800272B0CD011F8132082424FEA430403F19B
:102B98000103F5D121445DF8044B487870470020C3
:102BA8005DF8044B704700BFD4F6020870B544883E
:102BB80006460D46C4F30B042246002128462CF095
:102BC800D0FC3369094A934209D3094A934206D291
:102BD800224628461946BDE870402AF0F9B923B1C3
:102BE80021462846BDE87040184770BDA860030814
:102BF800BE610308064B07498B4202D300231846DF
:102C080070471A88C2F30B029042F8D01433F3E7E6
:102C1800485C0308A8600308024A136823EA000016
:102C28001060704744340020F8B5174D2B78A42B5A
:102C380028D16B78BE2B25D1022229464FF6FF708A
:102C4800FDF70AFC114FAC1C22884AB1A618BE42F7
:102C580018D2052A16D92146FDF7FEFB3446F3E7BC
:102C680021460222FDF7F8FB0222A118FDF7F4FB2A
:102C78000634074B641B1C8041F60F53C31A584295
:102C88005841F8BD0020F8BD00F003080000040812
:102C98009A4100202DE9F04FDFF848914C4F8BB056
:102CA8000326A7EB09071822002104A82CF059FCD9
:102CB800484BCDF8109005971A69120604D5464A74
:102CC8005A6002F188325A6001228DF82420342299
:102CD800DA60424B424C1B88ADF80030022269464C
:102CE80004A8FEF70DF8022269464FF6FF70FDF7BB
:102CF800B3FBDFF8F4A080464FF0000B544536D301
:102D08000AAC002524F8245D0222214604A8FDF718
:102D1800F7FF022221464046FDF79EFB40BAC0431A
:102D2800ADF80800022202A904A8FDF7E9FF0798F8
:102D380060B106ABC0F10402294618442CF011FC1E
:102D4800069904A8FDF783FF079508909DF824309D
:102D5800089A23B11F490B6943F080030B61013EB8
:102D68002DD0002A9FD1FFF75FFF50B32CE0658874
:102D78008DF80DB0C5F30B05AB1DADF808302388F1
:102D8800C3F30B02ADF80A201B0B062202A904A804
:102D98008DF80C30FDF7B4FF062202A94046FDF776
:102DA8005BFB616880462A4604A8FDF7A9FF6168B5
:102DB80040462A46FDF750FB143480469EE7002A19
:102DC800D1D0052002F038FB0BB0BDE8F08F00BF72
:102DD80000000408002002402301674522F702088A
:102DE800485C030800F00308A86003080378202B58
:102DF800024600F10100F9D0092BF7D02D2B2CD079
:102E08002B2B03BF5378B7EE000A0246B7EE000A31
:102E1800A3F13001C8B209289FED467A10D8F2EE26
:102E2800046A07EE901AF8EEE77A12F8013FE7EE27
:102E3800267AA3F13001C8B20928B0EE677AF0D932
:102E48002E2B4CD003F0DF03452B0BD0F7EE007A86
:102E580067EE276A20EE260A70475378BFEE000A0D
:102E68000246D5E710B451782D2959D02B290ABF2D
:102E78009178501C901C0024A1F13003092B53D8E1
:102E8800002303EB830301EB430310F8011FA1F1B7
:102E98003002092AA3F13003F3D9B3F59A7F28BF8A
:102EA8004FF49A73072B42D9DFED236A1A46F7EEDF
:102EB800007A083A072A67EEA67AFAD803F00703D9
:102EC8002BB1F2EE046A013B67EEA67AFBD124B37C
:102ED800C7EE276A5DF8044B20EE260A7047537840
:102EE800A3F13001C8B2092802F10102AAD8F2EE12
:102EF800046AF0EE665A07EE901AF8EEE77A12F8CE
:102F0800013F87EEA66AA3F13001C8B2092866EE30
:102F1800A56A37EE067AEED994E767EE276AD9E70D
:102F2800901C91780124A7E7F7EE007ACFE7F7EE37
:102F3800007AC5E70000000020BCBE4CB5EEC00A10
:102F4800DFED317AF1EE10FACCBF30EE270A30EE21
:102F5800670ADFED2E7A20EE270A30B5FDEEC07A3B
:102F680087B017EE904A054684EAE470002303A967
:102F7800A0EBE47001930093029319F007FC002C76
:102F8800ACBF20232D2303A88DF8003029F028F8A2
:102F9800012803A924D002282DD0032805BF3023F7
:102FA800684668468DF801302CF001FB684629F028
:102FB80017F80338C4B22246694628462CF055FB58
:102FC80000232B55284629F00BF82E22431C2A549F
:102FD8000DEB0401E8182CF007FB284607B030BDBC
:102FE800302368468DF801308DF802308DF80330B3
:102FF8002CF0DDFADAE7302368468DF801308DF8D9
:1030080002302CF0D4FAD1E76F12033A00007A4468
:103018002DE9F041064615460846B6FBF2F43CB9E0
:1030280005FB1464124B1B5D00F8013BBDE8F08101
:10303800B4FBF2F767B90E4B05FB174705FB1464A1
:10304800DA5D00F8012B1B5D00F8013BBDE8F0815B
:10305800B7FBF2F8B8F1000F02D04046FFF7D8FFEF
:1030680005FB1878024B13F8082000F8012BE3E75A
:10307800E820030830B402681146531C036011F8B5
:10308800024B0160D31C517803609378151D0560CD
:103098001B0443EA0123D078234343EA006030BC91
:1030A80070470368591C1A46016012F8021B026037
:1030B800587841EA0020704703685A1C0260187863
:1030C800704738B504460068154629F081FF226824
:1030D8002A44226038BD036810B40A0A5C1C0460E4
:1030E8001A7003685A1C026019705DF8044B704727
:1030F80003685A1C026010B4197003680A0A5C1C41
:1031080004601A7003680A0C5C1C04601A70036877
:10311800090E5A1C026019705DF8044B7047036869
:103128005A1C026019700368090A5A1C0260197057
:1031380070472DE9F047002488B080460F461E46A8
:10314800A14605AD531C0393117839B3252933D112
:10315800931CCDF810900393507830284ED04FF040
:10316800000AA0F13003DBB2092B42D96C2819D030
:10317800642800F0938024D825281CD063D95828C7
:1031880076D063281BD131784046B847039A531C40
:1031980003931178043601340029D7D1204608B0AA
:1031A800BDE8F087039B5A1C03921B78642B7CD0E4
:1031B8002AD8252B54D1252140460134B847039AF3
:1031C800C0E7732833D044D975284FD106F1040ECF
:1031D80030682B4600220A217646FDF739F8049A12
:1031E8000095534639464046FDF76FF8039A044464
:1031F800A8E704AA03A928F03FF9B7E7D31C03936B
:1032080090784FF0010AACE7732B10D05BD9752B7F
:103218003AD0782B96D1A3F15802B2FA82F23068EC
:1032280052092B4610210436FDF712F8D7E7336808
:10323800049A0093394600234046FDF746F80436C1
:103248000444039A7EE70028B9D1204608B0BDE8B7
:10325800F0876E28B3D1039A336804361C6071E78F
:103268002AD9582BD7D0632B8DD06BE77828A6D1D5
:10327800A0F15802B2FA82F2306852092B461021A6
:10328800FCF7E6FF0436AAE706F1040E30682B4681
:1032980000220A217646FCF7DBFFA0E7331D3068E1
:1032A80029461E46FCF7A7FF99E7331D30682946D3
:1032B8001E46FCF7A0FF92E7002B7FF443AF2046A1
:1032C80008B0BDE8F0876E2BC6D03BE70EB400B55A
:1032D80084B005AB019053F8042B0649039301A869
:1032E800FFF727FF019B00221A7004B05DF804EB7A
:1032F80003B07047C90200080FB430B583B006ABFD
:103308000A490B4853F8042B096800680193FFF732
:1033180010FF084C05462068FDF7C6FD0028FAD0C6
:10332800284603B0BDE8304004B070475C2E00204A
:10333800602E002034660020DFED2B7AB4EEE70A19
:10334800F1EE10FA4ADDDFED296A9FED297A01E0F6
:10335800B0EE670AB4EEC70AF1EE10FA70EE667ABC
:10336800F6DC9FED247AF4EEC77AF1EE10FA38D540
:10337800DFED1E6A9FED207A01E0F0EE407AF4EE70
:10338800C77AF1EE10FA37EEA60AF6D4DFED1B7A0B
:10339800B4EEE70AF1EE10FA14DDDFED137A37EE3A
:1033A800C00A60EE006A9FED166A9FED167ADFED9F
:1033B800167AA6EE867A20EE266AE6EE877AA6EEDA
:1033C800270A7047DFED117AB4EEE70AF1EE10FA3A
:1033D80044BFDFED087A37EEC00AE2E7F0EE407A44
:1033E800BFE7B0EE670AD1E7DB0F4940DB0FC94002
:1033F800E4CB1641DB0F49C0E4CB16C1DB0FC93F54
:1034080092E741B99730083C15A82ABEDB0FC9BF1F
:1034180080EAE073A3EBE0738B4205DB002801DD53
:10342800401A704702D1704700207047084470471F
:1034380009B909E0194690FBF1F301FB13030846AB
:10344800002BF7D1084670470146FBE710B507EE99
:10345800901A2DED028BB8EE678ADFED217A28EEFF
:10346800008A044628EE278AB0EE480A2AF004F8B3
:10347800F0EE408AB0EE480A29F060FFF7EE007AD5
:103488009FED187AF0EE675AE8EE875A0023A36199
:10349800B0EE676AC7EEA56A63612362E361A8EECE
:1034A800C76ABDEC028B77EEC07AB6EE007AF8EE0A
:1034B800005A27EE877A20EE250A27EE267A26EE8E
:1034C800266A67EEA67A20EE260A84ED046AC4ED21
:1034D800017A84ED007A84ED027A84ED030A10BD46
:1034E80027D4D236F304353F10B44C09012250F8E2
:1034F800243001F01F0102FA01F10B4340F8243097
:103508005DF8044B70474B0901F01F0150F8232068
:10351800012303FA01F1114214BF18460020704735
:103528002DE9F041754B1B78012B00F0D980744BC5
:10353800822703F1EA0628215A22782555242D20CE
:103548001F7059709A70DD7019715A719C71D87119
:103558004E33B342F4D16B4B6B4A598918889C8A15
:10356800B3F816E05E8B1F8BDD8DB3F804C021F431
:1035780000614FF0FA0820F40060598140F66111AB
:1035880024F400642EF4006EA3F85680188040F6E8
:103598002B08598203CA26F40066A3F810809C827F
:1035A80040F698181C8EA3F816E0DFF878E1574A21
:1035B800A3F8028027F4006725F4006540F6811817
:1035C8005E83534ECEF80000CEF804102CF4006C45
:1035D8000021A3F80C8024F4006440F6CC181F8363
:1035E800DD851C274FF40065212057709070A3F8E3
:1035F8000E80A3F804C01D81DD8031701C86DF8F2A
:10360800B3F84460DD8B1C8C588C9A8CB3F81C8002
:10361800B3F83CC0B3F832E027F4006726F400663C
:1036280025F4006524F4006420F4006022F40062AC
:10363800DF87A3F84460DF8C1E8DDD831C849D8D9D
:103648009C8E58849A84D88E1A8F27F4006726F4A3
:10365800006625F4006524F4006420F4006022F478
:103668000062DF841E8540F6691740F68A1628F442
:1036780000682CF4006C2EF4006E5F859D859C8696
:10368800D8861A87A3F81C80A3F83CC0A3F832E0B8
:103698005E87B3F84060B3F84250B3F846401D4A1D
:1036A800B3F84800517026F4006625F4006524F448
:1036B80000640127A3F84060A3F8425003261D25A3
:1036C800A3F84640302420F40060917051711770BF
:1036D80016719571D470D471A3F84800BDE8F081D3
:1036E8000D4A0E480E494FF4486640F22E45022412
:1036F8001680158284700B7019E700BFC441002042
:10370800163300203446002010210308A04600206C
:10371800D0670020584B0020304C0020C86800209B
:103728000C4B0020386000202DE9F041204D214C41
:1037380000264FF02608A5F1800785F80680EE716F
:1037480031462846C4F8A853FEF7E5F905F1880381
:103758000522184687F80E21803587F80F61C4F8CE
:103768009C3320F0BFFF2846202187F8068187F880
:103778000761C4F89053FDF784FD2846FEF71EFC48
:103788000D4A0E490E4B17680E4D0F4A84F89403E4
:1037980084F895633220C4F8B063C4F8B863C4F8F9
:1037A8009873C4F8B4030D601A60BDE8F08100BFD7
:1037B800BC6E00207C2300207C61002000290020B2
:1037C8002458002093040008A104000808230B7063
:1037D800AAE72DE9F84FDFF8B4A0DFF8B490DFF8D6
:1037E800B480274E012304208AF8003027F0B8FA65
:1037F800D9F80000FEF7B4FB052027F005FB0020F0
:1038080027F002FB062027F0FFFA002027F0FCFA39
:1038180098F80040042044F0010427F0F5FA204607
:1038280027F0F2FA33888BB1164D174F002415F89C
:1038380004B0072027F0E8FA584627F0E5FA2A5D91
:1038480033883A550134A4B2A342F0D8072027F0B0
:10385800DBFAFF2027F0D8FA98F80040042027F078
:10386800D3FA204627F0D0FAD9F80000FEF77DFBFE
:10387800022027F075FA00238AF80030BDE8F88F97
:1038880020070020C8380020F03A0020DA3A00204B
:10389800C8670020E13A00202DE9F0414A4E042093
:1038A80027F05EFA3068FEF75BFB484B1B78012B6C
:1038B8007BD062D3022B0AD1DFF83081082388F845
:1038C80000300D254FF4C373414F3B8010E0DFF803
:1038D8001C813F4F98F8003003F04003002B14BFC1
:1038E8004FF4F0734FF4C3733B8014BF10250D25BC
:1038F800002404F11000C0B227F086FA0134012038
:1039080027F082FAA3B2AB42F3D398F80040314DC6
:10391800002027F079FA204627F076FA2E4B1C78FB
:10392800022027F071FA204627F06EFA2B4B1C78FC
:10393800032027F069FA204627F066FA284B1C78FE
:103948000420044327F060FA204627F05DFA306827
:10395800FEF70BFB022027F003FA3A8821480021E2
:103968002BF0FFFD2B7833B11F4B1B7833B30023AB
:103978002B70BDE8F081BDE8F081A02027F044FA63
:10398800002027F041FA00F00603022BDFF85C80E4
:1039980007D000F00500012803D1482388F800303B
:1039A80008E0082388F800308BE7DFF840804823D8
:1039B80088F8003010254FF4F07385E7FFF709FF0A
:1039C80000232B70BDE8F081C8670020CC67002079
:1039D8002007002000000020D3670020D4670020C3
:1039E800E13A0020F03A0020DA3A002024070020CB
:1039F800B0F1FF3F0AD0022810B403DC5DF8044B95
:103A0800FCF7E4BF00205DF8044B704700207047C6
:103A18000378012B00D07047417990F904003123D5
:103A2800F422E5E7F0B55B4B5B4A97B01968914221
:103A380000AF00F0A3805949594A00234FF47000A1
:103A4800C1F888003B607B60136843F480331360DF
:103A580003E03B68B3F5A04F09D0136803F40033C3
:103A68007B603B6801333B607B68002BF1D04C4B9B
:103A78001B6813F4003318BF01237B607B68012B9C
:103A880052D0464C464B474AE260474A596A116051
:103A98005A6A42F080725A625A6942F4FC025A61C8
:103AA8000025032207F10801012341F6FF764FF0B4
:103AB8009040FD60BE603A73BB7325F09FF94FF6E6
:103AC800FF7307F108013948BB6025F097F907F142
:103AD80008013748374E25F091F907F108013648B3
:103AE80025F08CF907F10801344825F087F907F12A
:103AF8000801334825F082F907F1080024F034FF63
:103B0800BB683049304AA1FB031330499B0CF020B5
:103B18004FF0070E5C370B60566084F82300956001
:103B2800C2F800E0BD46F0BD294A1D4B12211160C4
:103B38005A685A605A685A605A6842F480625A60F1
:103B48005A6822F47C125A605A6842F4E8125A60A1
:103B58001A6842F080721A601A689201FCD5596896
:103B68000F4A21F003015960596841F00201596078
:103B7800536803F00C03082BFAD182E700221A607D
:103B880062B6144B1B6883F30888134B1B6898476D
:103B9800FEE700BFFC9F0020EFBEADDE00ED00E0B9
:103BA800001002400005FA05A84F00200004004854
:103BB800000800483F190100000C004800100048A8
:103BC8000014004883DE1B4310E000E08061002001
:103BD8000020024000D8FF1F04D8FF1F70B50F4C0B
:103BE8000F4DC0EBC00004EB8004686926693043C0
:103BF800686182B09209667BA1600025012101A855
:103C080063618DF804608DF805208DF806508DF8F5
:103C1800071024F09DFD02B070BD00BF1C0C0020F1
:103C280000100240074BC0EBC00030B403EB80002B
:103C3800054C056963692B4363610176427630BCA4
:103C4800704700BF1C0C0020001002402DE9F04F07
:103C58005E4C54F8204083B0002C71D0666D9846B5
:103C680091465B4B7268E264A160236004F15A01DB
:103C78004FF4807304F5AD726161A261E360236162
:103C88000746307E20F010FDF068A8B1514B0021A6
:103C98005A68904203F11C0300F0928001310C290C
:103CA800F6D100207A1CD2B20C21FFF7BBFFE36CDF
:103CB800F26822632433A364B068D8B1454B00216D
:103CC8005A68904203F11C0378D001310C29F7D1CE
:103CD80000257A1CD2B20B212846FFF7A3FF234602
:103CE800F27E3D492846FFF779FFE36CB2686263CC
:103CF8002833636494F85900FDF779FC054694F875
:103D08005800FDF774FC18F0080F824696F819B0B1
:103D18001AD0CDB118F0110F4FF00B0307F10107BE
:103D280014BF4E213E21EF715A46AB712846FDF76C
:103D380021FD18F0010F45D0236B5BB3636B4BB3C8
:103D4800204603B0BDE8F08F18F0010F0CBF4FF00C
:103D58002E084FF04E0819F0020F09D045B10B227A
:103D68007B1CAA71EB7128465A464146FDF702FDB5
:103D780019F0010FE0D0BAF1000FDDD001370C23A4
:103D88008AF807705A4641468AF806305046FDF7C9
:103D9800F1FCD1E7337FB27E8DF804209B09002126
:103DA800012201A88DF805308DF806108DF807203E
:103DB80024F0CEFC204603B0BDE8F08FCDB288E7F2
:103DC800C8B26FE72846FEF7CBF8B5E7C430002045
:103DD80024F702081C0C0020490E00080348D0F8FC
:103DE8003C3113B100F59A70184770471C0C00203D
:103DF8000348D0F8203113B100F58C70184770478C
:103E08001C0C00200348D0F804310BB1FC301847D3
:103E1800704700BF1C0C00200348D0F8E8300BB1F5
:103E2800E0301847704700BF1C0C00200348D0F84A
:103E3800CC300BB1C4301847704700BF1C0C0020B1
:103E48000348D0F8B0300BB1A8301847704700BF0E
:103E58001C0C00200348D0F894300BB18C30184764
:103E6800704700BF1C0C00200248836F0BB17030F4
:103E7800184770471C0C00200248C36D0BB1543022
:103E8800184770471C0C00200248036C0BB13830EF
:103E9800184770471C0C00200248436A0BB11C30BD
:103EA800184770471C0C00200248836803B1184764
:103EB800704700BF1C0C0020F0B53E4C059D00EB80
:103EC800800004EB80046468002C71D03A4E4900ED
:103ED8004FF42040CFB23065A169090454D460681A
:103EE800DFF8E0E047F4903100EA0E0001434FF4B8
:103EF80020406160306503E0411E002848D0084634
:103F0800A1698907F8D54FF42040A262306503E023
:103F1800421E00283CD01046A2695206F8D5274A0E
:103F28006168DFF8A0E0306542EA0342174301EA1E
:103F38000E0217436760C3B1013BDBB201332B4468
:103F4800A0694FF4204210F0040002F1FF3207D1BB
:103F5800511C26D0A06910F0040002F1FF32F7D0FE
:103F6800626A05F8012B9D42EAD14FF42040306582
:103F780002E0431E60B11846A3699B06F9D52023C9
:103F88003065E3610120F0BD411E08B10846A3E792
:103F98000B4A138801339BB24FF0FF311380316510
:103FA800F0BD074932650B8801339BB20B80F0BD29
:103FB8002046F0BDE43000207C23002000240002CD
:103FC80098410020009800FC70B590F904506C1CD2
:103FD80082B00AD0022D08DC16460A4641790096BE
:103FE8002846FFF769FF02B070BD002002B070BD1F
:103FF80070B50378012B82B004D106236A46F721F5
:10400800FFF7E2FF9DF801209DF804309DF800605D
:104018009DF803509DF802409DF8050007491201DC
:104028001B0142EA063243EA053342EA141243EA24
:104038001013CA648B6402B070BD00BF7C230020DB
:1040480000B583B0002000920A466821FFF734FFCC
:1040580003B05DF804FB421C76D0022874DC2DE91D
:10406800F843142303FB00F33C4FFA583B44002A5F
:104078006BD01C1D94E810030546907B20F014FBC0
:10408800374B9C4263D0374A136B23F010031363FA
:104098001023344A116B6E1C0B431363F6B2B8F14C
:1040A800000F04D0152388F8076088F80630142319
:1040B80003FB057340465B7C002B14BF3E211E2189
:1040C8000422FDF757FBB9F1000F04D0162389F835
:1040D800076089F80630142000FB057504226B7C04
:1040E800002B14BF3E211E214846FDF743FB2168E3
:1040F8002D7C1D4B1D481E4A21F0010121602168BD
:10410800002D08BF03460A4022602361226800236D
:1041180042F001022260A360E360A360A36843F455
:104128000043A36023682360636823F0784323F483
:1041380000436360236823F400332360236843F05B
:1041480001032360BDE8F8837047BDE8F88305499B
:10415800084B0A6B22F020020A639AE7E430002039
:104168000058004000100240300E50007A25E00050
:10417800FFE0CF00200000101749184B184A1948D3
:1041880010B4D1F8884044F47004C1F888401C6821
:1041980044F001041C605C6822405A601A6822F0EE
:1041A800847222F480321A601A6822F480221A601B
:1041B8005A6822F4FE025A60DA6A22F00F02DA62C2
:1041C8001A6B002410404FF0006218639C608A60EC
:1041D8005DF8044B704700BF00ED00E0001002409E
:1041E8000CC07FF8CCFC00FF38B50B4C23688BB1B2
:1041F8005A68821A002A054604DA0CE05A68AA1A94
:10420800002A07DB9A68226018461A6890472368D4
:10421800002BF3D138BD38BD905D00200D4B012136
:104228000022890710B4027203F1640402D51979D7
:10423800815401329C4203F1140308D0072A06DC9A
:1042480099798907F3D49C4203F11403F6D15DF8F8
:10425800044B7047CC1C030824230370704700BF2D
:104268000122102302704370704700BF436A8269BD
:10427800D154436A0169426B01338B4228BF002342
:104288004362002A2FD0EFF31181502383F3128861
:10429800436B1A68D2072CD470B45E686EB9456A4D
:1042A800826A954217D084691444DC600ED9AA1A30
:1042B8005A608562002280F850201A6842F0010294
:1042C800C9B21A6081F3118870BC70470469A21AD8
:1042D8005A608662EEE7012380F85030C9B281F354
:1042E800118870BC7047C26C136843F08003136078
:1042F8007047C9B281F31188704700BF026B10B4D0
:1043080062B1036CC2684469D11A013B615C5DF813
:10431800044B08BF13460364C8B27047016A436977
:10432800C4685B5C0131A14228BF114601625DF897
:10433800044BD8B2704700BF436B13B190F85000DC
:104348007047836A406A181AB0FA80F040097047CB
:10435800416A836A99420AD3CB1A416B026961B1F7
:104368004968501E0B4483420AD2C01A704702693A
:104378001144CB1A416B0029F2D1501EC01A704764
:1043880000207047036B43B1026C5B6893422FBFF8
:10439800981AC0689B1AC0187047C269036A9A4283
:1043A8002FBFD01AC0688018C01A704708B514F01B
:1043B8002FFB024B024ADA60FEE700BF00ED00E087
:1043C8000400FA052DE9F0470569C3681D4028D0A7
:1043D8000F4606464FF000484FF00009B5FA85F33E
:1043E80028FA03F2D2431B3B32611540042B16D83E
:1043F800DFE803F03129211903007B6A002B32D052
:1044080003F1FF3A1FFA8AFAC7F824903C6A34B1DC
:1044180023682046514698476468002CF8D1002D3F
:10442800DCD1BDE8F0873868716B036889B29847BA
:10443800002DD3D1F5E77868B16B036889B2984746
:10444800002DCBD1EDE7B868F16B036889B29847C6
:10445800002DC3D1E5E7F868316C036889B2984745
:10446800002DBBD1DDE7F36A1FFA83FACEE700BF60
:104478002DE9F04F2DED028BA0F10A0389B00C460F
:10448800E72B00F24D86DFE813F01C014B064B06C4
:104498004B064B064B064B064B064B064B064B068C
:1044A8004B064B064B064B064B064B064B064B067C
:1044B8004B064B064B064B064B0663054B064B0655
:1044C8004B0627054B064B064B0644064B06B00524
:1044D8004B0697054B068B054B0682054B061E06B9
:1044E8004B0604064B064B064B06FD05F5054B0629
:1044F80034034B064B062D034B0605034B064B06B0
:104508004B06F2024B064B064B064B06D3024B06F4
:10451800FC004B062D0465014B064B064B064B066B
:104528004B064B064B062D014B06FF034B06CB03F0
:104538004B0655034B0641034B064B064B064B06F1
:104548000405C904C2049104E8004B064B0657024F
:104558002D024B06F601DA014B064B064B064B06BD
:10456800CF014B064B06AE014B064B064B069F018F
:104578008801BF027D024B064B064B066E024B06B6
:104588004B0671044B064B064B064B064B064B0677
:104598004B064B064B064B064B064B064B064B068B
:1045A8004B0604054B064B064B064B064B064B06C3
:1045B8004B064B064B064B064B064B064B064B066B
:1045C8004B064B064B064B064B064B064B064B065B
:1045D8004B064B064B064B064B064B064B064B064B
:1045E8004B064B064B064B064B064B064B064B063B
:1045F8004B064B064B064B064B064B064B064B062B
:104608004B064B064B064B064B064B064B064B061A
:104618004B064B064B064B064B064B064B064B060A
:104628004B064B064B064B064B064B064B064B06FA
:104638004B064B064B064B064B064B064B064B06EA
:104648004B064B064B064B064B064B064B064B06DA
:104658004B064B064B0666043C04A84E337853B110
:10466800A74F002537F8021F2046FEF758FD33787C
:104678000135AB42F6DC012009B0BDEC028BBDE888
:10468800F08F9E4E3378002BF5D09E4F0025B8460C
:10469800236817F81520591C21601A7098F8011022
:1046A80001EB810101EB810101F2EE2189B2204683
:1046B800FEF735FD33780135AB4208F10208E7DC37
:1046C800D9E7914D284627F08BFC0028D3DD2B46EF
:1046D8000544226813F8011B501C9D42206011708C
:1046E800F7D1C8E70FF0FCFEFF28054600F0048666
:1046F80008A9002601F8116D0DF10E008DF80E6065
:104708000FF0CEFE08A800F8106D0FF0BDFE08A847
:1047180000F8086D0FF0ACFE23685A1C22601D706B
:1047280023689DF80E20591C21601A7023689DF893
:104738000F20591C21601A7023689DF81020591CFD
:1047480021601A7023689DF81820591C21600120E7
:104758001A7091E70B686D4E01255A1C0A601D708E
:104768000B68B278591921601A7015F047FF236851
:10477800674A68495F1927601870B1F90010B2F9E3
:104788000000FEF755FE23685A1922601870318818
:104798002046FEF7C4FC28466EE70A685E4B5F4970
:1047A8001878551C2560107022685878551C2560AB
:1047B800107022689B78501C206013702046C988AE
:1047C800FEF7ADFC012057E7544D08462988FEF74F
:1047D800A6FC69882046FEF7A2FC2046A988FEF7B9
:1047E8009EFC012048E74E4D05F16006A988204649
:1047F800FEF795FCE9882046FEF791FC29892046BA
:10480800FEF78DFC2368AA7A591C21601A70236868
:10481800EA7A591C21601A7055F80C1B2046FEF7DD
:1048280067FCAE42E2D126E73E4952232268501C7B
:104838002060137011F8013F002BF7D11BE73A48AD
:1048480000232268056803EB4301561C6D5C266053
:104858001570026825680A446E1C527826602A7012
:10486800026825680A4401339278691C0A2B216082
:104878002A70E6D1FFE62D4D0B682A68591C12787C
:1048880021601A702B6822689978531C23600023D2
:1048980011702A6821681A4401335279481C032B85
:1048A80020600A70F5D123682A68591C127A2160A1
:1048B8001A7023682A68591CD27821601A702368F4
:1048C8002A68591C127921601A702B682046598968
:1048D800FEF725FC2A682368527A591C21601A7051
:1048E8002A680CE1124B08461968FEF701FC114BC7
:1048F80020461988FEF713FC0120BDE68C370020FE
:10490800CE5400201066002038600020B0460020F9
:104918008C4900208E490020104B002020450020A3
:10492800C84100204CF7020850600020E85E0020D3
:10493800BC46002060600020A84D08462988FEF784
:10494800EEFB69882046FEF7EAFBB5F90430A44A75
:10495800D91782FB0323C1EBA301204689B2FEF7D6
:10496800DEFB012088E69F4D0846298AFEF7D7FB23
:10497800698A2046FEF7D3FB2046A98AFEF7CFFBBB
:10498800012079E6DFF894E20027FEB271460023A1
:104998002268501C206016702268501C206013701A
:1049A800226811F8010F0133551C062B2560107081
:1049B800EED10137062F0EF1060EE6D18A49002303
:1049C8002268501C206017702268501C20601370E9
:1049D800226811F8010F0133551C0B2B256010704C
:1049E800EED12368814A581C07212060197023687A
:1049F8000021581C20601970236892F8F020591C77
:104A0800216001201A7037E60B68794A79491078D5
:104A1800794A5D1C2560187023688978581C2060C5
:104A2800197023689278591C216001201A7023E6B6
:104A38000B68724D591C2A7921601A7023686A79AB
:104A4800591C21601A7029882046FEF768FB2368E4
:104A5800AA79591C21601A7069882046FEF75FFB05
:104A68002368EA79591C216001201A7004E60B6852
:104A780000255A1C0A60204629461D70FEF738FB9F
:104A880029462046FEF734FB20462946FEF730FB30
:104A98000120F1E50B685A4A5A4D11785A4A581CB8
:104AA8002060197011682046FEF722FB2368574AD8
:104AB800591C127A21601A7029882046FEF72FFBAC
:104AC800A9882046FEF72BFB29892046FEF727FBFD
:104AD80000212046FEF723FB20460021FEF71FFB9E
:104AE8000120C9E5084608224849FEF7EAFA0120EC
:104AF800C2E50B68464A581C9178206019702368F3
:104B08005278591C216001201A70B5E50B68394AA2
:104B18004049D078384A5D1C256018702368497967
:104B2800581C206019702368D278591C2160012014
:104B38001A70A1E500212046FEF7F1FA002120466F
:104B4800FEF7EDFA00212046FEF7E9FA2368324D18
:104B580000265A1C22601E7023682A68591C92F885
:104B68002C2021601A7023682A68591C92F8362074
:104B780021601A7023682A68591C92F8372021602E
:104B88001A7023685A1C22601E7023685A1C2260FF
:104B98001E7023685A1C22601E702B682046598F8D
:104BA800FEF7BDFA2B682046198FFEF7B8FA23687E
:104BB8002A68591C92F82E2021601A7023685A1C02
:104BC80022601E702B682046598EFEF7A8FA2B68C3
:104BD8002046998EFEF7A3FA01204DE530600020AB
:104BE80067666666304C002013600020305F002046
:104BF800C8680020184B0020284B0020A441002042
:104C0800544B002014310020443400207C4F0020F5
:104C1800344B0020C848002050600020EF5F00207F
:104C2800B54E0B687279B54D591C21601A702B6806
:104C38002046198CFEF773FA2B682046D98BFEF7AD
:104C48006EFA71892046FEF76AFAB1892046FEF7A6
:104C580066FA2B682046598CFEF761FA2B682046C5
:104C6800998CFEF75CFAF1892046FEF758FA318AEA
:104C78002046FEF754FA2A68236892F82620591C21
:104C8800216001201A70F7E49B4EF378002B00F0A6
:104C980025830B680822591C21601A702368012299
:104CA800991821601A702368954D591C2A7921603A
:104CB8001A702368AA78591C21601A70298820461E
:104CC800FEF72DFAE9892046FEF729FA2368F279DA
:104CD800591C21601A702368EA78591C2160012048
:104CE8001A70C9E40B6800255A1C0A601D700B680D
:104CF8005A1C0A601D700B685A1C0A6029461D70F0
:104D0800BFE6804B03F1700522681978501C2060BB
:104D1800117022685978501C2060117022689978A7
:104D2800501C206011702268D978501C20601170C6
:104D380022681979501C2060117022685979501C1A
:104D480020601170226899790733501C9D422060B9
:104D58001170D9D18FE46C4D0846E989FEF7DFF967
:104D68002046A989FEF7DBF9012085E40B68674F27
:104D7800591C3A7821601A703B78002B3FF47BACC1
:104D88000025EEB2304619F051FC23684278591CD0
:104D9800216030461A7019F049FC01892046FEF757
:104DA800BEF93B780135AB42EBDC64E4584D594E13
:104DB8009FED598ADFF88C81DFED588A05F12007CD
:104DC8000EE0FCEEE77ACDED017ABDF8041020463E
:104DD8000435FEF7A4F9AF4206F118063FF44BACD0
:104DE800717C0029F3D04E4BD5ED007A1B78012B4E
:104DF800E7D14C4B1B68DB0440F16882F5EE407A42
:104E0800F1EE10FA40F0918240F2DC51DFE70846FB
:104E180010224549FEF755F901202DE4434B9B8AA2
:104E2800B3F5006F00F26682B3F5806F00F27B8203
:104E3800B3F5007F34BF012702273D4D05F10C066D
:104E480055F8041B91FBF7F1204689B2FEF767F984
:104E5800AE42F5D1374D384F05F10C06B5EC010AD5
:104E6800D7ED087A80EE270A28F0BAFA81B22046F0
:104E7800FEF755F9AE42F1D1304D05F10C0655F863
:104E8800041B204689B2FEF74AF9AE42F7D1FFF774
:104E9800F2BB00258146DFF8B080DFF8B0B0059599
:104EA80004950695079501214FF6FF7A05E001352F
:104EB8000B2D00F0388118F9011F4F1C4AFA05F331
:104EC800F5D0DE07F3D5BBF800302B41D807EED577
:104ED80006A8FEF709FBEAE7194D08462988FEF7F8
:104EE8001EF9A9882046FEF71AF920462989FEF7F7
:104EF80016F90120FFF7C0BBC868002050600020E9
:104F0800304C0020BC420020184B00204C5400209C
:104F18005C490020B06C00200000404200E0824460
:104F2800544C0020706B00204C490020683F002042
:104F3800A03F0020646B0020DC680020B441002002
:104F480014310020DB9B91417CF702082C60002083
:104F5800944D05F15006287823F0E8F82368027A82
:104F6800591C21601A7023686A78591C21601A70CC
:104F78002368AA78591C21601A702368EA780435D6
:104F8800591CB54221601A70E5D1FFF774BB0B6854
:104F9800854A591C527D216001201A70FFF76CBBAD
:104FA800824D05F1800655F8041F2046FEF7A0F84B
:104FB800AE42F8D1FFF75FBB7D4D05F14006B5F86D
:104FC80080102046FEF7ABF8236895F88220591C1C
:104FD80021601A70236895F883200435591CB5425E
:104FE80021601A70EBD1FFF746BB6F4D0B682A7A28
:104FF800591C21601A70A98B2046FEF790F8298B5E
:105008002046FEF78CF8698B2046FEF788F823685F
:10501800EA7C591C21601A70A98C2046FEF77FF89B
:10502800E98C2046FEF77BF82368AA7F591C21608B
:105038001A70236895F82020591C21601A70698C11
:105048002046FEF76CF82368EA7A591C21601A702A
:10505800E9682046FEF74CF823682A7C591C216031
:105068001A70236895F82120591C216001201A70B4
:10507800FFF702BB0B6801229918216010461A70CD
:10508800FFF7FABA08460021FEF732F80120FFF7C9
:10509800F3BA484D484E05F1180795F9023096F9CC
:1050A80006209A4200F0F08096F90E209A4200F00D
:1050B800EB8096F916209A4200F0E6800835BD424A
:1050C800EBD1FFF7D8BA3D4B03F15A05226859795D
:1050D800501C2060117022681978501C20601170D3
:1050E80022685978501C2060117022689978501CE9
:1050F800206011702268D978501C206011702268D5
:1051080019790633501C9D4220601170DED1FFF7DB
:10511800B2BA0B682A4A581C117820601970EEE45C
:105128000020FFF7A9BADFF8A4A000254FF008086F
:105138000135C5F1200208FA02F2A5F120032AFA86
:1051480005F6164328FA03F31E43252D06F001023F
:105158004FF000030BD01343EAD0E8B21DF0FAFB7E
:105168000028E5D0294606A8FEF7BEF9E0E7154B6A
:105178001B78DA0700F1C7800025134E2F4602E09E
:105188000135252D24D029463046FEF7BCF90028E4
:10519800F6D0294606A8FEF7B6F9002840F0918017
:1051A8000137EDE7584B00207C4F00202C5F002092
:1051B800305F0020DC670020604F00207140002035
:1051C800544B0020F2660020AC66002090E33FF4C8
:1051D800744B754DB3F850102046FDF7A0FF734B84
:1051E8001988204689B2FDF79AFF714B19684B015F
:1051F80003F02002C1F340031343C1F3800243EAE2
:105208004203C1F3C00243EA8203C1F3401243EAF6
:10521800C20301F0100119432046FDF780FF04A9DD
:1052280004222046FDF74DFF23682978614A581C5F
:105238002060197011886429A8BF64212046FDF7F1
:105248006EFFB9F1960F63D000212046FDF767FF86
:105258002168B7F1190348BFA7F11203A3F3C403E8
:105268004A1C226020461A460B7005A9FDF729FF43
:105278002368514A581C1021206019702046118853
:10528800FDF736FFFFF7F7B92268511C216013704C
:1052980029882046FDF743FF2368EA78591C2160D6
:1052A8001A7023682A79591C21601A702368AA7910
:1052B800591C21601A7023686A79591C21601A7078
:1052C800FCE6394604A8FEF70FF969E7F4EEC87A58
:1052D800F1EE10FA45DA4FF47A7178E50B68B17897
:1052E800364A581C2060197023681278591C2160AE
:1052F8001A70D8E40827A0E523685A1C2260012008
:105308001D70FFF7B9B9069B43F00103069333E715
:1053180023680322591C21601A7023686A78591C73
:1053280021601A7094E7042787E5F4EEC87AF1EE55
:1053380010FA3FF569ADF4EEE87AFDEEE77AF1EEA2
:1053480010FA17EE901A1ED86FF4F973303903FB70
:1053580001F140F2E73391FBF3F101F2DB5189B23D
:1053680035E5FDEEE77A40F2E73217EE903A303B4A
:1053780002FB03F388FB0312D917C1EB622101F288
:10538800E93189B223E540F2F313A1F5836103FB08
:1053980001F140F2E73391FBF3F101F2DD5189B2FB
:1053A80015E500BF30070020546000209841002018
:1053B800D84600209C410020DE4600200C4B0020EF
:1053C80008B501210220FCF7DFFD094B1B7803F02B
:1053D8000503052B08D000210120FCF7D5FD00218D
:1053E8000846FCF7D1FDFEE713F0A4FBF3E700BF86
:1053F800642E0020022810B428BF0220064C074B58
:10540800207000EB8001064A5DF8044BC0EBC10038
:1054180003EB4000106070475460002016330020F2
:105428005060002008B521F0A1FBFDF733FCBDE872
:10543800084021F083BB00BF2DE9F04F013085B053
:10544800C3B203938E4D8F4F8F4C904E0A23029315
:105458003220DFF840921FF029FD4FF4FA7A4FF01E
:10546800100C4FF47A70D9F80430C3F30803002BFA
:1054780040F0C880EFF31183002B40F0C380296807
:10548800A26800BF2B689942F9D1D7F800E000FB69
:105498000EF39B1AB3FBFEF300FB01314FF0010E34
:1054A8000191D9F80430C3F30803002B40F08E8033
:1054B800EFF31183002B40F089802B68A16800BFAF
:1054C8002A689342F9D1D7F800B000FB0BF2521AC0
:1054D800B2FBFBF200FB0323019A9B1AB3F57A7F18
:1054E800DFD3BAF1010ABED1039B002B40F0C48080
:1054F8004FF47A7ADFF89C9150464FF0100CD9F8A7
:105508000430C3F30803002B40F09980EFF31183B4
:10551800002B40F094802968A26800BF2B6899424C
:10552800F9D1D7F800E000FB0EF39B1AB3FBFEF3AA
:1055380000FB01314FF0010E0191D9F80430C3F39B
:1055480008033BBBEFF3118323BB2B68A16800BFA3
:105558002A689342F9D1D7F800B000FB0BF2521A2F
:10556800B2FBFBF200FB0323019A9B1AB3F57A7F87
:10557800E3D3BAF1010AC2D1029B013B02937FF443
:1055880067AF4349434B4448444A0860DA6005B072
:10559800BDE8F08FEFF311888CF31288A1682368B7
:1055A800DB0344BFC6F800E0A1682B6832685FFAE5
:1055B80088F888F31188D7F800801A4400FB08F3AC
:1055C8005B1AB3FBF8F300FB0233CDE7EFF3118866
:1055D8008CF31288A1682368DB0344BFC6F800E097
:1055E800A1682B6832685FFA88F888F31188D7F8C1
:1055F80000801A4400FB08F35B1AB3FBF8F300FBC6
:10560800023369E7EFF311828CF31288D4F808E0CB
:105618002368D90303D501233360D4F808E02B6845
:105628003168D2B282F311883A68194400FB02F358
:10563800A3EB0E03B3FBF2F300FB01312EE7EFF30C
:1056480011828CF31288D4F808E02368D90303D5B3
:1056580001233360D4F808E02B683168D2B282F3B2
:1056680011883A68194400FB02F3A3EB0E03B3FB5D
:10567800F2F300FB01315DE718461FF0BDFA37E78A
:105688007C6100208061002010E000E0786100204B
:10569800FC9F002000ED00E0EFBEADDE0400FA053F
:1056A80038B5434B5A899989914224BF00225A81BF
:1056B800198ADA89914224BF0022DA81DA788AB31A
:1056C800072A2FD03B493C4D91F85700012400216F
:1056D8000A282C709C70D9713DD00C2865D0DFED5C
:1056E800377A8ABB364C9FED370AA278002918BF53
:1056F800F0EE407A062A04D8334901EB820191ED95
:105708000F0A217959B3013A032A4DD8F7EE007AE6
:1057180087EE800A27F064FE2388984228BF18463F
:10572800208038BDD97921B198780428B8BF0420E1
:105738009870204890F857000A280CD00C28CED131
:10574800DFED227A002ACDD0072ACBD00A282CD127
:10575800DFED1F7AC6E70A20DFED1E7AC1E79B78E6
:10576800154A07EE103A1178B8EEC77A27EE277A6D
:1057780007EE901AF8EEE77A67EE877AB4EEE70A52
:10578800F1EE10FA10DDC0EE077AFDEEE77A17EEBB
:10579800903A102BA8BF1023012BB8BF0123DBB20E
:1057A8008B4238BF0B46137038BDDFED0B7A99E793
:1057B800C8680020DC6800200C4B00206F120339F9
:1057C800304C00206F1203384CF702080AD7A3396F
:1057D8000F506E3A5304E9386F12833A2DE9F047B7
:1057E800B34FB44E21F0C2F9BE421ED2DFF84C834B
:1057F800DFF84C934446258862197DB14A450DD29D
:10580800052D0BD933886188C3F30B03994200F047
:10581800ED80144625886219002DEFD17168304655
:105828001436FDF7C3F9BE42E4D3A34A1378A3F1B3
:10583800170102290FD9A14911F83300002840F0B7
:105848000181D8000144497829B19D4911F83330C4
:10585800002B00F025819B4B5A78022A40F2EC80FD
:10586800002299495A701A789848022A016000F271
:10587800DF8002EB8201964BC2EBC10203EB4203CD
:10588800998C5A8C934C9142236001D300225A84FC
:10589800914B9A78042A00F0FA8032B91A88B2F546
:1058A800F07F84BF4FF4F0721A808C4DFFF7F8FE3A
:1058B8002B688B4A1A40002A00F0F580DE0700F1B9
:1058C800E180580400F1D980190700F1D1809A01CC
:1058D80000F1C8809B0400F1BE8016F04BFC10B9A3
:1058E800804823F043FB4020FDF796F98020FDF720
:1058F80093F94FF40070FDF78FF94FF40010FDF79E
:105908008BF94FF08060FDF787F94FF00060FDF7E5
:1059180083F91DF097F800213022734829F021FE01
:10592800206812F055FD714B266803F1500102E022
:10593800043399427AD01A78002AF9D19C78D87819
:105948008442F5D26A496B4B91F804E06A486B4D82
:105958005C6B6B4B2860C827642111FB0E71DFF864
:10596800E4E15960674F30F8061C674DAEF8001047
:1059780000219960D960196159619961D96183F8E9
:10598800201083F821103A702E600CB11AF090FDA7
:105998005E4B9FED5F5A1B885E4A9FED5F6A5579A3
:1059A8005E4C5F495F48086006EE903AF8EEE66A9A
:1059B8001388C5EE265A07EE103A53881279C4EDBB
:1059C800005A07EE903AB8EEC77A574BF8EEE77AE6
:1059D8001D725A7227EE067A67EE867ABDE8F0479E
:1059E80083ED017AC3ED007A21F0A8B863799B07AB
:1059F8007FF40FAF716894F804A03046FDF7D6F82D
:105A08003388BAEB133F04D01436BE42FFF4F2AE2B
:105A18000BE773887068AA1FC3F30B039A4204F15B
:105A28000601A8BF1A4627F0D3FAEDE7012289E755
:105A380000221A70264B23E7234902EB420201EBAE
:105A4800820110E7D8000C186468002C7FF4FAAEC5
:105A580017241470F6E63548FDF7DEF84020FDF708
:105A6800DBF83AE746F20900FDF7D6F82B6831E78C
:105A78002F48FDF7D1F82B6829E72E48FDF7CCF819
:105A88002B6821E72C48FDF7C7F82B6819E79A8A95
:105A9800B2F57A7FBFF409AF4FF47A729A8204E7BD
:105AA80018231370D7E643F000732B6006E700BF96
:105AB800A8600308485C0308544B002050160308EC
:105AC8004814030854600020443F0020E85E00208A
:105AD8001633002050600020304C00204434002051
:105AE80009600002DC670020882D0020584B002048
:105AF800A4410020683F00201E4B0020846600203F
:105B08009C380020190C0020BC2D0020F42B00200C
:105B1800C0C9FB48D827002017B7D138F82B002078
:105B2800584000203661023D344000200940000200
:105B380001600002092000020860000202F0030868
:105B480000000408F059002008B521F00FF8FDF70F
:105B5800A1F820F0F3FFBDE808403FE638B50D4C4A
:105B68000D4DAC4206D2616820461434FDF71EF88C
:105B7800AC42F8D3FDF7D4FC084A094B094C146031
:105B8800002209491A705A7008480860BDE8384070
:105B980010F0F2B9485C0308A860030850600020C0
:105BA8005460002016330020E85E0020443F0020A7
:105BB80008B5FFF7D3FF20F0D9FFFDF76BF8BDE874
:105BC800084020F0BBBF00BFF0B50C292BD8DFE898
:105BD80001F06F2A2A2A4C2A2A2A2B2A2A2A070065
:105BE800046AB2F80CE097881668674D24F480546C
:105BF8000462036A4468C16923F4005343EA0E331C
:105C080021F4E641A84243EA073341EA062100F0BD
:105C1800B58005F50065A84200F0B0809268446040
:105C2800C16102640362F0BD046A96899588D2F85E
:105C380000E0554F24F480740462036A4468C16923
:105C480023F4007343EA062321F07301B84243EAC0
:105C5800052341EA0E017ED04C4DA8427BD09268C4
:105C68004460C161C2630362F0BD046A9689958885
:105C7800D2F800E0444F24F010040462036A446838
:105C8800816923F0200321F0807143EA061321F48F
:105C9800E641B84243EA051341EA0E2148D03B4D9C
:105CA800A84245D092684460816182630362F0BD76
:105CB800046A9389B2F804E01768334E24F00104AB
:105CC8000462056A4468816943EA0E0321F480315D
:105CD80025F002059BB221F07301B04243EA0503A7
:105CE80041EA070114D0294DA84211D005F54065B5
:105CF800A8420DD005F58065A84209D005F5806554
:105D0800A84205D092684460816142630362F0BD95
:105D1800D689158A578A23F0080333433D43D6882A
:105D280024F4407423F00403ADB233432C43E9E771
:105D3800D589178AD68823F0800343EA051324F40B
:105D48004064558A23F0400344EA870443EA061373
:105D580044EA8504A6E7D589178AD68823F4006320
:105D680043EA052324F44054558A23F4806344EA23
:105D7800071443EA062344EA051470E7158A24F455
:105D8800804444EA851449E7002C0140003401406E
:105D98002DE9F04FC822002183B07948794CDFF80B
:105DA8000892794D794E7A4FDFF8008229F0D9FBB5
:105DB80078487949DFF8F8E1DFF8F8C1002213598B
:105DC800834200F0C280B3F1804F00F0CA80AB423A
:105DD80000F0C980B34200F0C880BB4200F0C78021
:105DE800734500F0C680634500F0C580434500F068
:105DF800C480DFF8C4A153457AD00AF5806A5345B8
:105E080008BF092375D01432782AD8D15D4C634D68
:105E1800634E614F04F1780802E01434A04564D061
:105E2800A379002BF9D023794FEA131909F1FF3927
:105E3800B9F1050F03F00F03EFD835F8190040FA50
:105E480003F2D207E9D54FF0010A0AFA03F3013B3E
:105E5800184026F0DFFD16F809305249184411EBB6
:105E6800C002DAD051F83000DFF850E1217A00F1B1
:105E780038439B0A1EF8033003F01F0E5B09022B00
:105E88000AFA0EFA63D0032B66D0012B58D09388F8
:105E98000093B3FA83F3C3F11F039BB2DA0800EB54
:105EA800820203F00703D2F820E09B004FF00F0CAA
:105EB8000CFA03FC2EEA0C0EC2F820E0D2F820E01F
:105EC80001FA03F343EA0E03136269460023022230
:105ED80014348DF804208DF805308DF806308DF8CF
:105EE800073022F08BFFA0459AD103B0BDE8F08FB0
:105EF800082309EBC3034FF0010B93F804A00AF041
:105F08001F034FEA5A1ABAF1020F0BFA03F311D022
:105F1800BAF1030F08D0DA457FF475AFD1F814A0B1
:105F280043EA0A034B616EE7D1F81CA043EA0A036F
:105F3800CB6168E7D1F818A043EA0A038B6162E7EE
:105F48007B694AEA03037B61A1E70023D1E7BB69C8
:105F58004AEA0303BB619AE7FB694AEA0303FB6168
:105F680095E70123C5E70223C3E70323C1E7042319
:105F7800BFE70523BDE70623BBE70723B9E700BF53
:105F8800185E0020CC1C03080004004000080040F4
:105F980000100040002C014000100240B42003080B
:105FA800C02003083C6E0020382003080040014050
:105FB800001400400034014000440140C41C0308A0
:105FC80001490248FEF7FEB9B85E002000400140D2
:105FD80001490248FEF7F6B9905E002000340140FE
:105FE80001490248FEF7EEB9905E002000340140F6
:105FF80001490248FEF7E6B9685E00200004004047
:1060080002494FF08040FEF7DDB900BF405E002036
:1060180001490248FEF7D6B9185E0020002C01405D
:1060280001490248FEF7CEB9185E0020002C014055
:106038002DE9F04104684A4DA30AAB4272D009D851
:10604800B3F5801F6AD04A3DAB425AD14FF0700E6B
:10605800022608E0434DAB4268D00335AB4252D12B
:106068004FF0C00E042647794FEA970C002961D0FB
:10607800B000634685190227D4F80C809F400CEBCA
:106088004503BFB2384D03F1040C47EA080745F849
:10609800231045F82C20E760EFF31181502282F39A
:1060A8001288821905EBC202136973B313620433B1
:1060B800821905EBC202576917B11F60536904338F
:1060C800821905EBC202976917B11F6093690433FF
:1060D800821905EBC202D76917B11F60D36904336F
:1060E8000027CAB21F6082F31188304405EBC00054
:1060F800036A6BB9E3684FF6FE721340E360BDE8CC
:10610800F081BDE8F081BDE8F08105EB0E03CFE733
:10611800E36843F00103E360BDE8F0814FF0480E07
:106128000126A0E74FF0200E00269CE74FF0980EBE
:10613800032698E7BF08022306FA03F0BB40DB43B7
:10614800E768094D9BB23B4087190CEB470CE360AD
:106158000CF1040345F82C1045F823209CE700BFF8
:106168004B0010004D001000185E00201F4B984295
:106178002CD0B0F1804F2BD0A3F59433984229D07E
:1061880003F58063984227D003F50063984225D031
:1061980003F58063984223D003F59033984221D0C9
:1061A80003F5406398421FD003F58063984207D0F7
:1061B80003F58063984208BF092202D00020704787
:1061C80008220B4B03EBC203187970470022F8E74B
:1061D8000122F6E70222F4E70322F2E70422F0E7BD
:1061E8000522EEE70622ECE70722EAE7002C014049
:1061F800382003082DE9F04F013085B0C3B203936E
:106208000B4602918B4C8C4E002B00F09A8032206A
:106218008A4D8B4FDFF82C921EF048FE4FF4FA7A25
:106228004FF0100C4FF47A70D9F80430C3F3080318
:10623800002B40F0DE80EFF31183002B40F0D98073
:106248002968A26800BF2B689942F9D1D7F800E005
:1062580000FB0EF39B1AB3FBFEF300FB01314FF07A
:10626800010E0191D9F80430C3F30803002B40F064
:106278008780EFF31183002B40F082802B68A168A0
:1062880000BF2A689342F9D1D7F800B000FB0BF29F
:10629800521AB2FBFBF200FB0323019A9B1AB3F5D7
:1062A8007A7FDFD3BAF1010ABED1039B002B40F0FD
:1062B800BD804FF47A7ADFF88C9150464FF0100C7D
:1062C800D9F80430C3F30803002B75D1EFF3118319
:1062D800002B71D12968A26800BF2B689942F9D1B7
:1062E800D7F800E000FB0EF39B1AB3FBFEF300FBAC
:1062F80001314FF0010E0191D9F80430C3F30803BE
:1063080013BBEFF31183FBB92B68A16800BF2A68A0
:106318009342F9D1D7F800B000FB0BF2521AB2FB46
:10632800FBF200FB0323019A9B1AB3F57A7FE3D3B0
:10633800BAF1010AC4D1029B013B0293002B7FF4FE
:1063480066AF05B0BDE8F08FEFF311888CF31288C3
:10635800A1682368DB0344BFC6F800E0A1682B6886
:1063680032685FFA88F888F31188D7F800801A44F1
:1063780000FB08F35B1AB3FBF8F300FB0233D2E728
:10638800EFF311888CF31288A1682368DB0344BFFC
:10639800C6F800E0A1682B6832685FFA88F888F3CD
:1063A8001188D7F800801A4400FB08F35B1AB3FB86
:1063B800F8F300FB023370E7EFF311828CF31288D5
:1063C800D4F808E02368D90303D501233360D4F84F
:1063D80008E02B683168D2B282F311883A68194410
:1063E80000FB02F3A3EB0E03B3FBF2F300FB013156
:1063F8007FE7EFF311828CF31288D4F808E0236862
:10640800D90303D501233360D4F808E02B68316839
:10641800D2B282F311883A68194400FB02F3A3EB65
:106428000E03B3FBF2F300FB013118E718461EF028
:10643800E3FB3EE710E000E0786100207C6100208B
:106448008061002000ED00E0204B5B68C3F3080387
:1064580030B4BBB9EFF31183A3B91D4B1D4C1868B9
:10646800A16800BF1A689042F9D11B4B1C684FF411
:106478007A7202FB04F3591AB1FBF4F130BC02FB47
:1064880000107047EFF31182102383F3128811492B
:106498008C680B6813F4803F104B02D00120186001
:1064A8008C680B49D2B20D68186882F311880A4BC0
:1064B80019684FF47A72284402FB01F31B1B30BCA5
:1064C800B3FBF1F302FB0030704700BF00ED00E0C2
:1064D8007C61002010E000E08061002078610020ED
:1064E8002DE9F84F8046FFF7AFFF254E2549DFF825
:1064F800A0E0254A254D844610274FF47A740120E0
:10650800DEF80430C3F30803D3B9EFF31183BBB942
:106518000B68D2F808A000BFD1F800904B45F7D11E
:10652800D6F800B004FB0BF9A9EB0A09B9FBFBF993
:1065380004FB0393A3EB0C034345E1D3BDE8F88FB9
:10654800EFF3118A87F31288D2F808B01368DB03D7
:1065580044BF2860D2F808B00B68D5F800905FFAFD
:106568008AFA8AF31188D6F800A0994404FB0AF342
:10657800A3EB0B03B3FBFAF304FB0933DAE700BF21
:10658800806100207C61002010E000E0786100203C
:1065980000ED00E02DE9F04FDFF830C1474A4849E7
:1065A800484E494D8046102718F1FF38C0F08480C6
:1065B800DCF80430C3F30803002B5CD1EFF311833C
:1065C800002B58D10B68946800BF08688342F9D142
:1065D800D6F800904FF47A7000FB09FEAEEB040E7B
:1065E800BEFBF9FE00FB03EEDCF80430C3F308033E
:1065F8004FF47A740120FBB9EFF31183E3B90B6808
:10660800D2F808A000BFD1F800904B45F7D1D6F8D2
:1066180000B004FB0BF9A9EB0A09B9FBFBF904FB71
:106628000393A3EB0E03B3F57A7FBDD2DCF80430F5
:10663800C3F30803002BDFD0EFF3118A87F3128826
:10664800D2F808B01368DB0344BF2860D2F808B05A
:106658000B68D5F800905FFA8AFA8AF31188D6F8A1
:1066680000A0994404FB0AF3A3EB0B03B3FBFAF372
:1066780004FB0933D5E7EFF3118487F31288D2F8C6
:1066880008901368D80303D501232B60D2F808902B
:106698000B682868E4B284F31188D6F800A04FF498
:1066A8007A7400EB030E04FB0AF3A3EB0903B3FBB4
:1066B800FAF304FB0E3E97E7BDE8F08F10E000E028
:1066C8007C610020806100207861002000ED00E0FE
:1066D80030B4EFF31183102282F312880649074C75
:1066E8000A680748013200250A602560DBB20268A3
:1066F80083F3118830BC70477C61002078610020EA
:1067080010E000E01D4B70B59C68E36C226BDD69FE
:10671800C2B1636B2BB12B0702D5E36C08221A6256
:1067280070BD2A06F7D5A26A616A8A421FD0511C39
:10673800A069A162825C2069E66C81423285EAD355
:10674800A362E8E7A906E4D5E26A1AB1988C80B298
:106758009047DEE7E1699B8C6069DBB24E1CE6611D
:106768004354E169E368994228BFE261D1E7E26CEA
:10677800136823F080031360CDE700BFC430002006
:1067880070B4EFF31186502383F31288436B1A68B1
:10679800D20720D45D686DB9446A826A944217D0E2
:1067A80081691144D9600ED9A21A5A608462002204
:1067B80080F850201A6842F00102F1B21A6081F3A1
:1067C800118870BC704701698A1A5A608562EEE7C1
:1067D800012380F85030F1B281F3118870BC704702
:1067E8002DE9F04F2DED028B93B0029013F0DEFAF5
:1067F800AA4B1D7825B113B0BDEC028BBDE8F08F14
:10680800A74B1B685C05F6D5A64FA74E3B68002B27
:1068180062D0A64C3168D4F810218A1A7C2A5BD938
:1068280094F81421C4F81011D4F81811013284F81E
:10683800142109B188473B68DFF8C4829FED9C8A20
:10684800A8F138094FF0240A5E20984750463B6863
:106858009847B9F81430F8EC016A07EE103AF8EEE8
:10686800E66AB8EEC77A0AF1010AC6EE877A5FFAD5
:106878008AFA67EE887AFDEEE77ACDED037ABDF9FC
:106888000CB05FFA8BF018F063FACBF3072018F01E
:106898005FFABAF1270F3B68D6D15E2098473B686C
:1068A80030209847834BD3F800805FFA88F018F0BF
:1068B8004FFAC8F3072018F04BFA3B685E20984758
:1068C80094F8143113F0030800F07881580701F0A8
:1068D8001480282B01F05583774B1B78002B6FD041
:1068E800724C0299D4F82031744ACB1A934200F2C0
:1068F8008D87DFF810A29AF80080B8F1000F34D124
:10690800DFF8C891D9F80000FAF7D4FAC0B2012824
:106918000FD902286A4F41F001843B78002B41F0DF
:106928002286D4F82831029AD31AB3F57A6F81F007
:106938007D8764480268002A42D09AF80030BBB9C3
:10694800614BD9F800001B689B781E3B012B4FF068
:10695800020141F2DC86043018F06CF901220023B0
:106968008AF8002084F8343127E0564802683AB3A0
:10697800D4F83031029F40F6B731FB1A8B421FD949
:1069880094F82C31002B01F0C583013BDBB284F86D
:106998002C31002B01F0ED8212F8011B94F83471B0
:1069A800026094F835314948CA190133006884F8FF
:1069B800342184F83531FAF780FA029BC4F8303173
:1069C800434BD6F800801B7843B1424F386828B152
:1069D800414B1B78013B012B41F239803F4B1B781F
:1069E80063B13F4F3B684BB1304CD6F800B0D4F898
:1069F8004C31ABEB0303632B00F26786DFF80881A9
:106A080098F80030022B01F08A822D4F97F87430E5
:106A1800032B00F05C87334B1B7873B1324D2B6826
:106A28005BB1224CFFF710FDD4F8583144F61F62D1
:106A3800C31A9342834600F215812C4B1B78002B16
:106A480040F086802A4B1B784BB1184C029AD4F838
:106A5800A83203F5C333A0339A4280F09786254BBA
:106A68001B78002B3FF4C7AE104E234C234D06F283
:106A7800C9272068FAF71EFA00283FF4BCAE206840
:106A8800FAF715FA2B7880465A1E002B3ED020685C
:106A98002A70FAF70FFA0028F1D1ACE6D93A0020AB
:106AA800706B0020245800207C610020E82700201B
:106AB80000007A4460600020724700203F0D030008
:106AC800180000201C5800201858002014580020D6
:106AD80074470020945500207C47002084470020FC
:106AE800085000208C47002090470020D047002005
:106AF800E1470020964700209C470020A04700203F
:106B0800A03F00202058002032640020032239468C
:106B1800781E28F00CFD96F8C83296F8C92286F837
:106B2800CB8283F47F4383F0FF039B1A1FFA88F814
:106B38009BB2B8EB132F9CD196F8CA22DBB29A42CB
:106B480097D1781E17F0F2FD2B781844287090E73B
:106B58003A4C2278002A40F0FA85394E3478002CD5
:106B68005FD1384D2878002841F08A84364C374D5B
:106B7800D4F8A0122A78364B93FBF2F3029A0B440E
:106B88009A42FFF45FAF114694F8A432314AC4F830
:106B9800A012D65CF70701F1AA86B10701F1648655
:106BA800720701F1FF8594F8A4322978013393FB29
:106BB800F1F201FB123384F8A43243E7D4F8102130
:106BC80041F288339A4201F25F823B685E2098471F
:106BD8003B6814209847204B204AB3F9043082FBC5
:106BE80003124FEAE378C8EBA2080FFA88F85FFAB5
:106BF80088F018F0ADF8C8F3072018F0A9F83B683A
:106C08005E2098473B681C209847002018F0A0F8A1
:106C1800002018F09DF83B685E20984794F81431DE
:106C280054E60F4D286E002841F0FB818046064B44
:106C3800029A86F80080C3F8A02203E76447002080
:106C4800D9470020D8470020E8270020E047002047
:106C5800A0860100DC470020306000206766666679
:106C6800E847002094F85E31002B41F0C481DB4BEB
:106C78001A6802F00803002B48F603414AF60B4055
:106C88004BF60F4349F6074704BF03460F4612F079
:106C9800040F4FF0190118BF1F46920684F85E11C1
:106CA80003D547F4804747F02007CD4B5A79C7F3FF
:106CB8000909002A41F066869B79002B41F07E87FE
:106CC800984664204FF0FF3A4FF0000C0A970B9754
:106CD800ADF834C0CDF83AC0CDF83EC0CDF842C0CA
:106CE800CDF83090ADF83680ADF838A08DF8460074
:106CF8000AAF0FCFDFF800E384F805C0AEE80F0055
:106D080097E80F00AEE807002EF8023B71464FF0F7
:106D1800010C1B0CFE271F20C82201F81E39A77082
:106D2800A27184F807C0E07094F86E01207180F0B9
:106D3800F10383EA0313DAB2130983F0E70343EAA2
:106D4800022383EAC2031BB283EA0312D2B2C3F35B
:106D5800072383EA121343EA022383EAC2031BB21E
:106D680083F0C80282EA0212D2B2C3F3072383EA8D
:106D7800121343EA022383EAC2031BB283EA0C0715
:106D880087EA0717FFB2C3F3072282EA171242EA1B
:106D9800072200EB0C0382EAC7070EEB0C0084F80D
:106DA8006E31278011F8013B7B4083EA0313DBB285
:106DB8001A0982EA172242EA032282EAC3031BB2B3
:106DC8009FB281422780EDD183F07C0383EA0313CD
:106DD800DBB24FEA131E8EEA172E8EEA032E8EEAD6
:106DE800C30E0FFA8EFE1FFA8EFADFF810C2A4F84F
:106DF80000A05FFA8EFE4FEA1A2A84F828A084F8C9
:106E080027E00CF5CB7804F12209DCF80000DCF867
:106E18000410DCF80820DCF80C3047460FC70CF1EA
:106E2800100CCC45B846F0D1DCF8000038606D4F46
:106E38009CF8043088F8043007F1270884F8BDE18D
:106E480084F8BEA117F8011F2868FAF736F8B84584
:106E5800F8D194F85F31002B41F0D2806249326852
:106E680009780A2084F85F01002901F023825F4F26
:106E780001293888069041F2A8860229B7F802E06D
:106E880001F09785B8880590032901F0A786F8884E
:106E98000490042901F0B8860529388901F0AF86E5
:106EA8000629B7F80A9001F0A6860729B7F80C80DA
:106EB80001F09E86FB89039394F86E110A920B46A3
:106EC80083F0300282EA0212D2B2170948490793C6
:106ED80087F07A0747EA02270988237187EAC202FE
:106EE800444FC1EB012187FB013A069B4FF0000C90
:106EF80063F30F0C059B6EF31F4C4FF0000E63F30A
:106F08000F0E049BCDF82CC012B28A440027C91773
:106F180063F31F4EC1EB6A2A039BCDF830E082EA87
:106F2800021160F30F070020C9B268F30F00C2F323
:106F3800072269F31F4782EA111263F31F404FF0DB
:106F480000090D978DF83DA00E908DF83C9042EA0F
:106F580001220DF1280C82EAC107BCE80F003FB2FC
:106F680087F0C80888EA0818DFF88CE084F80590EC
:106F78005FFA88F8C7F30727AEE80F0087EA181703
:106F880047EA08239CE8030083EAC8031BB283F09E
:106F980023024EF8040B82EA0212D2B2C3F307238B
:106FA800079F83EA1213704643EA022383EAC20268
:106FB80007F1010C20F814194FF023081621FE27B9
:106FC800C82384F86EC1228084F807800EF1020E6F
:106FD800A770E170A371114612E000BFD8460020E7
:106FE800A04600207F2900208C370020D0540020A4
:106FF800B646002003082080F0270020EA2700205A
:1070080010F8013B4B4083EA0313DBB21A0982EA0A
:10701800112242EA032282EAC3031BB299B27045E5
:107028002180EDD183F0F40383EA0313DBB24FEA46
:10703800131E8EEA112E8EEA032E8EEAC30E0FFA65
:107048008EFE1FFA8EF8E44FA4F800804FEA182C41
:107058005FFA8EFE84F81EE084F81FC07968BA686B
:107068003868FB6807F5CB78A8E80F0038697969B4
:10707800BA6904F29717A8E8070004F2B51884F86B
:10708800B5C184F8B4E117F8011F2868F9F715FFAE
:10709800B845F8D194F866C1BCF1000F40F0BB8741
:1070A800CE4B94F86E71B3F90010B3F90220B3F91E
:1070B80004309FEDCB6ADFF844E384F805C007EE9F
:1070C800103A33680A9387F06A0383EA031306EEDB
:1070D800901AD9B20B0983F0D50343EA012383EA56
:1070E800C1031BB283EA03115242C9B207EE902AC8
:1070F800C3F3072383EA111343EA0123F8EEE77A7F
:10710800F8EEE66AB8EEC77A83EAC1031BB267EE07
:10711800867A66EE866A27EE067A002083F0C8082B
:10712800CDED0C7ACDED0B6A8DED0D7A0E900F90AA
:10713800109088EA08160DF12809F6B2C3F307285B
:10714800B9E80F0088EA161848EA062888EAC60847
:107158000FFA88F8AEE80F0088F01E0699E80700D5
:1071680086EA0616F6B2C8F3072383EA161343EA3B
:1071780006238EE8070083EAC6061C20C8214FF0C4
:1071880005084FF01E0CFE237A1CE070A17184F8EC
:10719800668184F807C0A370AEF1100127710EF163
:1071A8000C00268084F86E2111F8013B734083EAB5
:1071B8000313DBB21A0982EA162242EA032282EAA0
:1071C800C3031BB29EB281422680EDD183F0270310
:1071D80083EA0313DBB24FEA131E8EEA162E8EEAF9
:1071E800032E8EEAC30E0FFA8EFE1FFA8EFC7A4F1C
:1071F800A4F800C05FFA8EFE4FEA1C2C84F825C064
:1072080084F824E007F5CB7804F122093868796816
:10721800BA68FB6846460FC610374F45B046F5D1E9
:10722800704E3B88A8F8003006F1240784F8BAE1CC
:1072380084F8BBC116F8011F2868F9F73EFEB7426B
:10724800F8D194F867A1BAF1000F40F0DE86664BDA
:107258001B68052213F0140F84F8672141F014808D
:10726800DFED627A94F86EC15C4B614AB3F90410A1
:10727800B2F906205F4E6048CDED0C7A8CF02203FF
:1072880083EA0313DFB23B0983F0590343EA072378
:1072980083EAC703B2F5FA6F1BB2A8BF4FF4FA62CC
:1072A80083EA0317FFB2B2F57A7FC3F3072383EAB1
:1072B8001713B8BF4FF47A724FF0640E43EA0723EE
:1072C800A2F57A720EFB02F283EAC70386FB02E696
:1072D80080FB01E01FB2D217C9174FF00008C2EBBC
:1072E800A612C1EBA00187F0C806ADF83A20ADF8A8
:1072F8003810CDF82880CDF82C80CDF834800DF1E9
:10730800280E86EA0616BEE80F00F6B2C7F307276E
:1073180087EA161747EA062787EAC606374FDEF8D0
:1073280000E084F804C00FC736B286F04A0383EA47
:107338000313DBB2C6F3072181EA13113A4641EA87
:1073480003210CF1010C81EAC303142042F810E96F
:10735800FE264FF04A0E002184F86EC14FF0C80C8B
:10736800E0702380043784F807E0A670617184F820
:1073780006C0184612F8011B414081EA0111C9B242
:107388000B0983EA102343EA012383EAC10109B206
:1073980088B2BA422080EDD181F0140181EA01114E
:1073A800C9B24FEA111E8EEA102E8EEA012E8EEA1D
:1073B800C10E0FFA8EFE1FFA8EF6074F26804FEA8F
:1073C80016295FFA8EFE84F81D9084F81CE079680F
:1073D8003868BA68FB6813E0EA27002030600020AC
:1073E80088C3E43A7F290020D84600200000000026
:1073F800D0540020D34D621067666666F0270020DF
:10740800B7F8188007F5CB7CACE80F0038697969C4
:10741800ACE8030004F29716ACF8008084F8B39146
:10742800B04684F8B2E104F2B31918F8011F2868CD
:10743800F9F743FDC145F8D1C94BCA4A1B78127800
:10744800013B12F00100DBB214BFC0214021172B11
:1074580003D8C54A134493F830A0C44B1A8893073D
:107468001ABF002341F01001012312F4027F18BF54
:10747800022312F0100F18BF062312F0200F18BFB6
:107488001023002841F0C4814FF0030C94F86E914A
:107498000A9389F0460383EA0313DAB2130983F0E7
:1074A800920343EA022383EAC2031BB283EA03106E
:1074B800C0B2C3F3072282EA101242EA002282EA2B
:1074C800C00212B282F0C80E8EEA0E1E5FFA8EFE5D
:1074D800C2F30722002382EA1E1203208DF82CA093
:1074E8008DF82FC08DF82D3042EA0E2C8DF82E1015
:1074F8008DF830000AAA07CA8CEACE0E0FFA8EFE63
:10750800DFF878A2E3718EEA0E1CAAE803005FFA9E
:107518008CFCCEF3072E8EEA1C1E4EEA0C2181EA63
:10752800CC0C94F808E08AF800200FFA8CFC8EEA5C
:107538000C0E8EEA0E1E5FFA8EFECCF3072282EA4C
:107548001E1242EA0E22607AA17A94F80BC0637187
:1075580082EACE0212B2504080EA001E5FFA8EFE26
:10756800C2F3072080EA1E1040EA0E2080EACE000F
:1075780000B2414081EA0111C9B2C0F3072282EA90
:10758800111242EA012282EAC10212B28CEA020C0A
:107598008CEA0C1C5FFA8CFCC2F3072282EA1C12EC
:1075A80042EA0C2294F80CE0607BA17B94F81080EE
:1075B80084F8049082EACC0212B28EEA020E8EEAB5
:1075C8000E1E5FFA8EFEC2F3072282EA1E1242EAFC
:1075D8000E2282EACE0212B2504080EA0010C0B2F7
:1075E800C2F3072282EA101242EA002282EAC002AB
:1075F80012B2514081EA0111C9B2C2F3072282EAEC
:10760800111242EA012282EAC102E17B13B281EA45
:10761800030282EA0212D2B2C3F3072383EA1213E7
:1076280043EA022383EAC2031BB288EA030282EA1E
:107638000212D2B2C3F3072383EA121343EA0223E6
:1076480083EAC2031BB283F0320282EA0212D2B288
:10765800C3F3072383EA121343EA022383EAC2032C
:107668001BB29AB24FF0FE0C4FF0090EC82009F178
:107678000101DBB284F802C084F803E04FEA122C5F
:10768800A07184F86E11228084F812C0637438687F
:107698007968BA68B7F80C900AF5C47EAEE80700B6
:1076A8000AF5CC7A8EF80280AEF8009084F8A8C16A
:1076B80084F8A73116F8011F2868F9F7FEFBB245D0
:1076C800F8D1C4F858B1FFF7B8B9DFF8B4A0DFF8BB
:1076D800B480DFF8B490412017F05CFABAF90230B0
:1076E80088FB0320DB17C3EBA00080B217F038FA41
:1076F800BAF9003088FB0320DB17C3EBA00080B287
:1077080017F02EFABAF9043088FB0320DB17C3EB15
:10771800A00080B217F024FA99F800103868F9F739
:10772800CCFB94F8503113F0010800F01B85104A87
:10773800C4F84CB10133DBB2A2FB0312D20802EB4E
:107748008202A3EB420384F85031FFF757B9094B83
:1077580009491868F9F785FB00232370FFF7FDB97D
:10776800544B0020F2660020A4F702082C60002089
:10777800CDCCCCCCD447002024470020F0270020D3
:107788003060002067666666D6530020114694F87C
:10779800AC32B34AC4F8A81202EB8302926C42B32B
:1077A80012AD04F2B323AF4E45F8203D002104F298
:1077B800C52331800B9380211523A52784F8B23285
:1077C800284684F8B11284F8B07290472846318868
:1077D800FBF7A5FC0A9DA44804F52C716D1A152D1C
:1077E800A8BF15252A4625F0F3FBA04A94F8AC3229
:1077F80015709F4A013382FB0312A2EBE37202EB7E
:1078080042029B1A84F8AC32FFF729B9994A9A4B7D
:1078180092F80BE03068D4F824211B889749801A25
:107828004FF47A72DFB202FB0EF21B0A8F770F75E4
:1078380090424FF00007CB774B758F700F7180F037
:1078480014848F4BDFF848E2D3F800808D4A029BFE
:107858008D48C4F820318EFB083C4FEAE873006875
:1078680017689268C3EB6C13DFF83CC28EFB008E7E
:107878008CFB07988CFB029CD217C2EBAC0203F579
:10788800FA734FEAE07C9BB2CCEB6E1CFF1700F555
:10789800EA4EC7EBA8070EF1300E8B761B0A0CF1E7
:1078A800780C4FEA2E2E3030CB764FEA2728131269
:1078B8000F7781F81D8081F8202081F8213081F828
:1078C80024C081F823E081F82200FFF712B8DFF81E
:1078D800DC91D9F80000F9F7E7FA00283FF49BA8F3
:1078E800D9F800000121F9F7DCFA0222002387F811
:1078F800742088F80030FFF78EB83B685E20984700
:107908003B6802209847614B614A9B6A323382FB8D
:107918000328DB17C3EB68185FFA88F017F018FA2A
:10792800C8F3072017F014FA3B685E2098473B68B5
:1079380003209847574B1B78D90740F1D9831BF090
:1079480035F8554B9FED557AD3ED037A67EE877A74
:10795800FCEEE77ACDED037ABDF80C30002800F094
:10796800DA86D8B24FEA132817F0F2F9404617F032
:10797800EFF9DFF83C8198F80530002B40F0AD8432
:107988000AA9474817F0A8F93B685E2098473B6862
:1079980013209847BDF928805FFA88F017F0D8F9C6
:1079A800C8F3072017F0D4F93B685E2098473B6876
:1079B8001B209847BDF92A805FFA88F017F0C8F9AC
:1079C800C8F3072017F0C4F93B685E2098473B6866
:1079D800232098474E2017F0BBF9002017F0B8F97C
:1079E8000AA92F4817F078F93B685E2098473B684A
:1079F80012209847BDF928805FFA88F017F0A8F997
:107A0800C8F3072017F0A4F93B685E2098473B6845
:107A18001A209847BDF92A805FFA88F017F098F97C
:107A2800C8F3072017F094F93B685E2098473B6835
:107A380022209847452017F08BF9002017F088F985
:107A48003B685E20984794F81431FEF742BF154C06
:107A5800DFF860904FF0010B4FF0000A35E000BFEF
:107A6800A4F70208E046002000590020155900201C
:107A78005655555548560020A8550020A4470020C3
:107A8800BC4600209C550020606000202049002052
:107A98001F85EB51F266002058560020CDCC4C3E95
:107AA80080969800E827002067666666A464002030
:107AB800A0460020180000201B2B00F046820D2B4A
:107AC80000F0118289F801B03868F9F7F3F9002855
:107AD80038D03868F9F7EBF983B27E2B32682AD0B0
:107AE80099F801100029EFD194F83621002AE3D043
:107AF8007D2B00F0098294F844E1BEF1000F04D018
:107B080080F02003DBB284F84411511CC9B222442E
:107B1800092984F8361182F8383100F0EB810829F8
:107B2800D2D8B4F84221134403EB132303F0FF0324
:107B3800A4F84231C8E784F836A184F837A189F857
:107B480001A0C1E794F8453133B194F8393184F88C
:107B58004501302B00F0FD8594F83721C04BDFF844
:107B68003CC3DFF834B3DFF838E3DFF838A3012784
:107B7800002A3EF433AF3168A1EB0801012900F275
:107B8800AD8194F84691B9F1000F40F0E78194F87F
:107B9800471133F8110010B984F84771E8E701314B
:107BA800B0F5826F84F8471100F0DC801ED9B0F57B
:107BB800E26F00F09A8034D9B0F5046F00F0A3802A
:107BC800B0F5116F00F02181B0F5E46FD0D1A54A6E
:107BD800176C918A642303FB07F393FBF1F117F009
:107BE8000FF8002384F83731FEF7F8BEB0F5007FB0
:107BF80000F095802DD8B0F5807F00F02081B0F599
:107C0800887FB5D1DCF800104907B1D5964B4FF401
:107C18008870196816F0F4FF002384F83731FEF7EE
:107C2800DDBEB0F5C06F00F08D80B0F5E06F9FD17C
:107C38008C4A906B918A642303FB00F34FF4E06055
:107C480093FBF1F116F0DCFF002384F83731FEF7DF
:107C5800C5BEB0F5047F00F02781B0F5806F87D1ED
:107C680094F848310133DBB2032B00F2528142F21F
:107C7800107184F8483101FB03F17C4B1B88002B01
:107C880040F0458101317A4B1B78DF07794B1B881F
:107C980048BF0431D80748BF0A319A0748BF143192
:107CA8001F0648BF2831D80548BF28315A0748BFA2
:107CB80064311F0748BFC831980548BF01F5C8712E
:107CC8009A0648BF01F57A71DF0648BF01F5FA61E7
:107CD800580648BF01F57A614FF4806016F090FFAE
:107CE800002384F83731FEF779BE5E4AD76B918A54
:107CF800642303FB07F393FBF1F116F081FF84F88B
:107D08003791FEF76BBE5C4BB3F9041001EB8101B0
:107D1800490016F075FF84F83791FEF75FBE9EF8AC
:107D2800061000293FF424AF544B55491B6881FBCA
:107D38000321DB17C3EBA10116F062FF84F837912A
:107D4800FEF74CBE9EF8061000293FF411AF4B4BCE
:107D58004FF4C060996816F053FF002384F8373158
:107D6800FEF73CBEDCF8001011F020097FF400AFEC
:107D780044490868010600F1D6849BF80C100029D4
:107D88003FF4F6AE94F84911032900F23486DFE88F
:107D980001F0322819023C4B1B6859799A79DB7932
:107DA80001F1407101EB022101EB0341002384F84A
:107DB80049314FF4826016F023FF002384F83731ED
:107DC800FEF70CBE314B1A68137A507992781B046F
:107DD80003EB002313444A1C84F8492103EB016197
:107DE800E7E72A4B1A68D379107952781B0403EB1A
:107DF80000231344EFE7254B1A689379D07812785B
:107E08001B0403EB00231344E5E79EF80510002943
:107E18003FF4AEAE9AF8001000293FF4A9AE1C4B0F
:107E28001B8803EB83035B004FF4116093FBF1F1B4
:107E380016F0E6FE002384F83731FEF7CFBDDCF8F4
:107E4800001048077FF594AE124B4FF48070196804
:107E580016F0D6FE002384F83731FEF7BFBD00BF09
:107E6800A4F70208683F002060600020DE4600207A
:107E7800F26600202C600020306000209C55002015
:107E880067666666706B0020E85E00205060002020
:107E9800A8550020BC46002048560020D84600209F
:107EA800A0460020565600209EF8051000293FF4F1
:107EB8005FAE9AF8001000293FF45AAE9A4B5B7BEC
:107EC800002B00F0AF84994B1B8893FBF1F101EB79
:107ED800810149004FF4047016F092FE002384F8E3
:107EE8003731FEF77BBD84F836B184F83831A4F811
:107EF8004221E9E5B4F84221C2F1FF0293427FF43E
:107F0800E1AD84F845B1DDE584F844B1DCE5023142
:107F1800B9E6012384F8483142F21071ADE6FEF764
:107F280093FA834B1B68C01A40F6B833984200F2A4
:107F3800B681DFF820B29BF804303A2B00F01A83A0
:107F4800002388F80030FEF766BD3868F8F7B2FFFE
:107F580000287FF4B7AD84F837B1B5E57549062038
:107F680016F06EFC002384F8460184F83731FEF7DA
:107F780035BD94F8341194F835316F484A1CFEF732
:107F880014BD4FF000083B68D6F8009084F81481BF
:107F98005E2098473B68694C17209847404616F082
:107FA800D7FE674BA3FB09239B0BA4FB03125209C3
:107FB800C2EB0212A3EB8203D8B216F0C9FE3B68EB
:107FC8005E2098473B68182098475E4BA3FB09231F
:107FD8009B09A4FB03125209C2EB0212A3EB820312
:107FE800D8B216F0B5FE404616F0B2FE3B685E20E9
:107FF8009847FEF771BC013B84F85E31FEF729BF54
:10800800013B84F85F31FFF745B80AF1FF3A84F87D
:1080180067A1FFF756BB0CF1FF3C84F866C1FFF778
:1080280010B90024484FA0464FF0500902E0DBB2D7
:1080380083F3118815F804A0601C5146284416F0F3
:10804800A3FC002840F040810AF101031C44EFF32F
:10805800118389F312882A6E9442E8DB0022DBB28E
:108068002A6683F31188FEF7E2BD384B32681B7825
:10807800C4F82421013B012B3FF6E3AB1022022375
:108088008A700B71FFF7DDBB3B68DFF8CCB0DFF817
:10809800CC905E2098473B6810209847DBF800306A
:1080A80089FB032ADB17C3EB6A1A5FFA8AF016F01A
:1080B8004FFECAF3072016F04BFE3B685E20984738
:1080C8003B6821209847DBF8003089FB0329D81743
:1080D8006422C0EB691002FB10300028B8BF404290
:1080E800C0B216F035FE404616F032FEFEF76DBD02
:1080F800DFF86C80164BB8F80890A3FB09394FEAF3
:1081080099095FFA89F016F023FE4FEA192016F054
:108118001FFE30E416F0C2FDFEF74FBC16F0AEFDB0
:1081280001233B70FEF705BC48560020A8550020E7
:108138003864002003EC01081458002089888888D6
:1081480073B2E745D34D6210359D0108CC46002037
:10815800CDCCCCCC20640020BC4600201F85EB5140
:10816800A0460020B64B1B88DA0515D4D80600F1C6
:108178002884990600F138845A0600F147841807C4
:1081880000F15184D90700F1528413F0020F0CBF9B
:108198004FF004084FF00C08AA4BAB4A1B78D27872
:1081A80003F001030AB143F002035320039316F0CE
:1081B800F1FCA64A128802EB820202EB82029000CE
:1081C80080B216F0CDFC002016F0CAFCA04AA149E6
:1081D80012883868C2EBC212520081FB0231114486
:1081E8004FEAE27ACAEB612A5FFA8AFA5146F8F74F
:1081F80064FE99F80020039B386848EA03088AEA75
:10820800020A002189F800A0F8F757FE41463868AD
:10821800F8F753FE99F80030386888EA0303DBB2B0
:10822800194689F80030F8F748FE94F85031002BC9
:108238007FF47DAA4F2016F0ADFC14F0F5FC14F085
:10824800F3FC14F0F1FC01213868F8F736FE824A95
:1082580099F8003092F80080386808F0010883F037
:108268000103414689F80030F8F727FE99F80030F5
:10827800386888EA0303194689F80030F8F71DFEC4
:1082880094F85031FFF753BA744B9FED757AD3EDDC
:10829800007AF8EEE77A67EE877AFEF7E3BF714A6D
:1082A800B2F8523100210133A2F8523188F8001097
:1082B800FEF7B1BB884689460846049105918E466B
:1082C80006910391FEF7F8BD39463A2016F0B8FA40
:1082D80040EA08085FFA88F8B6E6DFF898B19BF834
:1082E80000A0BAF1000F3FF44BAB584AB4F81CE1B8
:1082F80011883B6803924FEA0E1E64201FFA8EFE17
:1083080000FB01A14FEA4A00B1FBF0F14EEA012E51
:108318001FFA8EFEC1F303215E204EEA0109984739
:108328003B68062098475FFA89F016F011FD4FEA7E
:10833800192016F00DFDB4F81C31039A4A49B2F819
:1083480000904A7A01339BB2012A93FBFAF00AFBA8
:108358001033A4F81C3100F06E836E2343484A7B27
:1083680003FB09F380FB03014FEAE379C9EBA10999
:108378002AB11FFA89F99BF8003099FBF3F93B6899
:10838800DFF8F4A05E2098471FFA89F93B683A2085
:108398009847AAFB093A4FEA5A1A1FFA8AFB5FFA6A
:1083A8008BF016F0D5FC4FEA1B2016F0D1FC3B6889
:1083B8005E2098473B683B209847642303FB1A9349
:1083C8009BB22B48053380FB0320DB17C3EBA000CF
:1083D800C0B216F0BDFC002016F0BAFC3B68DFF80E
:1083E8009CA0DFF88C905E2098473B68282098472F
:1083F800DAF8003089FB0329DB17C3EBA9095FFA18
:1084080089F016F0A5FCC9F3072016F0A1FC3B681B
:108418005E2098473B6804209847B8F80830002B3E
:1084280040F0F882DAF8083083F310085FFA88F031
:1084380016F08EFCC8F3072016F08AFCFFF7A0BAE6
:108448002C600020F26600209C380020A8550020EF
:10845800B6460020030820809C460020BC46002029
:108468000AD7233CE827002048560020310CC330A7
:1084780067666666565600201F85EB519C5500209E
:10848800B849B94B0093A1F13F06B84BB84A0991D6
:1084980001F8404C0AA8B7490896FAF717FF089E52
:1084A800731C08933470089B2922591C08911A7070
:1084B800089BEA22591C08911A70089BC822591C6B
:1084C80008910AA81A7023F08BFD471C0AA93A469E
:1084D800089824F07DFD089AD31901330893D455E0
:1084E800089B5A1C08921C70089B5A1C08921C7006
:1084F800089B5A1C08921C70089B5A1C08921C70F6
:10850800089B5A1C08921C70089B5A1C08921C70E5
:10851800089B5A1C08921C70089B5A1C08921C70D5
:10852800089B5A1C08921C70089B5A1C08921C70C5
:10853800089B5A1C08921C70089B5A1C08921C70B5
:10854800089B0122991812A808911A7050F8283D22
:108558009B1B337011F0BAFB874B029A2C70C3F83F
:10856800A022FEF76FBA029BC4F8283187F8008072
:10857800FEF7DFB99BF80240C4B1013CE4B2013414
:108588005C445946002211F8013B534083EA031327
:10859800DBB2120ADF0042EA03228C4287EA131395
:1085A80082EA0302EFD1002A7FF4CAAC734A744FFF
:1085B800744B12887449704CFA61DFF8E0911A68BC
:1085C80009689B68FA62B4F85221F866FB64D9F826
:1085D8000000F963FA65FBF7D5FE824600287EF4B1
:1085E80015AA0221D9F80000F8F75BFC94F8543179
:1085F8009BF803200492642B4FF0040287F8742040
:1086080040F04C8294F85531072B08BF84F855A1E7
:1086180094F85531069307EB031ADAF8041003911E
:10862800084623F0DDFCDAF8081005915FFA80FAB5
:10863800084623F0D5FC5FFA80FB069B5348039954
:1086480003900AEB0B020832C27123F00F02827208
:108658004E4A03F00F0353734C4B0BEBCA0098734D
:10866800184652460F3024F0B3FC494B05990AF1DD
:10867800090018445A4624F0ABFC0398C37903F167
:10868800010ACBB1013B5FFA83FC0CF1080CDFF85F
:1086980010E184440023073010F8012B5A4093005E
:1086A800D10883EA420301F0180153404EFA01F25F
:1086B80053408445DBB2EFD1354A04980AF80230BA
:1086C80014F080FA94F855310022013384F85531BA
:1086D80084F85421039BDDF80CA09B785BB11AF851
:1086E8000510D9F80000F8F7E8FB01359AF80230D0
:1086F800EDB2AB42F3D894F854310322013384F835
:10870800543187F8742088F80020FFF7E2B8F8F7AA
:10871800C8FBFEF723B91F4A1268D2067FF521A9C4
:108728008046FFF721B91023042218460AA98DF8BC
:108738002A908DF82B908DF82C908DF82D908DF82F
:1087480028308DF8292016F03DFA84F83791FEF785
:1087580045B90621104816F017F984F84601FFF7C5
:10876800FBB900BF244700205960002034210308CA
:108778003C21030848210308E8270020A8550020C9
:10878800180000209C550020BC460020E04F002027
:10879800E64F0020706B002022290020A4640020EE
:1087A8000007090EAB4BAC4A0B93A3F140071268C4
:1087B800002103F8401C2123BB70D30040F108813D
:1087C800A6490326A64B1B88580500F1FE80DA0748
:1087D80000F10E8103F00203A24A002B1CBF0326FE
:1087E8001146DFF8B0823246404624F0F1FB06EB32
:1087F800080312A80133A8F1020140F8203D002225
:108808005B1A06F808207B7011F060FAFEF7CBB906
:10881800954AD278002A0CBF4FF0040C4FF0050C93
:10882800FEF734BE914B1988FFF751BB0123D9F8E5
:1088380000003B70F8F73BFB0746D9F80000F8F753
:1088480036FB7F067EF475A88E287EF472A89AF807
:108858000030002B7EF489A8854B864A1A602D23A8
:1088680084F82C31FEF76CB87A4B804A0B9312AF20
:10887800A3F13D0047F8200D1188DFF80482A3F129
:10888800400200204FF00A0E03F8400C082382F83B
:1088980001E038469370FAF71EFCD8F800307649A4
:1088A800DA1781FB0313C2EBA30399B23846FAF730
:1088B80012FC09F0C5FDD8F808800A9B4FEA184257
:1088C800591C0A911A700A9B4FEA1822591C0A91DE
:1088D8001A700A9B5A1C0A9283F800800A9B5A1C39
:1088E8000A921870384611F0F1F9FEF759B9DFF815
:1088F800A8819FED628AB8F90230564A0B9207EEBA
:10890800903AF8EEE77A12AF67EE887AA2F1400360
:10891800FDEEE77AA2F13D0147F8201D02F8400C70
:108928000822CDED037A5A701E229A70BDF80C10F9
:108938003846FAF7D0FBB8F9003007EE903AF8EE6F
:10894800E77A384667EE887AFDEEE77ACDED037A66
:10895800BDF80C10FAF7BFFBB8F9043007EE903AEF
:10896800F8EEE77A384667EE887AFDEEE77ACDEDDD
:10897800037ABDF80C10FAF7AEFB384611F0A6F9E9
:10898800FEF70BB939499A790B8803EB830303EB9C
:1089980083034FEA83081FFA88F8002A00F025812C
:1089A800374B1B680FFA83FA09F04AFD40B2FEF70D
:1089B8008BB9984699461846049305930393FEF796
:1089C8007BBA4FF03408FFF7E7BB03262D4908E7C9
:1089D8002D4B2E4A1B68214903F48003002B0ABF44
:1089E800114603260426EDE64FF02408FFF7D4BB12
:1089F80027490426F5E64B1CDBB2042B84F84931E1
:108A08004FEA01617FF4D5A9FFF7D0B94FF01008FC
:108A1800FFF7C2BB09F014FD16F09AF9002016F012
:108A280097F9FEF7ADBF4FF02008FFF7B5BB4FF041
:108A38000808FFF7B1BB3B685E2098473B683920C0
:108A480098475FFA89F016F083F94FEA192016F073
:108A58007FF9C3E424470020D046002018210308EA
:108A68002C600020302103089C380020A8550020E5
:108A78001C580020A44700206766666658A08B41F2
:108A88009C55002024210308706B00201C2103083A
:108A980028210308E74600203060002097F875A0D9
:108AA8005C491AF00F0F04BF0AF1010A5FFA8AFA4B
:108AB800BAF1070F28BF4FF0010A4FEA0A1B07EB6C
:108AC8000B035FFA8BFC187C534B03930A180023A3
:108AD80092F82410504A937202F10D0307EB0B022F
:108AE8004CEA000001291870D26803F1010E0CD974
:108AF8000239C8B2811C1944734603F8012B8B4212
:108B08004FEA1222F9D101308644BB4422F06003B7
:108B18000AF1010A9BF811205FFA8AFA1343BAF1A5
:108B2800080F8EF800300EF1010344D04FEA0A1BFB
:108B380007EB0B01394A087C364901449A1A91F827
:108B4800241002EB010E0CF1100CBEF1130F5FFAAA
:108B58008CFCC3DD5FFA82FB0BF10603DBB20398E2
:108B6800DFF8C4E043F04002C27103F1010CD3B155
:108B78000BF1050B5FFA8BFB0BF1080B8344002309
:108B88000EF1010010F8011B59408B0083EA4103E4
:108B9800CA084B40224902F0180241FA02F2534037
:108BA8008345DBB2EED104980CF80E3087F875A037
:108BB80014F008F88EE5194A9A1ACBE7194B904633
:108BC800B3F900A06420FEF77FB898469946184686
:108BD800049305939E460393FEF76EB9984699460B
:108BE800184604930393FEF767B94FF0FF33D9E6AD
:108BF8000393FEF761B998460393FEF75DB998466B
:108C080099460393FEF758B9984699461846039330
:108C1800FEF752B9A4F70208E04F0020ED4F0020FC
:108C28000007090E9C550020E64F00202DE9F04F63
:108C38002DED0C8B3C4B1B7895B0012B0A9001F065
:108C480049873A4C94F80021002A41F0EF80072B1D
:108C5800374D01F00D87002305936B68344898471A
:108C6800002800F06981B5F8B470002285F8552015
:108C7800002F40F03F87B5F93E00AA6AB5F93C607D
:108C8800696AB5F94030DFF8B4B0821AE86A6A63F5
:108C9800711A1B1A2963274895F85610AB6317F009
:108CA80089FBDBF80030990040F1F08095ED0D7AF2
:108CB800D5ED0C7A204A94ED715AD4ED725A94EDA0
:108CC800736AD4F8D0311268F8EEC76A95ED0E7A57
:108CD800F8EEE77AB8EEC77A013377EE857A36EEA2
:108CE800A58A77EE068A9342C4ED717A84ED728A7A
:108CF800C4ED738AC4F8D03101F03C840A4B1F7864
:108D0800142F03F0D9800023D4F8D8610693062ED7
:108D180000F2AF80DFE816F01F170B173C16A016FD
:108D280014006118FA1700BF38560020B42A002032
:108D3800DC6800200C690020645A0020706B002059
:108D4800D84B1A78D4F8DCE1DFF8CCC39FEDD67A9B
:108D58004FEACE000CEB000383ED007A002A7DD0A9
:108D6800D249B0EE476AF0EE476A0023F1EC017A87
:108D7800013367EEA77A05EE903AB4EEE77AF1EEA2
:108D880010FAF8EEE55AB8BFB0EE677A9A4276EE76
:108D9800A76AA7EEA56AE9D1F5EEC06A0CEB000355
:108DA800F1EE10FA83ED007A58DDC6EE265AC04B74
:108DB800C04A1288F7EE007A75EEE75AD3ED007ACA
:108DC80065EEA77AFDEEE77A17EE903A812B43F32A
:108DD800FC869342A8BF134607EE903AF8EEE77A6E
:108DE800B54B00EB0E0103EB810393ED057AD3ED50
:108DF800003A93ED066A93ED014AD3ED046AD3ED88
:108E0800034A93ED025AA3EEA77AA4EE276A66EE08
:108E1800C76AA7EE646ABDEEC77AE5EE276A17EE61
:108E2800101A812983ED056AC3ED066A43F3CA86E1
:108E38008A42A8BF0A4607EE902AF8EEE77AFCEEC7
:108E4800E77ACDED077ABDF81C300CEB0002938071
:108E5800BEF1000F02D1132F04F05083152F42F0FA
:108E6800EC856044DFF8B482838828F81E30D4F893
:108E7800D861924B013683FB06239A19F317C3EB8B
:108E8800A203C3EBC303F61AC4F8D8618C4B1B7852
:108E9800002B01F0D3818B4EDFF88492DFF87CA29F
:108EA80006F5BC780027884BD5ED087A1B78172B78
:108EB80001F0398496ED007AB8EEC78A082B28EEBF
:108EC800278A07D1B0EE480A069324F089FA069B50
:108ED8002AF81700DBF8002092000BD5002F04F0C9
:108EE800A187B0EE480AD5F8143208F17000984707
:108EF800B0EE408AB0EE480AD5F83431A8F17000D7
:108F08009847D5F8A431404698476F4B1B78032BF8
:108F1800B0EE408A01F01484D6F8F800D5F8B830DD
:108F2800B0EE480A98470137032F08F12408A9EC46
:108F3800010A06F10406B6D1634B93F80090B9F123
:108F4800070F00F0928694F8E031002B40F09A86E3
:108F58005E4B5B79002B40F0C78501235A4A84F8A1
:108F6800E0311278072A02F0D28100230B93584B84
:108F780094ED799A93ED007A564BD4ED41CA1B686B
:108F88000593F7EE007A37EEC9CA534B06932CEED9
:108F980007CA524B0893B4EEE7CA514B0993002510
:108FA800504BDFF88091DFF880B1DFED4F8A9FEDFD
:108FB8004FAADFED3DBADFED4E9A9FED4EBADFEDD9
:108FC8004EAADFF86881DFF868A14C4F0793F1EEED
:108FD80010FA88BFB0EE67CA2E46494B99ED008A51
:108FE8002B44D3ED007AF5EE407AF1EE10FA17D063
:108FF800444B2B44D3ED006A38EE667AB0EEC76A6C
:10900800F4EEC67AF1EE10FA08D5B5EEC07AF1EEB4
:1090180010FACCBF37EEA68A36EEE78A83ED008ACF
:10902800069B1A88930700F08580022E00F0828044
:109038000599354B91F82E102B4407EE901A93EDB5
:10904800007A4B42F8EEE76A07EE903A26EE877A06
:10905800F8EEE77AB4EEE77AF1EE10FA0AD407EE02
:10906800901AF8EE677AF4EEC77AF1EE10FA88BF34
:10907800F0EE477A254B264903EB460331F91600F3
:10908800B3F90C30C01A07EE100AB8EEC77AD00749
:10909800E7EE687A40F12C861E4B93ED008A27EEA6
:1090A800888A47E06A5A002000000000B42A00209D
:1090B8006C5A0020685A0020A05C00209324499232
:1090C800605A00200C69002038560020C86800202B
:1090D80044440020506000202C60002090000020B4
:1090E800F2660020606B0020CDCCCC3DAE47813FBE
:1090F8000000C84200003443610BB63B0849002019
:10910800384400209C2C0020502C0020184B0020B4
:109118003060002020440020885C00203C5600205D
:10912800646B0020E82B0020304300201449002005
:10913800FC480020079B94F8F4212B44D3ED01DA76
:1091480038EE6DDA002A38D0D54BD4F8F8210A99D0
:109158001B688A1A9A4230DD022E04F0AC85D14B86
:109168001B68990741F15E80CF4BD049DFF8ACE32B
:1091780031F916C09EED008ADFF8A4E3C7ED00BA06
:1091880003EB460028EE288AB0F90C00A0EB0C008F
:1091980007EE900AF8EEE77ADEF8000027EE888AF4
:1091A800824238EE6DDA01F39B82F7EE007AB4EE74
:1091B800E79AF1EE10FA01F16A82BD4B2B4493ED68
:1091C800000A2CEE800A022E20EE0D0AAAEC010AF3
:1091D80004F02F85089BDBED007A93ED007AB54B00
:1091E800D7ED006A93ED006AB34B67EE277A2B44FC
:1091F80027EE8C7AD3ED007A67EE277AF0EE665A7E
:10920800EDEE275AB1EE467AB4EEE57AF1EE10FAB1
:1092180008DCF4EEC65AF1EE10FA8CBFB0EE467ACE
:10922800B0EE657A94ED796AF7EE007AB4EEE76A03
:10923800F1EE10FAACBF0123002343B1F0EEE66A69
:10924800F0EEC77AF4EEE67AF1EE10FA01D587ED82
:10925800007A022E04F08F84984A994B52F826001F
:109268001B68B0EE6D0A9847964A974B52F826004D
:109278001B689847059B93F8373023B1069B1B88DA
:10928800002B00F09985B0EE6B8A904B9BED007A2D
:1092980038EE400A2B4493ED008A83ED000A059BC3
:1092A80030EE480A93F84830C0EE077A33B3099B8A
:1092B8001B78D80740F1128594F8F431B7EE007A9C
:1092C800B4EEC79AF1EE10FAC0F2E484002B40F035
:1092D800E4847F4A92ED007AF0EEE76AF4EEC76A1A
:1092E800F1EE10FA0ADD7B4A92ED007AF0EECD6AD3
:1092F800F4EEC76AF1EE10FA02F3F385764B94F8B0
:1093080004222B4493ED007A2CEE877A67EE277AB5
:10931800C8ED007A2AB94AED01BAC7ED00BAC8ED1E
:1093280000BA0136032E09F1040908F1040807F10F
:10933800040705F104057FF450AE684B1B78072B32
:1093480001F01284012B01F0E787002594F80C3214
:10935800002B40F03187624A624B10681B6810F49A
:10936800805E93F82C3040F093875F4A5F4992ED16
:10937800006A498B5E4A84ED876A92ED007A5D4AFD
:1093880084ED887A07EE901AF8EEE76AD2ED037A50
:10939800594A84ED856A37EE467A77EEE67AD2ED59
:1093A800006A84ED847A012284F82422C7EEA65A42
:1093B8005249534A91ED005A52499FED536A91ED33
:1093C800004A5249DFED526AD1ED004A92ED007A27
:1093D80035EE045AF7EE007AF4EEE75A35EE245AE1
:1093E800F1EE10FA88BFF0EE675A25EE065AF4EE51
:1093F800E65AB1EE476AF1EE10FAB4EEC65AB8BFB3
:10940800F0EE665AF1EE10FAC4ED8A5A01F1848141
:10941800B4EEC75AF1EE10FA88BFB0EE475A374A91
:10942800DFED396AD2ED017A364A92ED014A374AC0
:1094380077EE847AD2ED014A77EEA47A67EEA67ABF
:10944800B4EEE76AF1EE10FA08DCB4EEE77AF1EE72
:1094580010FA8CBFB0EE676AB0EE476A274ADFEDB4
:109468002A6AD2ED027A274AD2ED024A294A77EED1
:10947800A47A92ED007A67EEA67AB1EE473AF4EE56
:10948800C37AF1EE10FA08D4F4EEC77AF1EE10FAC6
:109498008CBFB0EE473AB0EE673A1F4A527841E0C7
:1094A8004C440020D8460020184B00203060002093
:1094B800F443002068440020004400203843002082
:1094C800344300208C43002088430020B02C002027
:1094D8005C440020584400200C44002038560020EA
:1094E800706B0020506000209C4900207C4F0020B9
:1094F800FC4A00205856002028450020FC4800203F
:109508006C440020084900206F12833A1449002057
:109518000000000070440020544B0020204400202C
:10952800484400200AB9B1EE433A002B41F0F084D8
:10953800F7EE003AF04E3278002A03F03380EF4B12
:10954800DFEDEF7AD3ED024AD3ED016A93ED037AAA
:1095580066EE244AE5EE264AE3EE074A63EEA44A9D
:10956800F4EEE74AF1EE10FAB4BFB0EE674AB0EE97
:10957800644A98BFF0EE647A012ACDED0C4A03F0F4
:10958800368093ED067AD3ED052AD3ED076A26EEE9
:10959800077AA5EE227AA3EE267A23EE877AB4EE2E
:1095A800E77AF1EE10FAB4EEC47A8CBFF0EE676A8F
:1095B800F0EE476AF1EE10FA88BFF0EE676AB4BFC2
:1095C800F0EE447AF0EE477A022A8DED0D7A00F03B
:1095D800DE8093ED0A7AD3ED092A93ED0B4A26EE45
:1095E800077AA5EE227AA3EE047A23EE877AB4EE00
:1095F800E67AF1EE10FAB4EEE77A8CBFB0EE664A7E
:10960800B0EE474AF1EE10FA98BFF0EE446AA8BFF0
:10961800F0EE477A032A8DED0E7A00F0B88093EDCC
:109628000E7AD3ED0D2A93ED0F4A26EE077AA5EEB2
:10963800227AA3EE047A23EE877AB4EEE67AF1EE84
:1096480010FAB4EEE77A8CBFB0EE664AB0EE474A3D
:10965800F1EE10FA98BFF0EE446AA8BFF0EE477A30
:10966800042A8DED0F7A00F0928093ED124AD3ED23
:10967800112A93ED137A26EE044AA5EE224AA3EEA8
:10968800074A23EE844AB4EEE64AF1EE10FAB4EE45
:10969800E74A8CBFB0EE667AB0EE447AF1EE10FA83
:1096A80098BFF0EE476AA8BFF0EE447A052A8DED20
:1096B800104A6CD093ED164AD3ED152A93ED177A1C
:1096C80026EE044AA5EE224AA3EE074A23EE844A70
:1096D800B4EEE64AF1EE10FAB4EEE74A8CBFB0EE0B
:1096E800667AB0EE447AF1EE10FA98BFF0EE476A67
:1096F800A8BFF0EE447A062A8DED114A47D093EDC3
:109708001A4AD3ED192A93ED1B7A26EE044AA5EEE0
:10971800224AA3EE074A23EE844AB4EEE64AF1EE63
:1097280010FAB4EEE74A8CBFB0EE667AB0EE447A2F
:10973800F1EE10FA98BFF0EE476AA8BFF0EE447A4F
:10974800072A8DED124A22D093ED1E7AD3ED1D2AF9
:1097580093ED1F4A26EE077AA5EE227AA4EE037A45
:1097680027EE237AB4EEE67AF1EE10FAB4EEE77A51
:109778008CBFB0EE666AB0EE476AF1EE10FA8DED76
:10978800137A98BFF0EE466AA8BFF0EE477A77EEF4
:10979800E67AF7EE006AF4EEE67AF1EE10FAC4ED36
:1097A800797A43F3938686EEA77A022ADDED0D7A5D
:1097B80067EE244A67EE877ACDED0C4ACDED0D7A37
:1097C8002DD0DDED0E7A67EE877A032ACDED0E7A7D
:1097D80025D0DDED0F7A67EE877A042ACDED0F7A72
:1097E8001DD0DDED107A67EE877A052ACDED107A67
:1097F80015D0DDED117A67EE877A062ACDED117A5C
:109808000DD0DDED127A67EE877A072ACDED127A50
:1098180005D0DDED137A27EE877A8DED137A394B73
:109828001F6817F0805701F06E81F6EE005AC4EDFC
:109838008A5A002A02F0AB86334B94ED885A93F883
:10984800039094F924320999D4ED874A91F800C01D
:10985800DFF8C0802D49DFF8C0A0B1F9061098EDF7
:10986800007A059106EE903ABDEEC55A284B9AF853
:1098780000A0B3F81AB094ED846AD4ED857A15EE99
:10988800103ABDEEE45A00F0100800F480000CF025
:10989800010CF8EEE66A15EE101A0690B9F1000F01
:1098A80041F06A83B8F1000F41F07381DFF84C8012
:1098B8009DED0C5A98ED007ADFF860E025EE877A86
:1098C800A6EE857AB0EE675AA6EE075ABDEEC57ABF
:1098D80017EE107A17EE100A9F42A8BF1846B94231
:1098E800C8BF084607EE100AB8EEC77A012A8EEDFF
:1098F800007A00F0F18013E04C54002098440020D6
:1099080000000000D04600209C380020D0540020E1
:109918007C4F002074440020544C00205C490020F7
:1099280098ED047A9DED0D5A25EE877AA6EE857A94
:10993800B0EE675AA6EE075ABDEEC57A17EE107A52
:1099480017EE100A9F42A8BF1846B942C8BF08467A
:1099580007EE100AB8EEC77A022A8EED017A00F0F7
:10996800BB8098ED087A9DED0E5A25EE877AA6EE13
:10997800857AB0EE675AA6EE075ABDEEC57A17EE9D
:10998800107A17EE100A9F42A8BF1846B942C8BFFE
:10999800084607EE100AB8EEC77A032A8EED027A57
:1099A80000F09A8098ED0C7A9DED0F5A25EE877A93
:1099B800A6EE857AB0EE675AA6EE075ABDEEC57ACE
:1099C80017EE107A17EE100A9F42A8BF1846B94240
:1099D800C8BF084607EE100AB8EEC77A042A8EED0B
:1099E800037A79D098ED107A9DED105A25EE877A92
:1099F800A6EE857AB0EE675AA6EE075ABDEEC57A8E
:109A080017EE107A17EE100A9F42A8BF1846B942FF
:109A1800C8BF084607EE100AB8EEC77A052A8EEDC9
:109A2800047A59D098ED147A9DED115A25EE877A6B
:109A3800A6EE857AB0EE675AA6EE075ABDEEC57A4D
:109A480017EE107A17EE100A9F42A8BF1846B942BF
:109A5800C8BF084607EE100AB8EEC77A062A8EED88
:109A6800057A39D098ED187A9DED125A25EE877A45
:109A7800A6EE857AB0EE675AA6EE075ABDEEC57A0D
:109A880017EE107A17EE100A9F42A8BF1846B9427F
:109A9800C8BF084607EE100AB8EEC77A072A8EED47
:109AA800067A19D098ED1C7A9DED135A65EE875AFF
:109AB800E6EE855AE6EE257AFDEEE77A17EE900A8D
:109AC8008342A8BF03468142C8BF0B4607EE903ABF
:109AD800F8EEE77ACEED077ABCF1000F40F0798313
:109AE800002A40F0718374E3C14B1B78013BDBB261
:109AF800FFF734BABF4B07934FF47A761B68B6FB6F
:109B0800F3F3C3EB4316BC49DFF81C8391F801A0BB
:109B1800BA49B8F9060091F8009003EB8603DE0015
:109B2800B6B2B74202F0AA82D5F88810B5F93CE07F
:109B3800EB6E4A1C07EE90EA7344012AC5F88820A8
:109B4800EB66F8EEE77A02F0A482D5ED1E5AD5ED61
:109B5800206A07EE102A37EEE56AB8EEC75A012FD9
:109B680086EE057A37EE257A77EEC77A85ED1F7A85
:109B7800E7EE866A85ED1E7AF0EE667AC5ED216A13
:109B8800C5ED206A02F06A86D5F89C10B5F93EE06A
:109B98002B6F4A1C07EE90EA7344012AC5F89C20F3
:109BA8002B67F8EEE77A02F08D82D5ED235AD5EDD2
:109BB800256A07EE102A37EEE56AB8EEC75A012F74
:109BC80086EE057A37EE257A77EEC77A85ED247A20
:109BD800E7EE866A85ED237AF0EE667AC5ED266AA9
:109BE800C5ED256A02F06286D5F8B010B5F940E0F7
:109BF8006B6F4A1C07EE90EA7344012AC5F8B0203F
:109C08006B67F8EEE77A02F07682D5ED285AD5ED43
:109C18002A6A07EE102A37EEE56AB8EEC75A012F0E
:109C280086EE057A37EE257A77EEC77A85ED297ABA
:109C3800E6EE276A85ED287AF0EE667AC5ED2B6A9E
:109C4800C5ED2A6A02F05B86A8F806006B4B013F57
:109C580093F80090A5F8B47007990023B9F1070F9D
:109C68004B608B60CB607FF46EA9FCF7EDFB059B26
:109C7800DFF8B481C01A94F8E031A8F80000002B8E
:109C88003FF466A9013B84F8E03115B0BDEC0C8BBC
:109C9800BDE8F08F002B3FF431ABD4F8F8310A9AC5
:109CA800D31A574A12689A427FF728AB554B93ED5F
:109CB800007AB0EECDDAB4EEC7DAF1EE10FA12D4CB
:109CC800514B99ED007AD3ED006AB0EEC77AB4EE45
:109CD800E67AF1EE10FA7FF711AB04E094F8F4316C
:109CE800002B3FF40BAB002384F8F431FFF706BBDD
:109CF800B1F9002094ED6A7AB1F90200D4ED6B6AEB
:109D0800424982EAE273A3EBE273F4EEC76A80EA9F
:109D1800E072F1EE10FAA2EBE072B8BFF0EE476A1B
:109D28009342B8BF134607EE103A0B78B8EEC77ADD
:109D380027EE287A002B40F0EE82354B93ED006A2F
:109D4800B4EECA6AF1EE10FA41F13282F7EE005A27
:109D580075EEC65A3BEE477A65EEAA5A2D4BA7EE2A
:109D6800256A93ED007A26EE076AB5EEC06AF1EE31
:109D780010FA40F2C486C9EE865AB7EE007AB0EE01
:109D8800476AA6EEE56AF0EE466AF4EEC76AF1EEB7
:109D980010FA88BFF0EE476AF5EEC06AF1EE10FAE5
:109DA800B8BFF0EE6B6A1C4B93ED007A67EE877ACA
:109DB800A7EEA68AFFF7BEB9184B194A2B4493EDB4
:109DC800007AD2ED007A174B67EE277AF7EE006A31
:109DD800F4EEE67AF1EE10FA93ED007A88BFF0EE31
:109DE800667A67EE877A27EE888AFFF74EBA00BF51
:109DF8000C4B0020606B0020C868002038560020FB
:109E08004C44002058440020604400202C4400208A
:109E18003444002028440020244400205C2C0020E6
:109E28001C440020184400203C560020072B02F058
:109E3800D98300230793CF4ECF4D33680693590536
:109E480001F11382CD4BCE491F68B1F906807A899A
:109E58009045C0F28F82B8F5FA6F81F27382387A32
:109E6800A8EB020303FB00F3C2F5FA6293FBF2F3DB
:109E7800C3F1640307EE903AF8EEE77A9FEDC17AF2
:109E880067EE877AC4ED417ADFF82093DFF820A3E4
:109E9800B9F818B0B1F900309AF904209AF800001E
:109EA8009AF801C0A3EB0B0686EAE67E002AAEEB21
:109EB800E67E14BF01224FF0FF32BEF5FA7FA8BF3D
:109EC8004FF4FA7E704580F20186AEEB000607EE8D
:109ED800906AF8EEE77AAC4E5B45C6ED007A03DA95
:109EE800F1EE677AC6ED007AB1F902E0AEEB0B034A
:109EF800002BB8BF5B42B3F5FA7FA8BF4FF4FA73E3
:109F08009842059380F2B9851B1A07EE903AF8EE4D
:109F1800E77ADE45C6ED017A03DAF1EE677AC6ED37
:109F2800017AB1F90410A1EB0B0383EAE370A0EB0B
:109F3800E370B0F5FA7FA8BF4FF4FA706045CCBF64
:109F4800A0EB0C0C4FF0000C02FB0CFC07EE90CAC7
:109F5800F8EEE77A5945069BC6ED027ABCBFF1EEEA
:109F6800677AC6ED027A13F48053059300F0898569
:109F7800B8F5FA6F4246A8BF4FF4FA62B2F57A7F95
:109F880094F80831B8BF4FF47A72A2F57A72002BB0
:109F980040F090857D49DFF81CE281FB0230D31741
:109FA800C3EB6013581C6FF0630C3EF910003EF9C8
:109FB80013E00CFB0323A0EB0E0003FB00F381FB73
:109FC8000321DB17C3EB61139E440FFA8EFE07EEE5
:109FD80090EA059BB8EEE78A86ED038A002B41F0EC
:109FE80069816B4B1A8812F0400B40F0E086694B90
:109FF8001B6813F0140F03D012F4027F41F0A981FB
:10A00800654B1B789BB1B9F81A3043450FDB634B9E
:10A018001B78012B02F09B80192B02F098800E2BE5
:10A0280005D0082B03D00023B360C4F83C3194F862
:10A03800423113B1920742F06E8294F84831002BF6
:10A0480041F0BB8099F81E20002A00F09383022A71
:10A0580002F0A080032A01F06E83514A518899F8D2
:10A068001F200232D2B2002B02F08680002902F0B3
:10A0780083804C480068B1FBF0FA0FFA8AFAA4F81A
:10A0880078A1AAB307EE90AAF8EEE77AF7EE006A8D
:10A0980086EEA77A012AD6ED007AD4ED636A77EEC8
:10A0A800E67A67EE877AC4ED5F7A21D0D6ED017A39
:10A0B800D4ED646A77EEE67A022A67EE877AC4ED11
:10A0C800607A15D0D6ED027AD4ED656A77EEE67A35
:10A0D800032A67EE877AC4ED617A09D0D6ED037A50
:10A0E800D4ED666A77EEE67A67EE877AC4ED627A2F
:10A0F8002D490978092903F0CE82BAF1000F40F3FF
:10A108003F8392B394ED637AD4ED5F7A77EE877AE2
:10A11800012AC4ED637AC6ED007A21D094ED647A01
:10A12800D4ED607A77EE877A022AC4ED647AC6EDB8
:10A13800017A15D094ED657AD4ED617A77EE877A55
:10A14800032AC4ED657AC6ED027A09D0D4ED667AA1
:10A1580094ED627A77EE877AC4ED667AC6ED037A73
:10A16800013A022AB8BF0222D2B2002B18BF02223B
:10A1780007E300BF706B0020DC680020E85E002069
:10A18800D05400200AD7233C585600201F85EB5195
:10A198002C600020D8460020190C0020544B0020C9
:10A1A8008C3700203C4B0020385600207C4F002084
:10A1B800104B0020EC5E0020099BD84E1B78D90775
:10A1C80000F1DD80327822B19200D549D54822F0DD
:10A1D800FFFED54B1B68002B40F0A282D34B1B78A7
:10A1E8009BB1307870B1DFF83C83DFF87C930027AF
:10A1F800F8B2D9F80030B8EC010A9847307801373E
:10A208008742F5DBCA4B1B689847CA4B1B78072B5C
:10A2180000F07E84012384F8003115B0BDEC0C8B6E
:10A22800BDE8F08FC44BC7ED00BA1B689342BEF679
:10A23800BCAF002384F8F431FEF7BFBFBF4EDFF890
:10A248002C9306F5F47806F51577F6EC017A95ED7A
:10A25800080AD5F81432F8EEE77A404627EE800A65
:10A268009847A8F1E000D5F834319847A8F1700074
:10A27800D5F8A4319847D6F8F400D5F8B8309847FF
:10A2880008F124084745A9EC010ADED1FEF754BEBF
:10A29800099A1278D20703D4A94A128BA4F8182273
:10A2A800A84AA949128891ED037A07EE902AF8EE98
:10A2B800E77AB4EEE77AF1EE10FA41F22B81A3497E
:10A2C800098807EE901AF8EEE77AB4EEE77AF1EE2D
:10A2D80010FAC1F2A0809E499E4AD1ED006A92ED23
:10A2E800006A9D49C4ED876ABCEEC75A76EE665A85
:10A2F80015EE102AC4ED856AC4ED845A84ED886A87
:10A30800A4F818220122D1ED006A84F8242277EEFD
:10A31800677AFFF74BB8914B93ED005AB5EEC05AE8
:10A32800F1EE10FA40F3EB838D4BD3ED004AF5EED6
:10A33800C04AF1EE10FA40F3E28334EEC77A66EED3
:10A34800E95A87EE246AC5EE856AB7EE007AB4EE5C
:10A35800C76AF1EE10FA88BFB0EE476AB5EEC06A78
:10A36800F1EE10FA76EE876AB8BFB0EE6B6A66EE69
:10A37800266A0AE54FF07E53C4F8043184E5337841
:10A38800002B3FF426AFD4ED6B3A94ED6A6AD4ED16
:10A39800857A744A94ED847AD2ED005A94ED684A2D
:10A3A800D4ED674ADFF8C881DFF878E1F4EEC63A01
:10A3B800F3EE046AF1EE10FA37EEA65A01F10C81B9
:10A3C80098ED026A26EE446AF0EE674AE6EE074A1E
:10A3D800F4EEC54A34EEE66AF1EE10FA48BFB0EE84
:10A3E800656A012B8EED006A3FF4F3AE98ED066ABC
:10A3F80026EE446AF0EE674AE6EE074AB4EEE45AFF
:10A4080034EEE66AF1EE10FA88BFB0EE656A022B08
:10A418008EED016A3FF4DDAE98ED0A6A26EE446AD5
:10A42800F0EE674AE6EE074AF4EEC54A34EEE66A0D
:10A43800F1EE10FAB8BFB0EE656A032B8EED026A32
:10A448003FF4C7AE98ED0E6A26EE446AF0EE674A0E
:10A45800E6EE074AB4EEE45A34EEE66AF1EE10FA94
:10A46800C8BFB0EE656A042B8EED036A3FF4B1AE47
:10A4780098ED126A26EE446AF0EE674AE6EE074A5D
:10A48800F4EEC54A34EEE66AF1EE10FAB8BFB0EE63
:10A49800656A052B8EED046A3FF49BAE98ED166A4B
:10A4A80026EE446AF0EE674AE6EE074AF4EEC54A3D
:10A4B80074EEE66AF1EE10FAB8BFF0EE656A062BA4
:10A4C800CEED056A3FF485AED8ED1A6A66EEC46A29
:10A4D800F0EE674AE6EE874AB3EE046AB4EEE45A51
:10A4E80074EEC66AF1EE10FAC8BFF0EE656A072B83
:10A4F800CEED066A3FF46DAED8ED1E6A26EEC44A6C
:10A50800E4EE077AF4EEC57A77EEC67AF1EE10FA41
:10A5180048BFF0EE657ACEED077A5AE64C54002033
:10A52800784400205C4900202C4300205C4F002028
:10A53800504C002038560020484400200C69002068
:10A548007C4F00202C450020585600202E45002026
:10A5580018450020FC4A00203445002028440020EB
:10A568003044002074440020484C0020646B0020D4
:10A578009844002007EE103A744BDFF8F0811B78FE
:10A58800C4F8D071B8EEC77AB7EE005A132B85EE2F
:10A59800079AB8F90400B4F8D46195ED080A01F0F7
:10A5A800D4846B4B6B4A93ED001AD3ED053A93EDC7
:10A5B800122A93ED173AD3ED091AD3ED0E4A93ED0B
:10A5C800016A93ED064A93ED0A7AD3ED0F5AD3ED5B
:10A5D800132AD3ED186A93ED045AD3ED030A67EEF4
:10A5E800897A69EE288A29EE088AE1EE273A02EB91
:10A5F80086070021A2EE283AC4F8C411C4F8C8118D
:10A60800E1EE884AA6EE274AE7EE085A93ED167A55
:10A6180093ED0D6A93ED021AD3ED0C1AC7ED003ACB
:10A62800E2EEA86A25EE635A27EE437A93ED0B2AE9
:10A63800D3ED152AC7ED204AA0EEE34A26EE646A58
:10A64800D3ED143A83ED054AA1EE275AF0EE477A86
:10A65800E1EEE45AA2EE086AE2EEC36AE3EEA87AF3
:10A6680083ED065AC3ED0E5A83ED0F6A87ED403A23
:10A67800C3ED176AC3ED187AC4F8CC11731C03F044
:10A688001F03A4F8D431A8F80400FEF737BB0799D4
:10A69800314BD1ED017A93ED007AF0EEE77AF4EEE2
:10A6A800C77AF1EE10FA7EF588ADD1ED027AF0EEB8
:10A6B800E77AB4EEE77AF1EE10FA7EF77EADD1EDE7
:10A6C800037AF0EEE77AB4EEE77AF1EE10FA7EF765
:10A6D80074AD224B1B689B077FF5ABAD2049214B1E
:10A6E800B3F90C20B1F900E01F48AEEB020E006888
:10A6F8008EEAEE72A2EBEE728242BEF65EADB3F95E
:10A708000E30B1F90220D21A82EAE273A3EBE273A7
:10A7180098427EF752AD8CE5B0EE465AFEF77FBE02
:10A728000DF070F85AE596ED007A05EB4702B8EEA1
:10A73800C78A928F2AF8172028EE278AFEF7CABB05
:10A7480022F04EFE2AF81700FEF7E6BB3856002026
:10A758000C5D0020885A002054440020D846002070
:10A7680030600020184B0020504400203C56002048
:10A778000AD7233CA4F878219246002B00F0658183
:10A7880002223B785FED066AB97807EE903AF8EE58
:10A79800E77AB0EE007A67EEA67AE14BF4EEC77A74
:10A7A800F1EE10FA187840F3E48337EEC77ADFED5C
:10A7B800DD6AB0EE676AA7EE266AB0EE467A9FEDCC
:10A7C800DA6AD6ED006A66EE866AB0EEE66AC4ED2D
:10A7D800676A84ED6A6A99B105EE901AB8EEE55A8F
:10A7E800DFEDD25A66EEA64A25EE255AF7EE005A54
:10A7F80075EEC55A64EE864AE4EE855A66EEA56A99
:10A80800DFEDCB5A7B7927EE257A27EE267ACBB176
:10A81800DFEDC66ADFEDC75A26EE266A06EE903AE5
:10A82800F8EEE66A26EE266AB4EEE56AF1EE10FA6C
:10A8380000F3A586F7EE005A35EEC66AC5EE866ABD
:10A8480027EE267A0C289FEDBC8ADFEDBC6A00F063
:10A858001786B4EEC87AF1EE10FA98BFB0EE478AC0
:10A86800B4EEE68AF1EE10FAB8BFB0EE668A84ED6F
:10A878004D8A002A00F0DE80B0EE007AF4EEC77A46
:10A88800F1EE10FA05DD37EEC77ADFEDA66AE7EEDE
:10A89800267A96ED017ADFEDA46A27EE267AB0EEE5
:10A8A800C76A84ED687A84ED6B6A99B106EE901AEE
:10A8B800DFED9E5AF8EEE66A27EE075A66EEA56ABD
:10A8C800F7EE005A75EEE65A25EE065AE5EE265AD8
:10A8D80027EE257ADFED966ABB7967EEA67A67EEF2
:10A8E800877AABB107EE103AB8EEC77ADFED8F5A28
:10A8F800DFED906A27EE067A27EE257AB4EEE67A3F
:10A90800F1EE10FA40F32D86DFED8D6A67EEA67A38
:10A918000C2800F0D285DFED886A9FED887AF4EE86
:10A92800E67AF1EE10FA88BFF0EE667AF4EEC77AAE
:10A93800F1EE10FAB8BFF0EE477A012AC4ED4E7A6C
:10A9480078DD7B78DFED796A07EE903AF8EEE77A02
:10A95800B0EE007A67EEA67A7B7AF4EEC77AF1EE6B
:10A9680010FA05DD37EEC77ADFED6E6AE7EE267A74
:10A9780096ED027ADFED6C6A27EE267AB0EEC76AAA
:10A9880084ED697A84ED6C6A9BB106EE903ADFED4E
:10A99800675AF8EEE66A27EE075A66EEA56AF7EEFA
:10A9A800005A75EEE65A25EE065AE6EE855A27EE67
:10A9B800257ADFED5F6AFB7967EEA67A67EE877A1C
:10A9C8000BB307EE103AB8EEC77ADFED585ADFED51
:10A9D800596A27EE067A27EE257AB4EEE67AF1EE82
:10A9E80010FA0CDCB5EEC07AF1EE10FA01F1BA8378
:10A9F800B7EE006A36EE477AC6EE076A01E0DFED89
:10AA0800506A67EEA67A0C2800F03085DFED4A6AB6
:10AA18009FED4A7AF4EEE67AF1EE10FA88BFF0EE8E
:10AA2800667AF4EEC77AF1EE10FAB8BFF0EE477A1C
:10AA3800C4ED4F7A092800F00D8599F82160002EA1
:10AA480040F0A484002384F848313E4B1B7823B996
:10AA58003D4EB378002B41F0F083314B1B78072B28
:10AA680000F04C850022072B84F800217EF4F3A81F
:10AA7800FBF7EAFC0590FEF7F0B8DFED347AFFF754
:10AA880048BAB9F81A209045C0F25984B8F5FA6F57
:10AA9800D4BFC2EB0803C2F5FA634FF47A7101FB25
:10AAA80003F194F80801C2F5FA63B1FBF3F2002848
:10AAB8003FF470AA94F80931254902FB03F281FB9F
:10AAC8000213D217C2EB6312FFF764BADFED1F7AE5
:10AAD800FFF701BA1F4B204C1A68204BDFF884801F
:10AAE80094F80001D2691B88A8F80020A8F8023061
:10AAF80000287FF49EA90590194DFEF7AEB8DFED4A
:10AB0800136AFFF750B943023EF58FAEFEF791BEC8
:10AB1800FBF79AFC134B401BD880FFF77BBB00BFA9
:10AB280038560020D7A368416F12033B0AD7233C4D
:10AB380000004843A4707D3F00C0F94400C0F9C438
:10AB48000000C842D93A0020B046002000000000AA
:10AB58001F85EB51EC480020B42A00209C410020BE
:10AB6800DC6800203C560020FBF76EFCD64B0B9AA5
:10AB78001B78DFF89083801A012BA8F8020000F0F8
:10AB8800CD83072B7EF4E1ABFBF75EFC0546FEF7B1
:10AB9800DDBBDFF87483BCF1000F41F03A8598ED16
:10ABA800007A9DED0C5ADFF864E325EE877AA5EE6E
:10ABB800267AB0EE675AA7EE065ABDEEC57A17EEAA
:10ABC800107A17EE100A9F42A8BF1846B942C8BFAC
:10ABD800084607EE100AB8EEC77A012A8EED007A09
:10ABE8003FF4F2AA98ED047A9DED0D5A25EE877A86
:10ABF800A5EE267AB0EE675AA7EE065ABDEEC57ADC
:10AC080017EE107A17EE100A9F42A8BF1846B942ED
:10AC1800C8BF084607EE100AB8EEC77A022A8EEDBA
:10AC2800017A3FF4D1AA98ED087A9DED0E5A25EEE7
:10AC3800877AA5EE267AB0EE675AA7EE065ABDEED9
:10AC4800C57A17EE107A17EE100A9F42A8BF184669
:10AC5800B942C8BF084607EE100AB8EEC77A032AF9
:10AC68008EED027A3FF4B0AA98ED0C7A9DED0F5A5A
:10AC780025EE877AA5EE267AB0EE675AA7EE065A31
:10AC8800BDEEC57A17EE107A17EE100A9F42A8BFDC
:10AC98001846B942C8BF084607EE100AB8EEC77A88
:10ACA800042A8EED037A3FF48FAA98ED107A9DED71
:10ACB800105A25EE877AA5EE267AB0EE675AA7EEE7
:10ACC800065ABDEEC57A17EE107A17EE100A9F42A3
:10ACD800A8BF1846B942C8BF084607EE100AB8EE22
:10ACE800C77A052A8EED047A3FF46EAA98ED147A95
:10ACF8009DED115A25EE877AA5EE267AB0EE675AB1
:10AD0800A7EE065ABDEEC57A17EE107A17EE100AAE
:10AD18009F42A8BF1846B942C8BF084607EE100AA6
:10AD2800B8EEC77A062A8EED057A3FF44DAA98ED5B
:10AD3800187A9DED125A25EE877AA5EE267AB0EE9E
:10AD4800675AA7EE065ABDEEC57A17EE107A17EEC7
:10AD5800100A9F42A8BF1846B942C8BF084607EE66
:10AD6800100AB8EEC77A072A8EED067A3FF42CAAA5
:10AD780098ED1C7A9DED135A65EE875AE6EE855AD2
:10AD8800E6EE257AFDEEE77A17EE900A8342A8BF31
:10AD980003468142C8BF0B4607EE903AF8EEE77AC1
:10ADA800CEED077A002A7FF40FAAFFF712BA474BB5
:10ADB8004748B3F90430B4F81011DFED466A9FED47
:10ADC800467A80FB03E0DB17C3EBA0035B1A1BB2D8
:10ADD80007EE903AF8EEE77A67EEA67A77EE876A9A
:10ADE800BDEEE66A16EE103A2033402B41F2DD81C3
:10ADF800DFED3A6ABDEEE77A17EE103A2033402BC2
:10AE080001F2CF819FED367AF4EEC77AF1EE10FAAF
:10AE180042F36883DFED335A9FED336A01E0F0EEC9
:10AE2800477AF4EEC67AF1EE10FA37EEE57AF6DCF8
:10AE3800DFED2E7AB4EEE77AF1EE10FA42F14E83A6
:10AE4800DFED285A9FED2A6A01E0B0EE677AB4EE8A
:10AE5800C67AF1EE10FA77EE257AF6D49FED1E7ACF
:10AE6800F4EEC77AF1EE10FA00F38C859FED217AA3
:10AE7800F4EEC77AF1EE10FA44BF9FED1C7A77EE34
:10AE8800677A67EEA75A9FED1C5A9FED1C6A9FEDE3
:10AE98001C7AA5EE856A27EEA55AA5EE867AE5EE18
:10AEA800077A96ED016AD6ED005A27EEC67A65EE66
:10AEB800A77AA5EEA67AE6EE267A86ED007AC6EDA2
:10AEC800017AFFF794B800BF3856002030600020A0
:10AED8006766666635FA8E3CDB0FC93F00000000E6
:10AEE800DB0F4940DB0FC940E4CB1641DB0F49C0FB
:10AEF800E4CB16C1DB0FC9BF92E741B99730083CD4
:10AF080015A82ABE3C560020984400205C49002021
:10AF1800DC4B5A79002A3EF40BABDB4A1278002A44
:10AF28003EF406AB1B78DFEDD94A07EE903AD84BD2
:10AF3800B8EE677A1B8807EE902A06EE903AF8EE8C
:10AF4800E77AF8EE666A67EE277AB7EE007AC7EE18
:10AF5800A63AF4EEE43AF1EE10FA88BFF0EE643A5D
:10AF6800F4EEC73AF1EE10FAB8BFF0EE473AFEF742
:10AF7800E1BAB0EE677A22E4B8F1000F00F0E58399
:10AF8800DFF82883BCF1000F41F0FA87BAF1000F0F
:10AF980041F0508698ED005ADDED0C4ADFF810E3D9
:10AFA80025EE855ABDEEC77A17EE101AB0EE457A2F
:10AFB800A4EEA67AB0EE675AA7EE065ABDEEC57A99
:10AFC80017EE107A17EE100A9F42A8BF1846B9422A
:10AFD800C8BF084607EE100AB8EEC77A012A8EEDF8
:10AFE800007A3FF4F1A898ED047A9DED0D5A25EE0C
:10AFF800877AA5EE267AB0EE675AA7EE065ABDEE16
:10B00800C57A17EE107A17EE100A9F42A8BF1846A5
:10B018008F42B8BF084607EE100AB8EEC77A022A70
:10B028008EED017A3FF4D0A898ED087A9DED0E5A7E
:10B0380025EE877AA5EE267AB0EE675AA7EE065A6D
:10B04800BDEEC57A17EE107A17EE100A9F42A8BF18
:10B0580018468F42B8BF084607EE100AB8EEC77AFE
:10B06800032A8EED027A3FF4AFA898ED0C7A9DED95
:10B078000F5A25EE877AA5EE267AB0EE675AA7EE24
:10B08800065ABDEEC57A17EE107A17EE100A9F42DF
:10B09800A8BF18468F42B8BF084607EE100AB8EE98
:10B0A800C77A042A8EED037A3FF48EA898ED107AB9
:10B0B8009DED105A25EE877AA5EE267AB0EE675AEE
:10B0C800A7EE065ABDEEC57A17EE107A17EE100AEB
:10B0D8009F42A8BF18468F42B8BF084607EE100A1D
:10B0E800B8EEC77A052A8EED047A3FF46DA898ED7C
:10B0F800147A9DED115A25EE877AA5EE267AB0EEE0
:10B10800675AA7EE065ABDEEC57A17EE107A17EE03
:10B11800100A9F42A8BF18468F42B8BF084607EEDC
:10B12800100AB8EEC77A062A8EED057A3FF44CA8C5
:10B1380098ED187A9DED125A25EE877AA5EE267AB3
:10B14800B0EE675AA7EE065ABDEEC57A17EE107A2A
:10B1580017EE100A9F42A8BF18468F42B8BF08468C
:10B1680007EE100AB8EEC77A072A8EED067A3FF482
:10B178002BA898ED1C7A9DED135A65EE875AE6EEDA
:10B18800855AE6EE257AFDEEE77A17EE900A8342B5
:10B19800A8BF03468142D8BF194607EE901AF8EEB9
:10B1A800E77ACEED077A002A7FF40EA8FFF711B8E8
:10B1B800384B93ED006AFEF7D8BD374A3749D2F8C5
:10B1C800EC20096844F620608242A8BF0246B2F526
:10B1D8007A7FB8BF4FF47A7292B2C806A4F84A21AF
:10B1E80041F120830599002940F0C4832C49D1F806
:10B1F80000C0BCF932E02B48D4F84C11A0FB020285
:10B208009009642292FBF0F2142AFDEEC87A04EB4E
:10B218004108A8BF142201318A42C4F84C1117EE24
:10B22800900ADCBF0021C4F84C1104EB4101A8F8D6
:10B238005001B1F9502107EE902AF8EEE77A38EE7E
:10B24800678AFDEEC87ACDED057ABDF9141081EA5A
:10B25800E172A2EBE172724502F32981124A1146AA
:10B268004FF07E520A60FEF7EDBEAB68002B3EF44D
:10B27800E9AD05F150012846984733680693FEF773
:10B28800E1BD00BFA046002056560020713DAA3FF0
:10B29800A85500202844002030070020D046002070
:10B2A80050600020D34D6210900000209844002088
:10B2B8005C4900201D21B448F8F725F900283EF420
:10B2C80090AEB24BDB78002B7EF48BAEDFEDB07A1C
:10B2D800B04938EE678ACBF5FA62FDEEC87A12B249
:10B2E800CDED087ABDF920301B0381FB0301DB1784
:10B2F800C3EBA11302FB03F343F30F335B4407EEE5
:10B30800903AB8EEE78A86ED038AFEF76ABEFBF745
:10B318009BF80B90FDF72BBEDFF8B882FBF794F88B
:10B328009D4AD4F808321268C4F80802C31A9A1A57
:10B338000546A8F80430A8F80620FEF707B819460D
:10B34800FFF7AFBB3B7AC3F1640307EE903AFEF711
:10B3580093BD924B1B7813F0100301F03A8494F8D4
:10B368001411D4F8183196ED017A00290CBF012187
:10B378004FF0FF3103FB01F307EE903AF8EEE77A5E
:10B3880077EE877AC6ED017AFEF73ABE1E217E482F
:10B39800F8F7B9F800283FF455ABBBF1000F7FF47C
:10B3A80051AB94F8B431B34242F0FA807C4BD4EDFF
:10B3B8006E7A93ED010AD4ED4F5A9FED7A6ADFED6C
:10B3C8007A6A27EEE57A67EE887AA0EE087AE5EEE3
:10B3D800807AB4EEC67AF1EE10FA88BFB0EE467AFB
:10B3E800B4EEE67AF1EE10FAF4EEC67AB8BFB0EE33
:10B3F800667AF1EE10FA88BFF0EE467AF4EEE67A55
:10B40800F1EE10FAB8BFF0EE667A84ED4D7AC4ED2D
:10B418004F7AFFF717BBB4F81812914240F27685BD
:10B428006249634AD1ED007A92ED007A6149C4ED30
:10B43800877A77EE676AC4ED857A0122C4ED846A5B
:10B4480084ED887AD1ED006ADFED5B7A84F82422F6
:10B45800FDF7ACBFFDEEC87ADFF8788117EE903AB9
:10B46800A8F804A0A8F80630FFF7E7BABDEEE77A17
:10B47800DFF8608117EE103AA8F80430FFF7C6BA73
:10B48800B4EEC87AF1EE10FA98BFB0EE478ABDEE76
:10B49800C77AB4EEE68ADFF83C81F1EE10FA17EECF
:10B4A800103AB8BFB0EE668A84ED4D8AA8F800302D
:10B4B800002A7FF4E1A9FFF7C0BA9FED3A7ADFEDE1
:10B4C8003A6ADFF81081F4EEC77AF1EE10FA98BF05
:10B4D800B0EE677AFDEEE77AB4EEE67AF1EE10FAAE
:10B4E80017EE903AB8BFB0EE667A012A84ED4E7A2C
:10B4F800A8F802303FF725AAFFF79FBAFAF7A4FF8A
:10B50800079ADFF8D0802D4B801A1B78A8F8040022
:10B51800FFF7A8BA2A4A2B49D2ED006A2A4A91EDC8
:10B52800006A1278C4ED876A84ED886A002A40F0C0
:10B53800D48476EEC65AF0EE466ABCEEC76A234952
:10B54800C4ED845A16EE102AC4ED856AA4F81822B0
:10B55800FF22D1ED006A84F8242277EEC77AFDF73E
:10B5680025BFB5EEC07AF1EE10FA00F1F785B7EE17
:10B57800006A36EE477AC6EE076AFFF7C7B9DFED0D
:10B58800146AFFF75DB900BFD04600209C38002040
:10B5980000007A44D34D62103C4B00209C460020AA
:10B5A8009000002000C0F94400C0F9C418450020EC
:10B5B800FC4A0020344500200000000038560020D6
:10B5C8009C4900201C450020544C00203045002098
:10B5D8000000C8423C56002098ED016A26EE646AD5
:10B5E800B0EE674AA6EE074AB4EEC45A34EE666A6D
:10B5F800F1EE10FAC8BFB0EE656A012B8EED006A55
:10B608003EF4E7AD98ED056A26EE646AB0EE674A47
:10B61800A6EE074AB4EEC45A34EE666AF1EE10FAA2
:10B62800C8BFB0EE656A022B8EED016A3EF4D1AD5B
:10B6380098ED096A26EE646AB0EE674AA6EE074AF4
:10B64800B4EEC45A34EE666AF1EE10FAC8BFB0EE32
:10B65800656A032B8EED026A3EF4BBAD98ED0D6A68
:10B6680026EE646AB0EE674AA6EE074AB4EEC45AFC
:10B6780034EE666AF1EE10FAC8BFB0EE656A042BC4
:10B688008EED036A3EF4A5AD98ED116A26EE646A64
:10B69800B0EE674AA6EE074AB4EEC45A34EE666ABC
:10B6A800F1EE10FAC8BFB0EE656A052B8EED046A9C
:10B6B8003EF48FAD98ED156A26EE646AB0EE674ADF
:10B6C800A6EE074AB4EEC45A74EE666AF1EE10FAB2
:10B6D800C8BFF0EE656A062BCEED056A3EF479AD7B
:10B6E800D8ED196A66EEE46AB0EE674AA6EE874AB4
:10B6F800B3EE046AB4EEC45A74EE466AF1EE10FA78
:10B70800C8BFF0EE656A072BCEED066A3EF461AD60
:10B71800D8ED1D6A66EEE44AE4EE877AF4EEC57A5F
:10B7280077EEC67AF1EE10FAB8BFF0EE657ACEED94
:10B73800077AFEF74EBD99F82020C2EB421102EBC2
:10B748008102D20091B2FEF78ABCDFF8A885BAF16F
:10B75800000F41F0EB8098ED005ADDED0C4ADFF860
:10B7680098E525EE855ABDEEC77A17EE101AB0EEA9
:10B77800457AA4EEA67AB0EE675AA7EE065ABDEE51
:10B78800C57A17EE107A17EE100A9F42A8BF18461E
:10B79800B942C8BF084607EE100AB8EEC77A012AB0
:10B7A8008EED007A3EF498A998ED047A9DED0D5A35
:10B7B80025EE877AA5EE267AB0EE675AA7EE065AE6
:10B7C800BDEEC57A17EE107A17EE100A9F42A8BF91
:10B7D80018468F42B8BF084607EE100AB8EEC77A77
:10B7E800022A8EED017A3EF477A998ED087A9DED4C
:10B7F8000E5A25EE877AA5EE267AB0EE675AA7EE9E
:10B80800065ABDEEC57A17EE107A17EE100A9F4257
:10B81800A8BF18468F42B8BF084607EE100AB8EE10
:10B82800C77A032A8EED027A3EF456A998ED0C7A6F
:10B838009DED0F5A25EE877AA5EE267AB0EE675A67
:10B84800A7EE065ABDEEC57A17EE107A17EE100A63
:10B858009F42A8BF18468F42B8BF084607EE100A95
:10B86800B8EEC77A042A8EED037A3EF435A998ED2E
:10B87800107A9DED105A25EE877AA5EE267AB0EE5D
:10B88800675AA7EE065ABDEEC57A17EE107A17EE7C
:10B89800100A9F42A8BF18468F42B8BF084607EE55
:10B8A800100AB8EEC77A052A8EED047A3EF414A978
:10B8B80098ED147A9DED115A25EE877AA5EE267A31
:10B8C800B0EE675AA7EE065ABDEEC57A17EE107AA3
:10B8D80017EE100A9F42A8BF18468F42B8BF084605
:10B8E80007EE100AB8EEC77A062A8EED057A3EF4FE
:10B8F800F3A898ED187A9DED125A25EE877AA5EEF1
:10B90800267AB0EE675AA7EE065ABDEEC57A17EE4C
:10B91800107A17EE100A9F42A8BF18468F42B8BF88
:10B92800084607EE100AB8EEC77A072A8EED067A9F
:10B938003EF4D2A898ED1C7A9DED135A65EE875A0D
:10B94800E6EE855AE6EE257AFDEEE77A17EE900ADE
:10B958008342A8BF03468142D8BF194607EE901A12
:10B96800F8EEE77ACEED077ABCF1000F7EF431AC41
:10B97800FEF7B6B8DA49D1F800C0BCF832E04FEAB1
:10B988005E0E38E49FEDD77A77EE677AFFF779BADB
:10B99800DFF86893D4ED017A94ED006AB9F80000F5
:10B9A800D9F8143077EEA77AF0EE006AB0EE677A2D
:10B9B800A6EE267A013804EBC002D6EE267A083ABB
:10B9C8001033F6EE003A27EE237A67EEA37A84ED79
:10B9D800207AC4ED217AC44CA64604F1800192ED88
:10B9E800027A92ED036ADEED036ADEED027A53ED28
:10B9F800014A13ED025A37EE674A76EEC65A77EED9
:10BA0800277AE4EE845A0138A2F10802E5EE047AB6
:10BA18000EF1080E03F1080336EE267A01F108014B
:10BA2800E4EE877AE5EE475A67EEA37A25EEA37A25
:10BA3800C1ED007A81ED017AD1D1142F7DF419AAD4
:10BA4800FAF702FD069BDFF8B882C01AA8F80200D0
:10BA5800D4F8D861FDF70DBADFF8A89299F800205C
:10BA6800900802F00F80DFF8A0C200F101084FEA49
:10BA780048180CEB080E0CF12003ACF1700113ED23
:10BA8800076A53ED056A13ED037A53ED017A53ED16
:10BA9800025A13ED084A53ED064A13ED045A26EEEE
:10BAA800066A66EEA66A27EE077A67EEA77AA4EE1C
:10BAB800046A20339E45E4EEA46A01F11001A5EE64
:10BAC800057AE5EEA57AF1EEC65AB1EEE66AF1EE30
:10BAD800C76AB1EEE77A41ED085A01ED076A41ED10
:10BAE800066A01ED057ACAD1A8F12008C44404EB1E
:10BAF800001012F0030318BF0CF1080C0FD05CED16
:10BB0800017A1CED027A67EEA77A013BE7EE077A25
:10BB18000CF1080CB1EEE77AA0EC017AEFD1142F02
:10BB280001F0F3850136C4F8D861FDF70BB9DFF8E9
:10BB3800CC916D48D9F80820B9F80C1020F0F0F92C
:10BB48006A4B1F78142F01F04687D4F8D861013664
:10BB5800C4F8D8611EE7DFF8A491B9F800E0D9F875
:10BB680004C04FEA5E084FEA880204EB8E065FEADB
:10BB7800DE0E04EB020300F0A08010320EF1010E7D
:10BB88005B4803EB0E1E324410330CF1100706F12C
:10BB9800100151ED032A51ED043A10ED043A10ED6D
:10BBA800032A51ED026A11ED016A10ED020A10ED47
:10BBB800018A12ED044A12ED035A53ED044A53ED7B
:10BBC800035A13ED027A53ED017A52ED020A12ED8F
:10BBD800011A73EE238A72EE221A40ED048A40EDB0
:10BBE800031A70EE268A78EE061A40ED028A40EDB6
:10BBF800011A74EE848A75EE851A43ED048A43EDC2
:10BC0800031A77EE208A77EE811A43ED028A43ED14
:10BC1800011A73EE633A75EE655A17ED035A32EE60
:10BC2800623A74EE644A65EE631A17ED044A23EE2D
:10BC3800052A64EE652AE3EE041A10339E4524EEC5
:10BC4800843AA3EE842A00F1100007F11007A5EE4C
:10BC5800853A01F1100102F11002E4EE852A41ED66
:10BC6800071A01ED082A02ED073A42ED082A57EDB6
:10BC7800055A17ED065A70EE666A38EE466A30EED7
:10BC8800C77A71EE677A26EE253A65EEE63A25EE32
:10BC9800674A67EE054AE6EE053AA6EE853AA7EE4C
:10BCA800254AE7EEA54A01ED063A41ED053A02EDCF
:10BCB800064A42ED054A7FF46CAF1FFA88F86246DF
:10BCC800414609481FF0F8F84146D9F804203046A3
:10BCD8001FF0F2F8054B1B78142B7FF4B9AEAFE6D2
:10BCE80050600020DB0F4940B42A0020385600205D
:10BCF800C42A0020984400205C490020705A002083
:10BD08003C5600206A5A0020342B0020D4F8DC81ED
:10BD1800B4F8D4A1C74BCAF120095FFA89F90AEB34
:10BD2800481E03EB8E0E5FEA990301F0138401337A
:10BD38001801C149C14A0EEB000C0EF1100313EDB6
:10BD4800024A13ED035A13ED016A13ED047A51ED1B
:10BD5800024A51ED035A51ED016A51ED047A64EE3D
:10BD6800244A65EE255A66EE266A67EE277A10336E
:10BD78009C4542ED024A42ED035A42ED016A42ED0A
:10BD8800047A01F1100102F11002D8D1AC49A0F1F6
:10BD98001002964401EB020C224419F0030309D067
:10BDA800BEEC017AFCEC017A67EE277A013BE2EC03
:10BDB800017AF5D1BAF1000F41F07B80142F7DF4A0
:10BDC80058A8FAF741FB069BDFF8A882D4F8D86197
:10BDD800C01AA8F80200FDF74CB8D4F8DC91994ACB
:10BDE800994BDFED9A7AD3ED008A994B4FEAC90156
:10BDF8000A44F8EE688A928809EE102A643AC82A3A
:10BE0800A8BFC82268EEA78AF8EE497A782AB8BF90
:10BE1800782268EEA78A07EE902A4944B0EE680AAD
:10BE280003EB8108B8EEE78A21F026FBB8EEC99A41
:10BE3800F0EE409AB0EE680A21F080FA38EE097AFE
:10BE480079EE487A28EE098A67EE877AB7EE006AB3
:10BE580088EE277A142FF8EE007A77EE076A60EEFC
:10BE6800277A89EEA67A77EE065A36EE477AC6EE34
:10BE7800256A67EEA67A27EE267AC8ED006A88ED6D
:10BE8800047AC8ED026AC8ED017AC8ED037A01F0B8
:10BE98002E84704B704A09F1010983FB0938A8EB1D
:10BEA800E97808EB48080136A9EB08081778C4F8C0
:10BEB800D861C4F8DC812BE7FAF7C6FA664B06901E
:10BEC8001F78142F05BFDFF8AC81D4F8D861D4F8F7
:10BED800D861A8F80060FCF71ABF76EE665AFFF73B
:10BEE8002CBB5E4A99ED007AD2ED006AB0EEC77AB3
:10BEF800B4EEE67AF1EE10FA7DF500AA01220A996D
:10BF0800C4F8F81184F8F421FDF7CBBE544A55491A
:10BF1800D2ED007A544A91ED007A1278C4ED877A0E
:10BF280084ED887A002A01F0BC8277EE676A4F496F
:10BF3800C4ED857AC4ED846AFF22D1ED006ADFED95
:10BF48004E7A84F82422FDF731BA494FDFF8E4909D
:10BF5800D7ED005A97ED055A97ED016A97ED064A15
:10BF6800D7ED044AD7ED036A97ED027A67EE897A2E
:10BF780009EB8603A5EEA75AA6EE274A64EEC54A42
:10BF8800A6EEC54AE7EE274A20EE050A87ED054AE0
:10BF9800C7ED064A29EE088A69EE288A83ED005A19
:10BFA80021F01EFAD7ED0E5AD7ED176A97ED091A48
:10BFB800D7ED121A97ED0F5A97ED187A97ED0A2ACE
:10BFC800D7ED132A97ED0D6AD7ED167A97ED0C3A4F
:10BFD800D7ED0B3A97ED154AD7ED144AE1EE085A1A
:10BFE800002109EB8602E8EEA16A00B2C4F8C41188
:10BFF800A2EE085AC4F8C811C4F8CC11A8EEA27A67
:10C0080026EE656A67EEE67AA3EE655AA3EE886ABD
:10C01800A6EEC47AE8EEA47A87ED0E5AC2ED205A4D
:10C0280087ED0F6AC2ED406A87ED177AC7ED187A77
:10C03800FEF724BB885A0020185C0020C42A002080
:10C04800085C0020885C0020606B002027D4D23672
:10C05800F46A002056555555385600206044002093
:10C068009C4900201C450020544C002030450020ED
:10C078000C5D00203C56002000000000B5F93C3063
:10C088006A6207EE903A0122F8EEE77AEB66C5F8A5
:10C0980088200023012FC5ED1F7AC5ED1E7AC5F84B
:10C0A800803001F02782B7427DF46EADB5F93E309D
:10C0B8002B6707EE903A00220123F8EEE77AAA628E
:10C0C800C5F89C300023012FC5ED247AC5ED237AED
:10C0D800C5F8943001F00A82B7427DF485ADB5F910
:10C0E80040306B6707EE903A00220123F8EEE77ABA
:10C0F800EA62C5F8B0300023012FC5ED297AC5EDF5
:10C10800287AC5F8A8307DF49FAD1FED258AB9F1CE
:10C11800030F2BD0BAF1000F09D007EE90AAF8EE62
:10C12800E77AF4EEC87AF1EE10FA01F1B084C04A69
:10C138006B6F1268A8F80600002103EB560393FB07
:10C14800F6F6EE6291621163D162FDF77FBDB94BDD
:10C158009B7B002B3DF467AFFDF769BFF7EE006AE4
:10C16800FEF7D4BBF7EE006AFEF74BBCB0EE480A08
:10C1780021F036F900B2CDE7B4F878A10AF1FF3A18
:10C188000FFA8AFABAF1000FA4F878A13DF7B9AF0F
:10C19800FEF7F3BAB4F84A2102F57A7291B2FDF7C4
:10C1A8005EBFDFEDA57AFEF77CBEF4EEC77AF1EE4E
:10C1B80010FA41F3BA82DFEDA15A9FEDA16A01E0BE
:10C1C800F0EE476AF4EEC66AF1EE10FA36EEE57A5A
:10C1D800F6DCDFED9C6AB4EEE67AF1EE10FA41F196
:10C1E8008282DFED965A9FED986A01E0B0EE667A9A
:10C1F800B4EEC67AF1EE10FA77EE256AF6D49FED22
:10C20800937AF4EEC76AF1EE10FA40F3CE849FED0C
:10C21800907A77EE666A66EEA65A9FED8E5A9FED83
:10C228008E6A9FED8E7AA5EE856A26EEA55AA5EE52
:10C23800867AE5EE076AFEF7DDBD894F3A78013A5E
:10C248000A2A1CD8DFE812F0B0005C012201D900EC
:10C258001B001B009B008A00660051000B00814AEE
:10C26800814952680968C8328A4203D319F04AFDE5
:10C2780028B1B378032B01F0CA8401233B70F3780B
:10C28800002B3EF4EAAB794B1B78D80740F1958038
:10C29800DFF8D481D4F8C021D8F800309A4200F2EF
:10C2A80098803B78012B3EF4D8AB94F8BC21002A47
:10C2B8003EF4D3AB0B2B0DD801229A4040F6030174
:10C2C80012EA01060CD112F4C06F03D0093B012B0E
:10C2D80041F2C385634BD8F800205A600B233B70AA
:10C2E800002384F8BC31FEF7B8BB614B1B78002BE8
:10C2F80001F07D831A2016F02DFB002841F077838A
:10C3080094F8BC31002B41F0728309233B700EF086
:10C318004DFCB4E71A2016F01DFB0028F7D0554B4A
:10C328001B88002BF3D1544B4520D3F8008019F01B
:10C338000DFD0E2019F00AFD40460EF005F9DDF856
:10C34800288040460EF000F94C4A4D4B12681A609E
:10C3580040460A233B700EF067F9D8E719F0B0FCA5
:10C368000EF05AFC00288AD019F0CCFC002886D0A0
:10C37800424A434B12681A600A233B707FE719F060
:10C388009FFC404B002105208DE80300A3F1080223
:10C39800029153200FF036F900287FF470AF314A2C
:10C3A800082310603B706AE7304B1B78DB0701F10C
:10C3B800D583F378002B3EF450AB0CF03BFF0028FC
:10C3C8003FF466AF284B1B6803F59C530833C4F849
:10C3D800C0313B78012B7EF440AB94F8BC31002B84
:10C3E8007EF43BABB378032B01F0E9840FF0D4F96A
:10C3F800012384F8BC31FEF730BB19F061FC224AF6
:10C408000292A2F10C03262101930091A2F10A03E2
:10C418005021163A49200FF0F5F800287FF42FAF85
:10C42800104B4FF0FF310722186059603A7026E729
:10C43800EC480020F867002000000000DB0FC9402E
:10C44800E4CB1641DB0F49C0E4CB16C1DB0FC93F73
:10C45800DB0F494092E741B99730083C15A82ABE3E
:10C468002F340020004B00207C610020F266002061
:10C47800A84B0020804900207C49002090490020DA
:10C488008849002018FA02085EF80208DFF8A48339
:10C4980019F016FCE64AD8F804301268643393425F
:10C4A800BFF4EDAE402019F0EFFB00287FF4E7AEB3
:10C4B800D8F80030DFF89CA3DFF87CB34FF04009D0
:10C4C8000FE019F043FCDBF80020D8F80030013AFF
:10C4D8000133B9F10109CBF80020C8F8003001F0A8
:10C4E80012841AF803301846002BEAD100234FF0C3
:10C4F800FF32C8F800300423C8F804203B70BEE6B9
:10C50800CB4BCC4A1B685360CB49002313600322F2
:10C518000B603A70B3E6C94ADFEDC97A92ED080AB2
:10C528000893B4EEE70AF1EE10FA40F2188520F00D
:10C53800EDFFD4ED517A20EE270A20F051FFB0F537
:10C54800617F089B00F3518607EE900AF8EEE76AD0
:10C55800DFEDBC7A66EEA76A07EE903AB8EEE77AA6
:10C56800FDEEE67A17EE903A2033402B41F24482F2
:10C578009FEDB50A20F034FF00B207EE900AF8EEFE
:10C58800E77A38EE278A86ED038AFDF756BD099BC0
:10C5980093F800C00CF0010CBCF1000F7DF419AE4B
:10C5A800FDF79EBAA94BDFEDAA7A1F68C4ED797A28
:10C5B80017F0805740F0328310F4800700F0AC8108
:10C5C8000027B6EE007A67EE877AF4EEE75AF1EEC6
:10C5D80010FA48BFF0EE675A40F12083C4ED8A5A3A
:10C5E800FDF727B9F9F730FF0790FDF724BC74EE83
:10C5F800677AB7EE007AF4EEC77AF1EE10FAC4ED76
:10C60800797A40F3638784EEA77A8DED0C7AFDF78B
:10C6180006B9BEF1000F00F02E8698ED007A9DED68
:10C628000C5ADFF834E225EE877AA5EE267AB0EECA
:10C63800675AA7EE065ABDEEC57A17EE107A17EEBE
:10C64800100A9F42A8BF1846B942C8BF084607EE5D
:10C65800100AB8EEC77A012A8EED007A3DF4B9AD1A
:10C6680098ED047A9DED0D5A25EE877AA5EE267A87
:10C67800B0EE675AA7EE065ABDEEC57A17EE107AE5
:10C6880017EE100A9F42A8BF1846B942C8BF08460D
:10C6980007EE100AB8EEC77A022A8EED017A3DF449
:10C6A80098AD98ED087A9DED0E5A25EE877AA5EE9D
:10C6B800267AB0EE675AA7EE065ABDEEC57A17EE8F
:10C6C800107A17EE100A9F42A8BF1846B942C8BF91
:10C6D800084607EE100AB8EEC77A032A8EED027AEA
:10C6E8003DF477AD98ED0C7A9DED0F5A25EE877ADB
:10C6F800A5EE267AB0EE675AA7EE065ABDEEC57AC1
:10C7080017EE107A17EE100A9F42A8BF1846B942D2
:10C71800C8BF084607EE100AB8EEC77A042A8EED9D
:10C72800037A3DF456AD98ED107A9DED105A25EE3A
:10C73800877AA5EE267AB0EE675AA7EE065ABDEEBE
:10C74800C57A17EE107A17EE100A9F42A8BF18464E
:10C75800B942C8BF084607EE100AB8EEC77A052ADC
:10C768008EED047A3DF435AD98ED147A9DED115AAD
:10C7780025EE877AA5EE267AB0EE675AA7EE065A16
:10C78800BDEEC57A17EE107A17EE100A9F42A8BFC1
:10C798001846B942C8BF084607EE100AB8EEC77A6D
:10C7A800062A8EED057A3DF414AD98ED187A9DEDC4
:10C7B800125A25EE877AA5EE267AB0EE675AA7EECA
:10C7C800065ABDEEC57A17EE107A17EE100A9F4288
:10C7D800A8BF1846B942C8BF084607EE100AB8EE07
:10C7E800C77A072A8EED067A3DF4F3AC98ED1C7AE9
:10C7F8009DED135A65EE875AE5EE265AE6EE257A40
:10C80800FDEEE77A17EE902A9342A8BF13468A42B4
:10C81800A8BF194607EE901AF8EEE77ACEED077A28
:10C82800FDF7D7BC0699C9003EF5DCACFDF70ABC9C
:10C838007C610020004B00206C6200200C4000202E
:10C848008FC2753CD06D393A00000000D0460020F8
:10C8580000000080F8F702085C490020012A40F334
:10C86800498607EE101AB8EEC77AC7EE876AB1EEA6
:10C87800E68AB9F1030F13D0BAF1000F09D007EE19
:10C8880090AAF8EEE77AF4EEC87AF1EE10FA01F120
:10C89800FE80EB6E03EB560393FBF6F36B6202E448
:10C8A800B0EE480A20F09CFD00B2E5E7012A40F30B
:10C8B8001D8607EE101AB8EEC77AC7EE876AB1EE82
:10C8C800E68AB9F1030F14D0BAF1000F09D007EEC8
:10C8D80090AAF8EEE77AF4EEC87AF1EE10FA01F1D0
:10C8E800D6802B6F03EB560393FBF6F3AB62FFF78F
:10C8F800F3BBB0EE480A20F073FD00B2E4E7012A6A
:10C908007FF703AC07EE101AB8EEC77AC7EE876A4E
:10C91800B1EEE68AFFF7FBBBB6EE007AF4EEC75A33
:10C92800F1EE10FA3FF74DAEFCF783BF98ED005AD1
:10C938009DED0C4ADFF844E625EE855AFDEEC73A30
:10C94800A4EE265AB0EE674AA5EE064A13EE901AF0
:10C95800F4EEC44AF1EE10FAB0EE445A88BFB0EED5
:10C96800475ABDEEC55A15EE100A15EE107A9842D0
:10C97800A8BF1F468142C8BF0F4605EE107AB8EE21
:10C98800C55A012A8EED005A3DF4A6A898ED045A1E
:10C998009DED0D4A25EE855AA4EE265AB0EE674A5B
:10C9A800A5EE064AF4EEC44AF1EE10FAB0EE445A87
:10C9B80088BFB0EE475ABDEEC55A15EE100A15EEFF
:10C9C800107A9842A8BF1F468842B8BF0F4605EEA6
:10C9D800107AB8EEC55A022A8EED015A3DF47CA8A9
:10C9E80098ED085A9DED0E4A25EE855AA4EE265A72
:10C9F800B0EE674AA5EE064AF4EEC44AF1EE10FA24
:10CA0800B0EE445A88BFB0EE475ABDEEC55A15EE8F
:10CA1800100A15EE107A9842A8BF1F468842B8BF80
:10CA28000F4605EE107AB8EEC55A032A8EED025A63
:10CA38003DF452A898ED0C5A9DED0F4A25EE855A03
:10CA4800A4EE265AB0EE674AA5EE064AF4EEC44AAA
:10CA5800F1EE10FAB0EE445A88BFB0EE475ABDEE78
:10CA6800C55A15EE100A15EE107A9842A8BF1F464F
:10CA78008842B8BF0F4605EE107AB8EEC55A042AA8
:10CA88008EED035A3DF428A898ED105A9DED104AF2
:10CA980025EE855AA4EE265AB0EE674AA5EE064A58
:10CAA800F4EEC44AF1EE10FAB0EE445A88BFB0EE84
:10CAB800475ABDEEC55A15EE100A15EE107A98427F
:10CAC800A8BF1F468842B8BF0F4605EE107AB8EED9
:10CAD800C55A052A8EED045A3CF4FEAF98ED145A57
:10CAE8009DED114A25EE855AA4EE265AB0EE674A06
:10CAF800A5EE064AF4EEC44AF1EE10FAB0EE445A36
:10CB080088BFB0EE475ABDEEC55A15EE100A15EEAD
:10CB1800107A9842A8BF1F468842B8BF0F4605EE54
:10CB2800107AB8EEC55A062A8EED055A3CF4D4AFF1
:10CB380098ED185A9DED124A25EE855AA4EE265A0C
:10CB4800B0EE674AA5EE064AF4EEC44AF1EE10FAD2
:10CB5800B0EE445A88BFB0EE475ABDEEC55A15EE3E
:10CB6800100A15EE107A9842A8BF1F468842B8BF2F
:10CB78000F4605EE107AB8EEC55A072A8EED065A0A
:10CB88003CF4AAAF98ED1C5A9DED134A65EE855A00
:10CB9800E6EE845AE6EE257AF4EEE74AF1EE10FA6C
:10CBA800C8BFF0EE477AFEF7CFBE9FEDEF7AF4EEFE
:10CBB800C76AF1EE10FA44BF9FEDEC7A77EE666A29
:10CBC800FFF729BB8223FCF740B9DFEDE97AFCF7D0
:10CBD80007B99AF803E0BEF1000F00F02083B4F91A
:10CBE8001CE19AF80200A8EB0E0C8CEAEC71A1EBA0
:10CBF800EC71814240F39E84F045C8BF404207EE85
:10CC0800900AF8EEE77A012138EE278AC4F8203135
:10CC180084F8241186ED038AFDF7F2B9B7EE007A9D
:10CC280077EE677AF4EEE75AF1EE10FA88BFF0EE85
:10CC3800675AD3E498ED005A9DED0C4ADFF83CE3BF
:10CC480025EE855AFDEEC73AA4EE265AB0EE674A9D
:10CC5800A5EE064A13EE901AF4EEC44AF1EE10FA65
:10CC6800B0EE445A88BFB0EE475ABDEEC55A15EE2D
:10CC7800100A15EE107A9842A8BF1F468142C8BF15
:10CC88000F4605EE107AB8EEC55A012A8EED005A05
:10CC98003DF49AAA98ED045A9DED0D4A25EE855A61
:10CCA800A4EE265AB0EE674AA5EE064AF4EEC44A48
:10CCB800F1EE10FAB0EE445A88BFB0EE475ABDEE16
:10CCC800C55A15EE100A15EE107A9842A8BF1F46ED
:10CCD8008842B8BF0F4605EE107AB8EEC55A022A48
:10CCE8008EED015A3DF470AA98ED085A9DED0E4A52
:10CCF80025EE855AA4EE265AB0EE674AA5EE064AF6
:10CD0800F4EEC44AF1EE10FAB0EE445A88BFB0EE21
:10CD1800475ABDEEC55A15EE100A15EE107A98421C
:10CD2800A8BF1F468842B8BF0F4605EE107AB8EE76
:10CD3800C55A032A8EED025A3DF446AA98ED0C5ABC
:10CD48009DED0F4A25EE855AA4EE265AB0EE674AA5
:10CD5800A5EE064AF4EEC44AF1EE10FAB0EE445AD3
:10CD680088BFB0EE475ABDEEC55A15EE100A15EE4B
:10CD7800107A9842A8BF1F468842B8BF0F4605EEF2
:10CD8800107AB8EEC55A042A8EED035A3DF41CAA4F
:10CD980098ED105A9DED104A25EE855AA4EE265AB4
:10CDA800B0EE674AA5EE064AF4EEC44AF1EE10FA70
:10CDB800B0EE445A88BFB0EE475ABDEEC55A15EEDC
:10CDC800100A15EE107A9842A8BF1F468842B8BFCD
:10CDD8000F4605EE107AB8EEC55A052A8EED045AAC
:10CDE8003DF4F2A998ED145A9DED114A25EE855AA5
:10CDF800A4EE265AB0EE674AA5EE064AF4EEC44AF7
:10CE0800F1EE10FAB0EE445A88BFB0EE475ABDEEC4
:10CE1800C55A15EE100A15EE107A9842A8BF1F469B
:10CE28008842B8BF0F4605EE107AB8EEC55A062AF2
:10CE38008EED055A3DF4C8A998ED185A9DED124A91
:10CE480025EE855AA4EE265AB0EE674AA5EE064AA4
:10CE5800F4EEC44AF1EE10FAB0EE445A88BFB0EED0
:10CE6800475ABDEEC55A15EE100A15EE107A9842CB
:10CE7800A8BF1F468842B8BF0F4605EE107AB8EE25
:10CE8800C55A072A8EED065A3DF49EA998ED1C5AFC
:10CE98009DED134A65EE855AE6EE845AE6EE257A4C
:10CEA800F4EEE74AF1EE10FAC8BFF0EE477AFEF763
:10CEB8006AB9304B4FEA890E5FEA9A0901EB0E0C0A
:10CEC80003EBC818A64400F0538609F101094FEA9C
:10CED800091908EB090008F110030CF110010EF113
:10CEE800100213ED024A13ED035A13ED016A13ED14
:10CEF800047A51ED024A51ED035A51ED016A51EDA0
:10CF0800047A64EE244A65EE255A66EE266A67EED0
:10CF1800277A1033984242ED024A42ED035A42ED15
:10CF2800016A42ED047A01F1100102F11002D8D130
:10CF3800A9F11009C8440CEB0901CE441AF0030A00
:10CF48003EF43CAFB8EC017AF1EC017A67EE277A4F
:10CF5800BAF1010AEEEC017AF4D1FEF72FBFDFED4A
:10CF6800067AFFF70EBB00BFDB0FC9BFDB0F49C056
:10CF780000000243885A0020000000005C4900209D
:10CF880098ED005A9DED0C4A25EE855AA4EE265AD6
:10CF9800B0EE674AA5EE064AB0EE445ABEF1000F5D
:10CFA80000F0E483BAF1000F06D0F4EE444AF1EE43
:10CFB80010FAC8BFB0EE475ABDEEC77A17EE10CACE
:10CFC800BDEEC57A05EE10CA17EE101A8C4500F3AF
:10CFD800B5859942A8BF194607EE101AB8EEC77A68
:10CFE800DFF8A8E5012A8EED007A3DF4F2A898ED65
:10CFF800047A9DED0D4A25EE877AA4EE267AB0EEE6
:10D00800674AA7EE064AB0EE447ABAF1000F00F07C
:10D018008485F4EEC44AF1EE10FA40F37E85614649
:10D028009942A8BF194607EE101AB8EEC77A022A25
:10D038008EED017A3DF4CDA898ED087A9DED0E4A63
:10D0480025EE877AA4EE267AB0EE674AA7EE064A5E
:10D05800B0EE447ABAF1000F00F05485F4EEC44AF9
:10D06800F1EE10FA40F34E8561469942A8BF194681
:10D0780007EE101AB8EEC77A032A8EED027A3DF44D
:10D08800A8A898ED0C7A9DED0F4A25EE877AA4EEB4
:10D09800267AB0EE674AA7EE064AB0EE447ABAF1AD
:10D0A800000F00F02485F4EEC44AF1EE10FA40F3C4
:10D0B8001E8561469942A8BF194607EE101AB8EEB8
:10D0C800C77A042A8EED037A3DF483A898ED107A86
:10D0D8009DED104A25EE877AA4EE267AB0EE674ACF
:10D0E800A7EE064AB0EE447ABAF1000F00F0F484D5
:10D0F800F4EEC44AF1EE10FA40F3EE846146994228
:10D10800A8BF194607EE101AB8EEC77A052A8EEDA1
:10D11800047A3DF45EA898ED147A9DED114A25EE47
:10D12800877AA4EE267AB0EE674AA7EE064AB0EEF2
:10D13800447ABAF1000F00F0C484F4EEC44AF1EE68
:10D1480010FA40F3BE8461469942A8BF194607EE1B
:10D15800101AB8EEC77A062A8EED057A3DF439A87A
:10D1680098ED187A9DED124A25EE877AA4EE267A74
:10D17800B0EE674AA7EE064AB0EE447ABAF1000F5D
:10D1880000F09484F4EEC44AF1EE10FA40F38E8471
:10D1980061469942A8BF194607EE101AB8EEC77A39
:10D1A800072A8EED067A3DF414A898ED1C7A9DEDB9
:10D1B800134A65EE875AE4EE265AE5EE867ABAF106
:10D1C800000F00F06A84F4EEE47AF1EE10FA40F110
:10D1D800648462469A42A8BF1A4605EE102AB8EE41
:10D1E800C55A8EED075AFCF7F4BF07EE903ADFED0B
:10D1F800DC6AB8EEE77A66EEA65A9FEDDA5A9FED3A
:10D20800DA6ADFEDDA7AA5EE856A26EEA55AE5EE4A
:10D21800867AE5EE276A26EE870AFFF7ABB9B4F9F6
:10D228001CC19AF80210A8EB0C0383EAE370A0EB88
:10D23800E370884240F3708103EBD37301215B10E4
:10D24800C4F82C3184F8301184F82411D4F818313A
:10D258006344B3F5FA6FA8BF4FF4FA63B3F57A7F66
:10D26800B8BF4FF47A7307EE903AB8EEE78A86EDC6
:10D27800038AFCF7C5BE98ED005ADDED0C4A25EE91
:10D28800855AA4EEA65AF0EE674AE5EE064ABDEEC8
:10D29800E45A15EE10EA714500F359819E45A8BF7E
:10D2A8009E4605EE10EAB8EEC55A002F00F07C85C0
:10D2B800DFF8D8E2012A8EED005A3CF48AAF98EDE7
:10D2C800045ADDED0D4A25EE855AA4EEA65AF0EE75
:10D2D800674AE5EE064ABDEEE45A15EE10CA614506
:10D2E80000F3CD819C45A8BF9C4605EE10CAB8EE58
:10D2F800C55A002F00F0F885022A8EED015A3CF439
:10D3080068AF98ED085ADDED0E4A25EE855AA4EE71
:10D31800A65AF0EE674AE5EE064ABDEEE45A15EE67
:10D3280010CA614500F3DC819C45A8BF9C4605EE08
:10D3380010CAB8EEC55A002F00F0CB85032A8EED2F
:10D34800025A3CF446AF98ED0C5ADDED0F4A25EE33
:10D35800855AA4EEA65AF0EE674AE5EE064ABDEEF7
:10D36800E45A15EE10CA614500F3B7819C45A8BF81
:10D378009C4605EE10CAB8EEC55A002F00F0478546
:10D38800042A8EED035A3CF424AF98ED105ADDEDD3
:10D39800104A25EE855AA4EEA65AF0EE674AE5EE45
:10D3A800064ABDEEE45A15EE10CA614500F36D81D8
:10D3B8009C45A8BF9C4605EE10CAB8EEC55A002F7A
:10D3C80000F01A85052A8EED045A3CF402AF98ED58
:10D3D800145ADDED114A25EE855AA4EEA65AF0EE50
:10D3E800674AE5EE064ABDEEE45A15EE10CA6145F5
:10D3F80000F348819C45A8BF9C4605EE10CAB8EECC
:10D40800C55A002F00F08F84062A8EED055A3CF489
:10D41800E0AE98ED185ADDED124A25EE855AA4EED5
:10D42800A65AF0EE674AE5EE064ABDEEE45A15EE56
:10D4380010CA614500F32C819C45A8BF9C4605EEA7
:10D4480010CAB8EEC55A002F00F0CB84072A8EED1B
:10D45800065A3CF4BEAE98ED1C5ADDED134A65EE53
:10D46800855AE6EEA45AE6EE257AFDEEE77A17EE3F
:10D47800902A914203DC9A42A8BF1A46114607EE49
:10D48800901AF8EEE77A002F7FF4C8A9069B002BC4
:10D498007FF4C4A9059B5B45B8BFF0EE477AFFF758
:10D4A800BDB977EEC76AF0EE477AFEF740BDBCF823
:10D4B80034209FED2F7A07EE902AF8EEE77A2D4A6E
:10D4C80067EE877AC2ED007AFCF7BCBD2A4B1F686D
:10D4D80017F080577FF475A8FFF76EB8F0EE477A1B
:10D4E800FDF7BCBCB0EE677AFDF7A2BC9FED2B8AB6
:10D4F800FFF7E7B99FED298AFFF7BBB99FED1F0A30
:10D50800DFF88C8025EE800A1FF06AFFD4F8D86116
:10D51800A8F80600FBF7ADBC94F82431002B3FF4C3
:10D5280095AE174B84F830E11B6884F824E1C4F801
:10D5380028318BE694F8241129B1114984F8243153
:10D548000B68C4F82831D4F81831734481E605EE25
:10D55800101AA8E60B490C4A8C46FEF71EBC00BF01
:10D5680084F9223F92E741B99730083C15A82ABEB2
:10D578006F12833A90000020D04600200000C84275
:10D58800BC460020085C0020B42A00205C4900202A
:10D598003C56002035FA8E3CDB0FC93F00000000E6
:10D5A80007EE906AF8EEE78A5FED067A1FED060A45
:10D5B80084F8B46168EEA78A38EE800AFDEEC07A76
:10D5C80017EE903A2033402B40F2B5821FED0D0A3A
:10D5D800584BFDEEE87A83ED010A17EE903A2033B6
:10D5E800402B00F2A582DFED547AF4EEE78AF1EEE3
:10D5F80010FA40F39583DFED516ADFED517A01E0CF
:10D60800F0EE478AF4EEE78AF1EE10FA38EEE67AA1
:10D61800F6DCDFED4C7AB4EEE77AF1EE10FA40F181
:10D628007C839FED466ADFED486A01E0B0EE677AD9
:10D63800B4EEE67AF1EE10FA77EE067AF6D49FEDBC
:10D64800437AF4EEC77AF1EE10FA40F37B829FED4D
:10D658003A7A77EE677A27EEA76ADFED3D5ADFED73
:10D668003D6A9FED3D7AE6EE256A67EE865AA6EE9C
:10D67800267AE5EE877AC4ED6E7AFDF79CBE05EE54
:10D68800101A34E605EE101AB9E605EE101A94E6FB
:10D6980005EE101AD5E696ED000A059306921FF0DE
:10D6A8009FFE2E49DFF8BCE0D1F8EC10DFF8B88017
:10D6B800069AA8F800008EFB013EC917C1EBAE110F
:10D6C80007EE901AF8EEE77A059BFDEEE77A17EE7B
:10D6D800901AA8F80210FCF710BD05EE101A4AE6D9
:10D6E80005EE101A25E6F0EE476AFEF788BDF8F752
:10D6F800ABFE069BDFF87080D4F8DC91D4F8D861D3
:10D70800C01AA8F80200FEF7C4BBF8F79DFE144B38
:10D71800DFF854801F78069B99F80020D4F8D86168
:10D72800C01AA8F80400FEF7FDB9B0EE667AFEF755
:10D7380050BD00BF90000020DB0F4940DB0FC940FF
:10D74800E4CB1641DB0F49C0E4CB16C1DB0FC93F60
:10D7580092E741B99730083C15A82ABE3007002047
:10D7680038560020D34D62103C560020BAF1000F05
:10D7780006D0F4EE444AF1EE10FAC8BFB0EE475AAC
:10D78800BDEEC74ABDEEC55A14EE10CA15EE101A02
:10D798008C4514EE109A00F337829942A8BF1946B7
:10D7A80005EE101AB8EEC55A002F00F01083DFF806
:10D7B800ECE5012A8EED005A3CF40BAD98ED045AC5
:10D7C8009DED0D4A25EE855AA4EE265AB0EE674A1D
:10D7D800A5EE064AB0EE445ABAF1000F00F00B82EB
:10D7E800F4EEC44AF1EE10FA40F30582614699421C
:10D7F800A8BF194605EE101AB8EEC55A002F00F05A
:10D808005E83022A8EED015A3CF4E3AC98ED085A87
:10D818009DED0E4A25EE855AA4EE265AB0EE674ACB
:10D82800A5EE064AB0EE445ABAF1000F00F0DA81CC
:10D83800F4EEC44AF1EE10FA40F3D48161469942FD
:10D84800A8BF194605EE101AB8EEC55A002F00F009
:10D858002C83032A8EED025A3CF4BBAC98ED0C5A8B
:10D868009DED0F4A25EE855AA4EE265AB0EE674A7A
:10D87800A5EE064AB0EE445ABAF1000F00F0A981AD
:10D88800F4EEC44AF1EE10FA40F3A38161469942DE
:10D89800A8BF194605EE101AB8EEC55A002F00F0B9
:10D8A800FA82042A8EED035A3CF493AC98ED105A90
:10D8B8009DED104A25EE855AA4EE265AB0EE674A29
:10D8C800A5EE064AB0EE445ABAF1000F00F078818E
:10D8D800F4EEC44AF1EE10FA40F3728161469942BF
:10D8E800A8BF194605EE101AB8EEC55A002F00F069
:10D8F800C882052A8EED045A3CF46BAC98ED145A94
:10D908009DED114A25EE855AA4EE265AB0EE674AD7
:10D91800A5EE064AB0EE445ABAF1000F00F047816E
:10D92800F4EEC44AF1EE10FA40F34181614699429F
:10D93800A8BF194605EE101AB8EEC55A002F00F018
:10D94800E882062A8EED055A3CF443AC98ED185A45
:10D958009DED124A25EE855AA4EE265AB0EE674A86
:10D96800A5EE064AB0EE445ABAF1000F00F016814F
:10D97800F4EEC44AF1EE10FA40F310816146994280
:10D98800A8BF194605EE101AB8EEC55A002F00F0C8
:10D99800B682072A8EED065A3CF41BAC98ED1C5A49
:10D9A8009DED134A65EE855AE6EE845AE6EE257A31
:10D9B800BAF1000F40F0E680FDEEE77A17EE902A04
:10D9C800944540F3E68007EE909AF8EEE77A002F48
:10D9D8007EF424AF5AE5F8F737FDDA4BDFF8C08359
:10D9E8001F78069BC01AA8F80200FEF7AEB80A987E
:10D9F8000CF01AFEFEF78BBCDFEDD37AF4EEE76A83
:10DA0800F1EE10FA40F33A82DFEDD05A9FEDD06A7A
:10DA180001E0F0EE676AF4EEC66AF1EE10FA76EE0F
:10DA2800E57AF6DCDFEDCB6AF4EEE67AF1EE10FA91
:10DA380040F12182DFEDC55A9FEDC76A01E0F0EEA3
:10DA4800667AF4EEC67AF1EE10FA77EEA56AF6D4A5
:10DA5800DFEDC27AF4EEE76AF1EE10FA05DDDFEDEC
:10DA6800BA7A77EEE66AFFF7C6BBDFEDBD7AF4EE69
:10DA7800E76AF1EE10FA44BFDFEDB67A77EEE66AB0
:10DA8800FFF7B9BBB74800F1800CFEF732B8A8F829
:10DA98000600A5F8B460FCF7DFB8FDEEE77A17EEEC
:10DAA800902A6245FFF69BABFFF794BBBDEEC77AA1
:10DAB80017EE101A6145BFF66CAB07EE10CAFFF7F8
:10DAC8006DBBBDEEC77A17EE101A6145BFF63CABC9
:10DAD80007EE10CAFFF73DBBBDEEC77A17EE101A66
:10DAE8006145BFF60CAB07EE10CAFFF70DBBBDEEE4
:10DAF800C77A17EE101A6145BFF6DCAA07EE10CAFE
:10DB0800FFF7DDBABDEEC77A17EE101A6145BFF60A
:10DB1800ACAA07EE10CAFFF7ADBABDEEC77A17EE8A
:10DB2800101A6145BFF67CAA07EE10CAFFF77DBA46
:10DB3800DFED8D7A9FE5F5F7FFFB49E507EE10CAA3
:10DB4800FFF74CBA9FED867AF4EEC77AF1EE10FA39
:10DB580044BF9FED807A77EE677A7CE580200EF0EF
:10DB6800D1FF08B11BF068FD0DF016FEFEF787BB6C
:10DB78006146FFF7E3B994F80432002B7BF4DDAB80
:10DB8800FBF7C9BBF4EEE74AF1EE10FA7FF714AFE2
:10DB980062469A42A8BF1A46914614E7BDEEC55A96
:10DBA80015EE101A6145BFF6EAAE6146EAE6BDEE2B
:10DBB800C55A15EE101A6145BFF6B9AE6146B9E609
:10DBC800BDEEC55A15EE101A6145BFF688AE61461E
:10DBD80088E6BDEEC55A15EE101A6145BFF657AE78
:10DBE800614657E6BDEEC55A15EE101A6145BFF6F7
:10DBF80026AE614626E6BDEEC55A15EE101A6145F9
:10DC0800BFF6F5AD6146F5E514EE101AC8E5DFF884
:10DC18009481D8F800001BF0F1FC544B1B780022CB
:10DC2800022BC8F800207EF428AB1BF02BFFFEF770
:10DC380024BB4F4A4F4B10681B689847089BDBED85
:10DC4800007A93ED007A4C4BD7ED006A83ED020A17
:10DC58004A4B67EE277A2B4427EE8C7AD3ED007A6D
:10DC6800474B67EE277AF0EE665AE7EE8D5A93ED4A
:10DC7800006AB1EE467AF4EEC75AF1EE10FA08D40B
:10DC8800F4EEC65AF1EE10FA8CBFB0EE467AB0EE5A
:10DC9800657A3C4B1B78012B02D0192B7BF4C2AA66
:10DCA800DFED397AB4EEE7DAF1EE10FACCBF0123F2
:10DCB8000023FBF7C2BADFED357AF4EEE7DAF1EECE
:10DCC80010FA27DCDFED327AF4EEE7DAF1EE10FA3B
:10DCD80020D4304BD3ED007AB1EE677AB4EEC7DAD0
:10DCE800F1EE10FA2AD4B4EEE7DAF1EE10FA88BFB2
:10DCF800B0EE67DA284BC7ED00BA1B689A427BF78B
:10DD080054AAFCF7E6BC1AF80330002B7EF4B7AA35
:10DD1800FEF7ECBB9FED14DAECE7F0EE477A8EE401
:10DD2800B0EE687A75E4069800287FF46DAB059824
:10DD38005845B8BFB0EE475AFFF766BBB0EE47DAB2
:10DD4800D8E700BF38560020DB0F4940DB0FC94039
:10DD5800E4CB1641DB0F49C0E4CB16C1DB0FC93F4A
:10DD6800DB0FC9BFB42A002000000000384B002098
:10DD7800DC430020F0430020FC4800200044002041
:10DD880068440020C54100200000964200C0F844C5
:10DD980000C0F8C464440020484400205C490020C6
:10DDA8003C56002070620020069800287FF480AA64
:10DDB80005985845B8BFB0EE475AFFF779BA8020A2
:10DDC8000EF0A0FE00287CF448AEFEF70FBB0699C3
:10DDD80000297FF4ECAC05995945B8BFB0EE475A15
:10DDE800E5E4069800287FF431AB05985845B8BF9C
:10DDF800B0EE475AFFF72ABB069800287FF4E2AA3C
:10DE080005985845B8BFB0EE475AFFF7DBBA0698F1
:10DE180000287FF4B5AA05985845B8BFB0EE475A10
:10DE2800FFF7AEBA132B05D1B0EE480A1FF0D8FAA7
:10DE3800AAF80000B0EE480AD5F814323A489847D4
:10DE48003A4B1B78132BB0EE408A7BF453A81FF093
:10DE5800C7FAAAF80200FBF74DB8452017F076FF7D
:10DE6800FF2017F073FF324817F05CFF304617F0B9
:10DE78006DFFFEF72FBAF0EE676AE9E5F0EE667A15
:10DE8800D0E5069900297FF434AD05995945B8BF06
:10DE9800B0EE475A2DE5069900297FF402AD0599A1
:10DEA8005945B8BFB0EE475AFBE4069900297FF4FC
:10DEB800D0AC05995945B8BFB0EE475AC9E40699A0
:10DEC80000297FF49EAC05995945B8BFB0EE475A72
:10DED80097E4069800287FF431AA05985845B8BFFA
:10DEE800B0EE475AFFF72ABA069800287FF404AA2A
:10DEF80005985845B8BFB0EE475AFFF7FDB90699DF
:10DF080000297FF446AD05995945B8BFB0EE475A88
:10DF18003FE5069900297FF414AD05995945B8BF26
:10DF2800B0EE475A0DE500BFF46A002038560020CD
:10DF3800AC2103082DE9F047B0F908500D81EDB286
:10DF4800382D92B00C4600F05081064632D9802D0B
:10DF580000F0E38077D8522D00F08F8040F22781BF
:10DF6800542D00F097816E2D40F0F180B24B0A6875
:10DF78001B88B24DFF2BA8BFFF23511C21601370D3
:10DF8800A96881F3100189B22046F5F7C8F8AC4BAF
:10DF980020461988F5F7C3F8296801F30F0189B2FB
:10DFA80020460125F5F7BBF82B462846638112B0B9
:10DFB800BDE8F087042D00F0618140F2E180202D5A
:10DFC80000F08F8040F2FD80242D00F0B481282DD0
:10DFD80040F0BD800B68DFF8A0829A4E591C0222DF
:10DFE80021601A70236806275A1C22601F70236854
:10DFF8000A22591C21601A70236801255A192260C7
:10E008001D70B8F800102046F5F789F8B8F8021026
:10E018002046F5F784F823685A1922601F70236890
:10E028005022591921601A70236800225919216059
:10E038001A7031882046F5F772F871882046F5F78E
:10E048006EF82B46B1E7822D23D0C0F08881A02D31
:10E0580000F07981FE2D7AD17B4D05F1080635F85F
:10E06800021B2046F5F75BF8B542F8D101252B468F
:10E078002846638112B0BDE8F0870A680021531C66
:10E088000125236028462B461170638112B0BDE834
:10E09800F0870B686D4A694D11786D4A581C2060ED
:10E0A800197011892046F5F73AF8634B22681B88E6
:10E0B800FF2B02F10101A8BFFF2321601370A9689B
:10E0C80081F3100189B22046F5F729F8296801F390
:10E0D8000F0189B22046F5F722F85E4B22681978BD
:10E0E800CDE70B685A4D591C6A7821601A7023686D
:10E0F8002A78591C21601A702368AA78591C216053
:10E108001A7029892046F5F70AF823686A79591C94
:10E1180021601A702268A979B1E74F4B1D780B3D31
:10E1280015F0FF05A2D04D4F00220A2621683B8832
:10E13800481C20600E702168FF2B02F10102A8BF65
:10E14800FF23481CAA4220600B70EFDB8EE72146B4
:10E158002846F6F78DF9002888D1742D00F07181D2
:10E16800772D40F04E81336872689A421BBF5A1C63
:10E178003260014619783A4A204619F083FF75E75C
:10E18800022D00F0368100F22381012DDFD10B68CA
:10E198000022591C21601A7023685A1C22601D70C5
:10E1A80022682421531C23602B461170FDE6442D60
:10E1B800CDD1002A3FF45AAF2A4B136001252B46D4
:10E1C800F3E6052DC3D10B2227492046F4F779FF42
:10E1D800082226492046F4F774FF0125072224491E
:10E1E8002046F4F76EFF2B46DFE60A68214B01252F
:10E1F800511C21601570226805215019206011708A
:10E2080022680A21501920601170226800215019D3
:10E2180020601170226819785019206011702268E6
:10E228005978501920601170226899785319236021
:10E238002B461170B9E600BFA85500209C55002058
:10E24800B6460020F82D00203C56002056560020E7
:10E25800A0460020CC4600204C540020082E002068
:10E26800F1730208B54300089C220308A82203089A
:10E278009855030801330020084B00202A46C74957
:10E288002046F4F71EFF00212046F4F748FF2268D5
:10E298000221F4E60B68C24AC24F581C11212060C3
:10E2A800197023681278591C21601A70236897F82E
:10E2B8005B20591C21601A70236897F85A20591C52
:10E2C80021601A70B7F856102046F4F728FF00218D
:10E2D8002046F4F724FFB7F858102046F4F71FFF3C
:10E2E800BD1E07F1480635F8021F2046F4F717FF50
:10E2F800AE42F8D12268AC4B0C21501C20605D184E
:10E308001170226813F8011F501C9D422060117083
:10E31800F7D123680222591C21601A70B7F85C10E3
:10E328002046F4F7FCFE0125B7F85E102046F4F706
:10E33800F6FE2B4639E69D4B196820460125F4F771
:10E34800D7FE2B4694E69A4B08461968F4F7D0FE98
:10E35800984B20461968F4F7CBFE974BECE7974BA0
:10E368001E780A3E16F0FF063FF480AE944B954F98
:10E378001E4403F101080A2313E0502B7ED0002528
:10E3880029462268501C206020461370F4F7C7FE07
:10E3980029462046F4F7C3FEB0453FF467AE18F8A7
:10E3A800013B0A2BE9D1884A9568116805EB850578
:10E3B8004FF6FF726D009542A8BF15469142A8BF5F
:10E3C800114625EAE57521EAE171ADB289B2D8E7CF
:10E3D8000B6803215A1C2260197023680222581CFA
:10E3E80020601A7022680125531923602B4611708A
:10E3F800DBE50422754920460125F4F762FE2B4629
:10E40800D3E53768392D3A4628D03AD8212D00F07F
:10E41800E980292D40F008817B1C33603B780A2B6A
:10E4280001F05F80502B40F00C873046F4F739FE3E
:10E43800674F38803046F4F734FE012578802B4644
:10E44800B3E5336872689A421BBF5A1C32600146B2
:10E458001978604A204619F015FE07E67B1C3360E0
:10E468003B780A2B01F043803046F4F725FE30460E
:10E47800F4F722FE3046F4F71FFEF7E5BD68396869
:10E4880094E7552D64D0572D40F0CE807B1C336027
:10E4980017F8378B0DF107020133336013F8011CAD
:10E4A80002F8011F9F42F7D1DFF8309199F8005028
:10E4B800002DFDD1DFF828A10126042089F800608D
:10E4C8001CF04EFCDAF80000F3F74AFD424B2846F0
:10E4D8001E701CF099FC28461CF096FC09201CF0C4
:10E4E80093FC40461CF090FC02AF3D460DF13E08FF
:10E4F800EE1BF6B20A201CF087FC30461CF084FCA8
:10E5080015F8016B0B201CF07FFC30461CF07CFCDE
:10E518000020F2F7DBFC4545EAD108201CF074FC2A
:10E52800A0201CF071FCA0201CF06EFC00201CF048
:10E538006BFC10F02006F6D1DAF80000F3F715FDB1
:10E54800012502201CF00CFC89F800602B462CE504
:10E558007B1C336097F80080B8F1FF0F00F0F68756
:10E56800B8F1FE0F00F0D4873046F4F79AFD33680F
:10E578007268D21A002A07DD5A1C32601B781BB950
:10E58800B8F10B0F40F2D787B8F1240F00F29B8245
:10E59800044B012523F818002B4606E55960002096
:10E5A800D0670020344600207D46002044340020F7
:10E5B800ACF7FF1FB0F7FF1FB4F7FF1F4C54002044
:10E5C80038FA0208FC2D0020C42D002094220308EC
:10E5D800F82D0020397F0208E23A0020DA3A0020BC
:10E5E800C86700203B467A1C32600E4D13F8022B98
:10E5F8006A7033607B782B70FB1C3360BB78AB7020
:10E608003046F4F74EFD33682881591C1A463160AC
:10E6180012F8021B697132605B78AB7101252B46D9
:10E62800C3E400BFA046002070680B3DC31BEF2D5C
:10E6380000F2498201A151F825F000BF57EF000808
:10E64800CFEA0008CFEA0008CFEA0008CFEA0008BE
:10E65800CFEA0008CFEA0008CFEA0008CFEA0008AE
:10E66800CFEA0008CFEA0008CFEA0008CFEA00089E
:10E67800CFEA0008CFEA0008CFEA0008CFEA00088E
:10E68800CFEA0008CFEA0008CFEA0008CFEA00087E
:10E69800CFEA0008CFEA0008CFEA0008F1EF000847
:10E6A800CFEA0008D7EF0008CFEA0008B5EF000866
:10E6B800CFEA0008CFEA0008CFEA00088DEF00088B
:10E6C800CFEA0008B3F00008CFEA000881F000089C
:10E6D800CFEA00080DF10008CFEA000845EF00086E
:10E6E800CFEA00082BF30008CFEA000891F20008EF
:10E6F800CFEA0008CFEA0008CFEA0008CFEA00080E
:10E7080075E00008CFEA000875F20008CFEA0008B3
:10E71800CFEA00085BF20008CFEA000801F200081F
:10E72800CFEA0008CFEA0008CFEA0008CFEA0008DD
:10E73800CFEA0008CFEA0008CFEA0008CFEA0008CD
:10E74800C1F10008CFEA000873F10008CFEA000819
:10E75800CFEA000833F10008CFEA0008CFEA000842
:10E76800CFEA0008CFEA0008CFEA0008CFEA00089D
:10E77800CFEA000829F40008CFEA0008B5F300083A
:10E78800CFEA0008D7EE0008CFEA000843EE0008F9
:10E79800CFEA00081BEE0008FDED0008CFEA0008EC
:10E7A800CFEA0008CFEA0008CFEA0008CFEA00085D
:10E7B800CFEA0008CFEA0008CFEA0008CFEA00084D
:10E7C800CFEA0008CFEA0008CFEA0008CFEA00083D
:10E7D800CFEA0008CFEA0008CFEA0008CFEA00082D
:10E7E800CFEA0008CFEA0008CFEA0008CFEA00081D
:10E7F800CFEA0008CFEA0008CFEA0008CFEA00080D
:10E80800CFEA0008CFEA0008CFEA0008CFEA0008FC
:10E81800CFEA0008CFEA0008CFEA0008CFEA0008EC
:10E82800CFEA0008CFEA0008CFEA0008CFEA0008DC
:10E83800CFEA0008CFEA0008CFEA0008CFEA0008CC
:10E84800CFEA0008CFEA0008CFEA0008CFEA0008BC
:10E85800CFEA0008CFEA0008CFEA0008CFEA0008AC
:10E86800CFEA0008CFEA0008CFEA0008CFEA00089C
:10E87800CFEA0008CFEA0008CFEA0008CFEA00088C
:10E88800CFEA0008CFEA0008CFEA0008CFEA00087C
:10E89800CFEA0008CFEA0008CFEA0008CFEA00086C
:10E8A800CFEA0008CFEA0008CFEA0008CFEA00085C
:10E8B800CFEA0008CFEA0008CFEA0008CFEA00084C
:10E8C800CFEA0008CFEA0008CFEA0008CFEA00083C
:10E8D800CFEA0008CFEA0008CFEA0008CFEA00082C
:10E8E800CFEA0008CFEA0008CFEA0008D3ED000815
:10E8F800CFEA0008CFEA0008CFEA0008CFEA00080C
:10E90800CFEA0008CFEA0008CFEA0008CFEA0008FB
:10E91800CFEA0008CFEA0008CFEA0008CFEA0008EB
:10E92800CFEA0008CFEA0008CFEA0008CFEA0008DB
:10E9380079ED0008CFEA000841ED0008CFEA0008A9
:10E9480065EC00084BEC00082FEC0008CFEA000843
:10E9580015EC0008CFEA0008EDEB0008CFEA000844
:10E9680093EB0008CFEA000865EB0008CFEA00083F
:10E97800CFEA000843EB000815EB000801EB00089C
:10E98800D9EA0008B1EA00088FEA0008CFEA0008CF
:10E99800CFEA0008CFEA0008CFEA0008CFEA00086B
:10E9A800CFEA0008CFEA0008CFEA0008CFEA00085B
:10E9B800CFEA0008CFEA0008CFEA0008CFEA00084B
:10E9C800CFEA0008CFEA0008CFEA000875EA000895
:10E9D800CFEA0008CFEA00081DEA0008CFEA0008DD
:10E9E800CFEA0008CFEA0008CFEA0008CFEA00081B
:10E9F800CFEA0008CFEA000805EA0008BE4B1B78FA
:10EA0800DB0760D40125F6F70DFDF6F7E7FE2B4688
:10EA1800FFF7CBBA7B1C33603B780F2B53D8BA1C5B
:10EA28003260C3EBC303B54A7978D154F91C31601D
:10EA38001344BA785A703A1D3260FA789A707A1D7F
:10EA480032603A79DA70BA1D32607A791A71FA1D31
:10EA58003260BA795A7107F108023260FA799A710C
:10EA6800012509F075FA2B46FFF79FBA3046F4F7EF
:10EA780018FBA34FF8813046F4F713FB0125B88142
:10EA88002B46FFF792BA3046F4F70BFB9D4F3882BE
:10EA98003046F4F706FB78823046F4F702FB01258E
:10EAA800B8822B46FFF781BA3B467A1C326013F8CE
:10EAB800020B3360FB1C79783360BA7815F0E4FCFC
:10EAC80000287FF4D3AA4FF0FF352B46FFF76DBA25
:10EAD8003B467A1C32608C4A13F8021B1170336073
:10EAE800874A7B789370FB1C3360884BBA789A709E
:10EAF80001252B46FFF759BA854B864918684E22DF
:10EB080001251EF065FA2B46FFF74FBA3A467B1CE3
:10EB18003360814B12F8021B197032607A785A7090
:10EB2800FA1C3260BA789A703046F4F7BAFA7B4B1E
:10EB38000125D8802B46FFF738BA3046F4F7B1FAEA
:10EB4800764F38803046F4F7ACFA78803046F4F7E0
:10EB5800A8FA0125B8802B46FFF727BADFF8CC8141
:10EB680098F80030002B3FF481AA6D4F00253046FD
:10EB7800F4F797FA09F0CAFE98F80030A7EC010AF2
:10EB880001359D42F3DBFFF771BA0D2B9BD17B1C3E
:10EB980033603D78072D96D8DFF8948130460C27EE
:10EBA800F4F77FFA07FB05F708EB0705A88030465E
:10EBB800F4F777FAE8803046F4F773FA3368288177
:10EBC8001A46591C316012F8021BA97232605B7830
:10EBD800EB723046F4F74EFA012548F807002B4649
:10EBE800FFF7E3B97B1C33603878060600F113851C
:10EBF800414B1B78DD073FF539AA032828BF0020C1
:10EC08000125F6F7F7FB2B46FFF7CFB93A4B1B78F0
:10EC1800D8073FF52BAA0125F6F7CAFFF6F7DEFD60
:10EC28002B46FFF7C2B9344B1B78DA073FF51EAA0B
:10EC38003C4A1378012543F0040313702B46FFF771
:10EC4800B4B92D4B1B78D9073FF510AA364B4FF4B2
:10EC5800C87201251A802B46FFF7A7B9092B7FF741
:10EC680032AFDFF8D0803B467A1CD8F800503260CB
:10EC780013F8022B2A7033607B78AB70FB1C33606F
:10EC8800BB78642BA8BF64233A1D6B713260FB7894
:10EC9800642BA8BF64237A1DAB7132603B79EB719A
:10ECA800BB1D33607B79642BA8BF6423FA1D2B72CC
:10ECB8003260BB79EB7007F108033360FB792B7185
:10ECC8003046F4F7EEF9726833686881D11A002982
:10ECD8000CDD591CD8F800003160521A002A197846
:10ECE800417203DD9A1C32605B784370012513F092
:10ECF800A9FE2B46FFF759B9F2660020BC42002056
:10ED0800184B0020304C0020C8680020284B0020F9
:10ED180050600020F8130308104B00202045002005
:10ED2800784400209C460020706F00204C5400203E
:10ED3800C8410020E85E0020BF4B1868FB1C024653
:10ED48002137991E316013F8031C1170591E316068
:10ED580013F8021C5170336013F8011C91700333CF
:10ED68009F4202F10302ECD109F0A0FCFFF77EB943
:10ED7800C3F34705122D3FF6A6AEB5B112AB0DF1A0
:10ED8800060803EB4507C146423F3046F4F789F9C8
:10ED980029F8020F4F45F8D1A84B38F8022F23F86D
:10EDA800022FC845F9D1112D09D8A54A6B00023B9D
:10EDB80013440021223223F8021F9A42FBD1A14AB0
:10EDC80001231D461370FFF7F0B83B467A1C3260EA
:10EDD80013F8025B3360FB1C78783360B978002D38
:10EDE80000F05984012D7FF441A902F057FE2B460B
:10EDF800FFF7DBB8944B1B7813F001017FF463AE87
:10EE08007B1C33603878012502F084FD2B46FFF720
:10EE1800CCB83B467A1C32608C4A13F8021BD1707E
:10EE280033608B4A7B785371FB1C3360894BBA780B
:10EE3800DA7001252B46FFF7B8B83046F4F731F9F8
:10EE48003046F4F72EF93046F4F72BF93046F4F74C
:10EE580033F93368784D1946581C2A68306011F820
:10EE6800020B82F82C003160597882F83610D91CD0
:10EE780031609B7882F837303046F4F71DF9304618
:10EE8800F4F71AF93046F4F717F930462F68F4F713
:10EE980008F978873046D5F80080F4F702F9376822
:10EEA8007368A8F83800DA1B012A0ADD7A1C2B6877
:10EEB80032603A7883F82E203046F4F7FDF8376848
:10EEC8007368DB1B032B00F3EC8328684CE77B1C7F
:10EED8003360594DDFF89C813B7888F8053030461F
:10EEE8002F68F4F7DEF838843046D5F80090F4F748
:10EEF800D8F873683768A9F81E00DA1B072A00F3E8
:10EF0800AE83DA1B032A00F39D83DB1B002B05DD90
:10EF18007A1C2B6832603A7883F82620F6F7C0FB13
:10EF28001BF0AEF94C4B1B68002B00F03A832868A5
:10EF3800012509F09BF82B46FFF737B87B1C336097
:10EF4800464B3A785A7501252B46FFF72EB8444AA6
:10EF5800102B4FF0000128BF102311605160916001
:10EF6800D1601174002B3FF481A83168013A0B4439
:10EF78000131316011F8010C02F8010F8B42F7D111
:10EF8800FFF774B87B1C3360364A39781170C31A9E
:10EF9800002B7FF76BA8BB1C33607B78003318BF4E
:10EFA8000123012553702B46FEF7FFBF3046F4F7C7
:10EFB80078F82D4F38603046F4F773F878603046AB
:10EFC800F4F76FF80125B8602B46FEF7EEBF274F20
:10EFD80000233B603046F4F74DF83B6801250343B6
:10EFE8003B602B46FEF7E1BF7B1C33603D78132D59
:10EFF8003FF669ADBB1C3360787819F07DF80028BE
:10F008003FF461AD1A4B027803F82520FA1C3260F0
:10F0180003EB8503BA785A703A1D3260FA789A7011
:10F028007A1D326004493A79DA700868012513F0CC
:10F0380097FC2B46FEF7B9BF5060002036630020CE
:10F04800386300205C630020F2660020184B002023
:10F05800C8480020284B00203C4B00207C4F002053
:10F0680038600020544B0020143100204434002024
:10F07800584B0020C8680020BF4D05F140073046B6
:10F08800F4F70FF83368A5F88000591C1A46316068
:10F0980012F8021B85F8821032605B7885F883309D
:10F0A8000435AF42EBD1FEF7E1BF7B1CB34D3360B3
:10F0B8003B782B723046F3F7F4FFA8833046F3F71A
:10F0C800F0FF28833046F3F7ECFF336868835A1C57
:10F0D80032601B78EB7473689A1A032A00F37C82F7
:10F0E8003768DA1B052A00F36782DB1B002B7EF7E3
:10F0F800BDAF7B1C33603B7885F8213001252B465A
:10F10800FEF753BF7A1C32603D781F2D3FF6DBAC0B
:10F11800052B7FF4D8AC3046F3F7ACFF964B43F899
:10F12800250006F029FFFEF7A1BF954B1B78012BA0
:10F138003EF69CAF39467B1C3360DFF8648211F8D9
:10F14800023B88F80230FA1C31607B783260821A00
:10F15800012AB97840F36A823046F3F7A2FF012505
:10F16800A8F800002B46FEF720BF7B1C336097F8F9
:10F178000080B8F1110F3FF6A6ACBB1C3360814D7F
:10F188007B7805F818303046F3F78BFF40F6CA0352
:10F198009842A8BF184640F2EE23984205EB480172
:10F1A800B8BF18460125A0F2EE222B46192092FB83
:10F1B800F0F24A70FEF7F9BE3B467A1C724D326097
:10F1C80013F8022B2A7133607B786B713046F3F7A2
:10F1D80068FF336828805A1C32601B78AB71304650
:10F1E800F3F75FFF336868805A1C32601B78EB7155
:10F1F80001252B46FEF7D9BE7B1C3360634B3A785A
:10F20800DFF8A0811A700023C8F800303046F3F701
:10F2180031FF3268D8F8003058495D4D0343501C1F
:10F22800C8F80030306013780B723046F3F739FFB6
:10F2380028603046F3F735FF68603046F3F731FF52
:10F24800A8603046F3F72DFF3046F3F72AFFFEF7A4
:10F258000DBF504B03F10802791C3160397803F86F
:10F26800011F9A423EF402AF3768F5E73B467A1C25
:10F278003260494A13F8021B917033607B785370EF
:10F2880001252B46FEF791BE0721B3FBF1F1C1EB37
:10F29800C1055B1B7FF417ACC9B24F1EFFB2002932
:10F2A8003EF4E4AEDFF8008101371D462EE098F900
:10F2B8000A209A4200F0EC8198F912209A427FF4D1
:10F2C80002AC4FF0020A08EBCA09304689F802304E
:10F2D800F3F7E7FE336828F83A001A46591C3160FC
:10F2E80012F8021B89F8031032605A7889F8042052
:10F2F800DA1C32609A7889F806201A1D32600135C6
:10F30800DB7889F80530BD423EF4B0AE531C33605B
:10F3180092F9003098F902209A42C8D14FF0000AB9
:10F32800D1E77B1C33603B780E2B3FF6CCABBA1C85
:10F338003260787803283FF6C6AB1849062202FBEC
:10F3480003F28B18FD1C58713560B87888543A1D43
:10F358003260FA785A707A1D32603A799A70BA1D1A
:10F3680032607A79DA70FA1D3260BA791A71012539
:10F378002B46FEF71ABE00BF305F00207C4F0020EE
:10F388002F34002010660020A4410020544B002098
:10F39800143100207B4F0020344B002071400020A6
:10F3A800B046002044340020DC6700203B467A1C2D
:10F3B8003260DFF8348313F8022B88F802203360B8
:10F3C800BD4A7B781370FB1C3360BC4DBB782B7136
:10F3D8003B1D3360FB78092BA8BF09233046AB706F
:10F3E800F3F75FFE376873682880DA1B012A05DDAA
:10F3F8003046F3F756FE37687368E881BB4240F041
:10F40800C780F6F74DF9336872689A423EF42EAE1B
:10F418005A1C32601B78EB7001252B46FEF7C5BDE0
:10F428003046F3F73EFE054605F05AF8FF283EF44D
:10F438001DAE12A9002301F8423DEF080DF10500A9
:10F448008DF80530013705F02BF89DF80530FFB22F
:10F4580005F00705BB4205F1010503D19DF806300B
:10F46800AB4203D02946384605F026F8336872685F
:10F47800D21A012A7EF7FAAD5A1C12A8326000226D
:10F488001D7800F8412D04F0FFFF9DF80730AB42CE
:10F498000AD08B4B1B683BB19A79AA4204D31B68EC
:10F4A8001B690BB128469847336812A85A1C32606A
:10F4B80000221D7800F8402D04F0DAFF9DF808308E
:10F4C800AB423EF4D3AD7E4B1B68002B3EF4CEAD71
:10F4D8001B685B69002B3EF4C9AD28469847FEF7C8
:10F4E800C5BD3046F3F7DDFD764FFEF7A2BFBB1C66
:10F4F8003360754B7A781A70FA1C3260BA785A7091
:10F508003A1D3260FA789A7001252B46FEF74DBDF8
:10F51800BB1C33607D78022D3FF6D5AA3046F3F741
:10F52800C0FD6A4B03EB45034FF0FF35A3F85C00C1
:10F538002B46FEF73ABD654B0030984418BF0120B2
:10F54800012588F84A002B46FEF72FBDBB1C336007
:10F558005F4B7A781A70FB1C3360DFF87081BB78D8
:10F5680088F85B303B1D3360FB7888F85A303046AA
:10F57800F3F797FDA8F856003046F3F792FD3046AA
:10F58800F3F78FFD0125A8F858002B46FEF70DBDAF
:10F598007B1C33603B78003318BF012388F80730A1
:10F5A8002FE74C484C494D4A4D4B036001250B60F1
:10F5B80013602B46FEF7F9BC7B1C33603B78EB727B
:10F5C8003046F3F757FD3368E8605A1C32601B7801
:10F5D8002B743768736888E53046F3F762FDA884B2
:10F5E8003046F3F75EFD37687368E884DA1B032A50
:10F5F8007FF777AD3B467A1C326013F8022BAA7767
:10F6080033607B7885F820303046F3F74AFD376859
:10F618007368688465E500F07F00032828BF002030
:10F62800012502F057FA2B46FEF7BFBC2D4A128877
:10F63800012512FB03F22B4692FBF1F2A8F80020F9
:10F64800FEF7B3BC3046F3F72CFDA8F80E003046A1
:10F65800F3F727FD37687368A8F8100055E43046BB
:10F66800F3F71FFDA8F80A003046F3F71AFDA8F8CB
:10F678000C0030462F68F3F714FD78843046D5F82F
:10F688000090F3F70EFD37687368A9F8240038E492
:10F698004FF0010A17E6012508F07EFE2B46FEF71B
:10F6A80084BC30462F68F3F7FCFC788630462E6819
:10F6B800F3F7F7FCB08608E40C4B0020304C002030
:10F6C8004C600020084B0020013300203446002005
:10F6D800D06700203443002088430020F0430020F6
:10F6E8005F0400088C490020C86800202DE9F04F0D
:10F6F800734B744A1C7893B000F59C4120318146C5
:10F7080007911160002C00F0C4846F4A126890427F
:10F7180040F2DC816D4A6E491768DFF8ECB16D4D37
:10F728000492013C03911C7007F48057002F40F0AD
:10F73800DA81694B05931E7806F00106039B5B7D11
:10F74800002B40F07B84049B1B68190400F1CB86D6
:10F75800624B9945AB7800F25883002B40F05883F0
:10F76800049BD3F8009019F4805A40F03984039B25
:10F77800BBF906805B8B9845B4BF4FF000084FF08B
:10F788000108574B1B6813F0805300F0E081002EEE
:10F7980000F0E1810399534A498C92ED037A07EE10
:10F7A800901AF8EEE77AB4EEE77AF1EE10FA80F202
:10F7B8004487B8F1000F40F0D6814B4C94F88C2068
:10F7C800002A40F0D081494A4949106890F82D0034
:10F7D80000220A604A608A60002840F0C481454AD5
:10F7E8001070002E40F0C581434B1A78002A50D182
:10F7F8000399BBF900E04E8B898BBBF90200764573
:10F80800B4BF8024002444F040037145D8BF234688
:10F818009B0843F080048642B8BF234643F0400467
:10F828008142D8BF1C46BBF904E0BBF90600A40816
:10F8380044F080037645B8BF1C4644F04003714548
:10F84800D8BF23469B0843F0800E274CB042C8BF60
:10F85800734643F0400E94F88E608842B8BF7346F2
:10F868009E4201F08F80A4F8902084F892202349CA
:10F8780084F88E300E78002E00F0E4875F2B01F0BC
:10F8880037806F2B00F03187059B1B78DE0740F12E
:10F89800F386049B1A4A1B68069203F00403002BA4
:10F8A80040F0398410AF174C00237B6004F15009F5
:10F8B800109340F6330A4FF0190840F2833628E0D7
:10F8C800546400203463002050640020706B0020D2
:10F8D8007C4F00209C380020F2660020404B4C00F2
:10F8E800D046002058560020EC2C00205060002004
:10F8F80008490020B82C00203C620020190C002088
:10F90800D8460020584B0020D054002004344C45E1
:10F9180020D0A278E3789A4218FB0260F6D2617888
:10F92800043118FB03623BF911305345A8BF534615
:10F93800B3F5617FB8BF4FF461739842E6DA9A4233
:10F94800E4DB21782429E1D838460434F3F7CCFDE8
:10F958004C45DED1B34BB44A1B7897E8030082E8E4
:10F968000300002B00F0FB830121AF48F3F7CBFD28
:10F97800002840F04981EB78002B40F04581AB4FDF
:10F98800A9483C8824F00104A4B202213C80F3F782
:10F99800BAFD002800F04181A20740F1BB86A44BC4
:10F9A80003931978DFF8D8A2A30708BF81F00201F2
:10F9B800DAF80400C1F34001F2F7DCFA24219A488E
:10F9C800F3F7A1FD30B9059A13785E0744BF23F019
:10F9D80004031370069B1B6813F00A0F40F056814E
:10F9E8003C8891480C21F3F78EFD002800F07381C4
:10F9F800904B1B7844F48074082B3C8000F0748191
:10FA08000E2B00F07181049B1B685C0544D58A4B62
:10FA18001B79002B00F0DA8014218348F3F773FD7B
:10FA2800002840F0D8800AF0C1F901201AF006F841
:10FA380090B3DFF8508200244FF0CC0902E0DCB22A
:10FA4800022C29D809FB04F6631C58F80650002D2F
:10FA5800F5D1C378794A90F9020052F8233001951C
:10FA68000322009201212A4619F0FEFD034604EB09
:10FA7800440000EB0010049353B1294608EB8000C2
:10FA8800CC221FF06EFD049B48F806300134E4B226
:10FA98001AF0E2F90028D3D1059B1B78D80740F16A
:10FAA80027816749674A01230B701370039BDAF8B3
:10FAB8000000197801F00101F2F75CFA069B1B6857
:10FAC8005B0700F1858113B0BDE8F08F5E4B5F4A9C
:10FAD8001F68049307F480570392DFF8ACB15C4DBC
:10FAE800002F3FF426AE00214F48F3F70CFD002805
:10FAF8007FF41FAE574B059319461B7813F0010688
:10FB08003FF41CAE544A967803F0FE030B70002EA7
:10FB18003FF414AE514C22780B2A0DD801219140A4
:10FB280040F603060E4041F0598211F4C06F03D02D
:10FB3800093A012A41F20D83DFF83CA1484ADAF874
:10FB4800001051600B2203F001062270F6E519F44B
:10FB5800800F7FF41CAE434C002284F88C20B8F14F
:10FB6800000F3FF430AE404A01211170002E3FF4DF
:10FB78003BAE19F0100F3FF437AE3C4A1278D2066C
:10FB88003FF532AEBAF1000F7FF42EAE002B7FF4B2
:10FB98002BAE19F4800F7FF427AE354B1B78002B62
:10FBA80001F05582334B9B78B8F1000F41F0E182A8
:10FBB8003BB1314A314B12681B689B1A002BC1F2CA
:10FBC8007082284C012384F88D300DE6059B1B7844
:10FBD800D9077FF528AF4FF40F700CF093FF00287A
:10FBE8003FF45AAF19F028FD4FF40F700CF020FFC6
:10FBF80000283FF451AF19F01FFD4FF40F700CF0BF
:10FC080017FF0028EED147E7069B1B6899077FF589
:10FC1800B6AE064F3C8844F0010424F00204A4B2B6
:10FC28003C80BCE6D93A0020D04600202C60002059
:10FC3800A8610020544B002048560020C415030832
:10FC4800F3660020FC2B0020706B00207C4F002006
:10FC58009C380020F2660020B04600202F34002097
:10FC6800004B0020EC2C0020B82C00209C460020E3
:10FC7800190C0020344B00207C610020E05E00203D
:10FC8800AC6100200C500020D05400200621AE4862
:10FC9800F3F739FC3C88002800F0AE84650640F193
:10FCA800AC850721A848F3F72EFC00283FF499AE4D
:10FCB800A64BA74AB3F90430A6493C8882FB030245
:10FCC800DB17C3EBA2030B809F480C21F3F71BFC47
:10FCD80000287FF48DAEA04B1B7824F48074A4B266
:10FCE800082B3C807FF48CAE24F040043C808AE6EC
:10FCF8009A4B93F80090B9F1000F5FD1DFF8A88212
:10FD0800974E18F8030C35784146A8F1030412F011
:10FD1800F7FD002800F09083002D40F0E28304F105
:10FD28000801607912F0ECFD002841F0E4808D496B
:10FD3800A07A12F0E5FD002800F09183022D41F031
:10FD4800DE808949E07B12F0DBFD002841F0DB8092
:10FD58008649207D12F0D4FD002800F09183042DFF
:10FD680041F0A8808249607E12F0CAFD002841F067
:10FD7800BA808049A07F12F0C3FD002800F091836B
:10FD8800062D41F0B4807C4994F8230012F0B8FDA8
:10FD9800002840F0A086794994F8280012F0B0FDB8
:10FDA800002800F09183082D40F07F86744994F86C
:10FDB8002D0012F0A5FD002840F09183714B01221F
:10FDC8001A701BF07DFB069B1B685B077FF57BAEFB
:10FDD800032012F0BFFD002800F0CF853B8813F008
:10FDE80008047FF470AE082019F010FF6648674DCC
:10FDF8006749684A684BBBF8066000682E8008604F
:10FE080014601C6013B0BDE8F08F0BB90123AB7010
:10FE18001B2012F09FFDDFF8948195F8217095F86A
:10FE280020305E4C8146B246052B00F20181DFE8A6
:10FE380013F0BF007F000600FB00FD00F100012F5A
:10FE480004BF052385F82030BAF1000F12D0039BB8
:10FE5800B8F80000B3F918100022134661F30F0335
:10FE680061F30F0260F31F4261F31F43CBF80420D4
:10FE7800CBF800304A4E6A6933689A4280F0AD8404
:10FE880047F230520323EA6185F82030238843F093
:10FE98000203238011F076FC3268EB6913440422D4
:10FEA800AB6185F82020012F40F0AD853368AA6941
:10FEB8009A4280F0BD803B4B187820B912F04AFD79
:10FEC800002840F0B580238823F00203238032689D
:10FED800B8F80230642101FB03234FF4806000224C
:10FEE8002B6185F82020EA7019F088FE95F82030FB
:10FEF8009AE712F05BFD012807D1294EB8F80230C5
:10FF08003268642101FB03232B61B9F1000F03D090
:10FF180098F80630002B7FD1012F00F08980204E01
:10FF28002A6933689A42C0F07885012385F8203021
:10FF3800012F6FD098F80730012B00F0A08007F050
:10FF4800CDFB95F820306FE7D046002030600020C8
:10FF580067666666C42B0020544B0020F3660020B9
:10FF680098000020654100206A4100206F41002070
:10FF780074410020794100207E4100208341002007
:10FF880088410020FC2B0020BC460020D02B0020FC
:10FF9800DC2B0020D42B0020CC2B0020DE460020B8
:10FFA8007C610020190C00205B410020A441002046
:10FFB800BAF1000F9DD14FF48060B9F1000F00F045
:10FFC800DF8219F023FE059B1E7800232B61049B1A
:10FFD800D3F8009019F4805A06F001063FF4C7AB35
:10FFE8001D219948F3F78FFA00287FF4C0AB974A90
:08FFF800039BD2881B8BBBF9AF
:020000040801F1
:100000000680991A884540F3168513449845B4BF75
:100010004FF000084FF00108FFF7B7BB8E4E5AE7CC
:1000200007F060FB03224FF47A7385F82020EB6120
:10003000894E2FE7884E3AE7059B1E7806F00106A9
:10004000FFF792BB039A013BD27D3BF91330002AA4
:1000500040F0DC82A3F57A73B3F57A7FA8BF4FF442
:100060007A7323EAE37307EE903A9FED7C7AF8EE19
:10007000E77A67EE877A7A4AFCEEE77A17EE903AEB
:100080001380FFF769BB07F02DFB032240F6B8335E
:1000900085F82020EB61704EFCE6724F3B78002B18
:1000A00000F0D286704BDFF8D481DFF8D4B1DFF8EE
:1000B000D4A1039345465E46049099460EE019F894
:1000C00004109847032C28DC88B93B782AF8020FE3
:1000D00001349C4205F1040580F2DA80072CE1B27C
:1000E0003046DBF80430EADD984700B2EDE738F837
:1000F00024206B88801A4FF47A719B1A01FB00F060
:1001000040F6CA0290FBF3F00844904240F2EE231E
:10011000A8BF10469842B8BF184600B2D5E7534C66
:1001200094F8963053B1059B1B78D90706D5039BED
:10013000BBF906205B8B9A4200F38E841121444860
:10014000F3F7E5F9002800F06A8294F89A302BB9A9
:1001500094F8943013B93223A4F89830012384F82A
:100160009A30FFF7A3BBDFF820A1DFF820813F4CD6
:100170001F460AF15A064FF0010951461AF8010CC0
:1001800012F0C2FBF8B19AF804009AF802309AF81B
:1001900003E000EB400104EB8101013BD1F8A0201A
:1001A00003EB4303434493420DD094F8CC2081F8F1
:1001B0009CE009FA00F022EA0000C1F8A030C1F882
:1001C000A47084F8CC000AF1060AB245D5D12849BA
:1001D000214A284B284C09681B78D2F800A00891C6
:1001E0000793A4F19C090026636853B31F7847B3B3
:1001F000A168AAEB010100290ADB99F8CC100120C3
:10020000B04021EA00010AF5FA7089F8CC10A0602C
:10021000079AB2B1217858780431C9B2002840F069
:100220001682039A3BF91110108B00F1C80E71452C
:1002300040F3C48399F8CC109B783141CA0740F150
:1002400036840136042E04F10C04CDD1FFF790BBA7
:10025000D0460020204500207C610020AAF1823F8A
:10026000B6460020A96400207C4F0020EC2C002022
:10027000E85E002090380020882D0020DC650020FA
:100280008C370020EA2C0020724000203CFA020843
:10029000DDF81090BE4A04921146BE4A0968A2FBDE
:1002A000092A42F201020A404FEA9A1A059200F026
:1002B000B281B94DB948BA4CBA4A95F800E0007815
:1002C00084F800E01070BEF1000F04D0B54A92F837
:1002D00000E08EF0010EB44C0F2084F82400002BB7
:1002E00000F09482B14B039E0C931B78B6F826C0A5
:1002F0000B931D463B78B78C039EAD4A368B0E960A
:100300002E46A2FB0552520802EB4202B21AD2B2AA
:10031000CDF824C001F48051089294F82580DFF8CC
:10032000A4B2DFF8D4C20A900AF5967276460F910D
:1003300004F1280500200692CDF83490A646002E40
:1003400000F0F1813EF910201FFA82F9B9454FEA19
:10035000400103D3099CA14540F229825CF820208A
:10036000924580F0E9813BF90120059C002C40F08A
:10037000FD81013098422BF8012005F10605DEDBF6
:100380000A998C4A8EF824100F290CBF01210021F4
:10039000DDF834908EF82580117000F03E82864D95
:1003A000864EDFF858A23488DAF80000A9686A6837
:1003B000E86044F00404401A9042784F3480794C4D
:1003C0004FF0010188BF00223970217088BF85F885
:1003D0002120002B00F03582049A03991768784E8B
:1003E000B1F824C0B1F818E0764817F480573446C5
:1003F00040F0458239460EE0627802EB820202EB61
:10040000820202F2EE2292B20131994220F8022BCE
:1004100004F102040ED016F81120002A00F0CB815E
:10042000022AE9D00131028820F8022B994204F116
:100430000204F0D10C9A137801331370FFF77AB9E4
:1004400008F10501607912F05FFA00283FF473ACFF
:10045000012D40F0548504F10D01A07A12F054FAF8
:10046000002840F050855849E07B12F04DFA0028F2
:100470003FF472AC032D40F04A855449207D12F0C0
:1004800043FA002840F01A855149607E12F03CFA88
:1004900000283FF472AC052D40F029854D49A07F1E
:1004A00012F032FA002840F026854B4994F82300D8
:1004B00012F02AFA00283FF472AC072D40F00F83A7
:1004C000464994F8280012F01FFA002840F0F18203
:1004D000434994F82D0012F017FA00283FF472AC4B
:1004E000092D3FF46FAC4FF009094B46E4E22E4C66
:1004F000D4F88830A9EB0303002BFFF62DA9394867
:10050000394B0278597C079BC4F88830374B039FDE
:1005100033F81110364BBC7D013202F00F0289B264
:1005200091FBF4F199541C78597802709A78D87834
:1005300021440A4419791C7B10445A790144987962
:100540000A44D97910441A7A0144587A0A44997AAB
:100550001044DA7A01440A44587B997B1444DA7BCC
:1005600003190B441A4442F30B12642AF97DA8BF05
:10057000642213B209B1C2F1640307EE903A9FED11
:100580001D7AF8EEE77A74E519F03CFB1FE500BF31
:10059000706B0020D34D62101063002048210020B2
:1005A0009038002049210020EC2C002055640020C8
:1005B000ABAAAAAACA3F00209C380020DE46002031
:1005C00010660020D05400206A4100206F410020B6
:1005D00074410020794100207E41002083410020A9
:1005E000884100203C64002084610020A06100203C
:1005F0004064002014AE2341586400207C61002038
:1006000024F04004A4B23C80FFF74FBBC3F53B632A
:1006100008331BB21EE5A94A92F800E053E694F8AD
:100620009430002B3FF442A9059B1B7813F0010383
:100630007FF43CA9012284F8943084F89520FFF7D8
:1006400035B99F4C012284F88C20FFF790BA01281D
:1006500000F0CA8399F8CC200123B340013613433C
:10066000042E89F8CC3004F10C047FF4BDADFFF703
:100670007FB9059B934A1B781060DB0700F1FA8174
:1006800094F8921000297FF408A9B4F99030322B25
:100690007FF703A994F88E200120572A84F892004E
:1006A00000F0F183049B1B6813F0040302D05A2A64
:1006B00000F0E0845D2A00F07C845B2A00F08384F3
:1006C0005E2A00F08384562A00F0E384972A00F023
:1006D000B684A72A40F038847B49049B0A781B68BB
:1006E00042F004020A70794A069203F00403FFF70D
:1006F000DAB8B2F5FA7FFFF6D0A894F89220002A73
:100700007FF4CBA8059B1B780121DF0784F89210AA
:1007100000F1108410F0ACFBFFF7BFB844F0020406
:100720003C80FFF740B9002F3FD05CF82020924575
:100730004FEA4001FFF417AE654A654C525C04EB8A
:100740000109002A00F08F80022A47D199F8012080
:1007500002EB820202EB820202F2EE2292B2032844
:1007600033DD059C12B2002C3FF403AE089C25F843
:100770001420B8F1000F03D10B9C022C7FF6F9ADC9
:100780006A88B5F80090B5F804804A449044514A0C
:100790000FFA88F882FB08424F4CA2EBE87224F86B
:1007A000018012B24FF00108E3E53A464100069C91
:1007B0004CF82040D9E5CAB2022A04D9032A7FF4B2
:1007C00031AE624620E672461EE6012404FA00F9C4
:1007D0000A9C24EA090412B20A94C6E53BF80120F7
:1007E000BDE73E4B1B78002B7FF44EABBAF1000FF8
:1007F0003FF44AAB012F7FF41FAC95F82030FFF790
:1008000017BB44F040043C80FFF74FBA3449354AE7
:100810000C91DFF8E0B0012111701B2132480593E3
:10082000F2F775FE059B00287FF4B9AD2F4DDFF878
:10083000C0A0EA68DAF80030AB609B1AC82B00F25F
:100840001483049B1F6807F48057F3E5314626485C
:10085000F2F75DFE00283FF40CAF84F8936010F0CF
:1008600007FBFFF715B8C2B2022A40F2BB82032A87
:10087000B4D10E9A0F9C002C08BF3A466FE70021B6
:100880000FE0627802EB820202EB820202F2EE22B9
:1008900092B20131994220F8022B04F102043FF494
:1008A000C9AD16F811201AB1022AEAD00288F0E781
:1008B000CAB2032AFAD87246EBE700BF903800208C
:1008C000EC2C0020E45E00209C460020D84600204E
:1008D00010660020565555555C2D0020A82C002090
:1008E00055640020CA3F0020D04600209C380020DC
:1008F0007C610020D0540020B2F5FA7FFEF6CDAF27
:1009000094F89230002B7EF4C8AF059E3378012115
:1009100013EA010084F8921000F09A82AE4A9278AD
:1009200023F001033370002A3EF4B7AFAB4C2378B9
:100930000B2B18D801FA03F240F603010A427EF4A9
:10094000ACAF12F4C06F0ED0093B012B0BD8452081
:1009500015F000FAFF2015F0FDF9A14815F0E6F9B1
:10096000002015F0F7F99F499F4A049B09681B680E
:1009700051600B2222709D4A069203F00403FEF799
:1009800092BF082019F03EF9FFF7A1B8984A99499B
:100990001068B4F99020C66981FB06018911F61729
:1009A000701A00F5FF407F3082423EF764AF891B2A
:1009B0000A4412B2A4F89020FEF75DBFC838814205
:1009C0003DDA99F8CC109B783141C8073FF539AC36
:1009D000C3F10008791E162900F2BF80DFE811F08C
:1009E000B601CA019C011401DE01EF018901760103
:1009F00061014C013701BD0014012401EF0189019F
:100A00007601E800D400C000AD009700830005998E
:100A10003268EB690E781344AB6106F00106FEF70D
:100A2000A3BE06F05FFE032240F6B83385F820200F
:100A3000EB61FFF72FBA4FF00108FEF7A6BE99F859
:100A4000CC300122B24023EA02030AF5FA7289F897
:100A5000CC30A260FFF7F5BB00216748F2F757FDE5
:100A600000287FF46BAB322384F89600A4F898300A
:100A7000FFF764BB614B1B78002B3EF40EAFEB78A5
:100A8000002B7EF40AAF94F893300133DBB2032BD2
:100A900084F893307EF601AF594B5B781BB9B8F1FF
:100AA000000F7EF4FAAE10F071FEFEF7F1BE98462C
:100AB00090E74FF008094B4603EB83031C4486F88C
:100AC0000090A178607803F0FBFC059B4D4A1B78F1
:100AD00001211170DA077FF578A9FEF7EBBF4FF01F
:100AE00007094B46E8E7D9F8D0003B4B90F83610A1
:100AF0009A7841446429A8BF642121EAE17180F811
:100B00003610002A40F04B8307F0D4FDA2E5D9F857
:100B1000D000314B90F837109A784144FE29A8BF95
:100B2000FE2121EAE17180F83710002AECD016206E
:100B300011F072FFD9F8D000E6E7089A264B5178F9
:100B40004144B1F5967FA8BF4FF4967121EAE17157
:100B500051709B78002B40F0B082D9F8D000D3E7D9
:100B6000D9F8D00081781C4B4144C829A8BFC821BE
:100B700021EAE17181709B78002BC5D0142011F01F
:100B80004BFFD9F8D000BFE7D9F8D0004178124B1D
:100B90004144C829A8BFC82121EAE17141709B786E
:100BA000002BB1D0132011F037FFD9F8D000ABE7FC
:100BB000D9F8D0000178084B4144C829A8BFC82102
:100BC00021EAE17101709B78002B9DD0122011F079
:100BD00023FFD9F8D00097E7B04600202F3400203B
:100BE000AC2103087C610020004B0020D846002087
:100BF000EC480020D34D6210D046002090380020F1
:100C0000344B0020FC2B0020089AC34B9179987834
:100C100041446429A8BF642121EAE171917100284F
:100C200040F05D820D2F98D00898BB4B41799A789F
:100C300041446429A8BF642121EAE1714171002A7D
:100C40008BD00E2011F0E8FED9F8D0005CE7D9F87F
:100C5000D000B14B017A9A784144C829A8BFC82175
:100C600021EAE1710172002A3FF44EAF0B2011F02E
:100C7000D3FED9F8D00047E7D9F8D000A64BC17908
:100C80009A784144C829A8BFC82121EAE171C171FD
:100C9000002A3FF439AF0A2011F0BEFED9F8D00087
:100CA00032E7D9F8D0009C4B81799A784144C82921
:100CB000A8BFC82121EAE1718171002A3FF424AF65
:100CC000092011F0A9FED9F8D0001DE7D9F8D0000D
:100CD000914B41799B784144C829A8BFC82121EA9A
:100CE000E1714171002B40F0F481112F7FF43AAF94
:100CF0000AE7D9F8D000884B01799B784144C8298C
:100D0000A8BFC82121EAE1710171002B40F0DB810D
:100D1000102F7FF43BAFF7E6089A11798844B8F1B9
:100D2000640FA8BF4FF0640828EAE87882F80480CE
:100D300011F08CFE784B9B78002B3FF40EAF032014
:100D4000414611F069FED9F8D000DDE6089A724BF1
:100D500011784144FA29A8BFFA2121EAE171117002
:100D60009B78002B3FF4F9AE012011F055FED9F825
:100D7000D000C9E6089A684B917841446429A8BF1D
:100D8000642121EAE17191709B78002B3FF4E5AE7C
:100D9000022011F041FED9F8D000B5E608985E4B6C
:100DA000C1799A78414481F30801C171002A3FF466
:100DB000D4AE052011F030FED9F8D000A4E6D9F861
:100DC000D000554BC1789B784144C829A8BFC821A1
:100DD00021EAE171C170002B40F0E5810F2F7FF413
:100DE000E9AE91E60E9ABAE43BF91110987840F614
:100DF00033039942A8BF1946B1F5617FB8BF4FF4DC
:100E000061710C2FA1F561714FF4966393FBF0F3C0
:100E100091FBF3F156D0182F7FF41CACD9F8D030E9
:100E2000C9B2C82993F817E00846A8BFC82086456C
:100E30003FF410AC384AD8759278002A3FF40AACD7
:100E4000384611F0E9FD05E4344A0392FFF722BA6F
:100E5000049B84F89200FA3A1B68A4F89020304A68
:100E6000069203F00403FEF71EBD2E4A049B1F6882
:100E7000138823F004031380012307F4805785F8B7
:100E80002130FFF7D7BA264A274B069210461A6838
:100E900026494FF47A73B3FBF2F3C3EB431203EB2F
:100EA00082030268DB005007A1F8B43000F19180A2
:100EB000049B1B6803F00403FEF7F5BC4FF0040924
:100EC0004B46F9E51A4B5B785FFA81F843453FF4EE
:100ED000C1AB404600F002FE0F4B9B78002B3FF465
:100EE000B9AB4146384611F097FDFFF7B3BB4FF061
:100EF00005094B46E0E54FF006094B46DCE54FF0AF
:100F000001094B46D8E54FF002094B46D4E54FF0B6
:100F100003094B46D0E500BFB04600207C4F0020BF
:100F2000D8460020DE460020606B0020DC680020F0
:100F300054600020049BA4491B680A60A34A0692DF
:100F400003F00403FEF7AFBC0021BB2A109173D05D
:100F5000B72A6DD0BE2A69D0BD2A46D0792A00F0C2
:100F6000F5807A2A00F0EB809E2A00F0E2809D2A2C
:100F700000F0D880AE2A00F0CE80AD2A00F0C48008
:100F8000EF2A00F0BE80FD2A00F0AD80FB2A00F0C1
:100F90000381FE2A00F0FD80F72A00F00A817B2AF7
:100FA0007EF47BAC4FF4FA61022000F0B7FCFEF750
:100FB00074BC874A00218748874C0260834A2170AD
:100FC0000692FEF770BC854A0121F4E7844A0221AB
:100FD000F1E7049B834A1B680A21118003F0040394
:100FE000FEF761BC0646FEF7ADBB4FF6FE737E4AC8
:100FF000764896890690D089334401449381D18103
:1010000015F0B8FDF1F74AFE15F09CFDF4F7EAFB88
:10101000049BB4F890201B68FA3A0021A4F89020B1
:1010200003F0040384F89210FEF73DBC0223DEE7D0
:101030000B464FF6FE71DAE70B460221D7E7049B19
:101040006A4A1B684FF4C8711180604A069203F027
:101050000403FEF728BCB8F1000F3EF4B6AD644CB3
:1010600094F88D30002B3EF4C3AB002384F88D3010
:10107000FEF7BEBB94F89420002A40F09D8094F8BF
:1010800096205249069182F0010284F89620FEF7DC
:101090000ABC15F06FFDF1F701FE15F053FDF4F7F2
:1010A000A1FB94F88E20FFF711BB514C10F06EFBA2
:1010B000002384F88D30FEF79BBB152011F0ACFCAB
:1010C000D9F8D00020E5102011F0A6FCD9F8D00006
:1010D0001EE6112011F0A0FCD9F8D00005E60D2085
:1010E00011F09AFC9EE50021012000F017FCB4F8F5
:1010F00090300022963BA4F8903084F89220FEF7BE
:10110000CCBB00210846F0E7FF2100201BF016FFB2
:1011100094F88E2034E7012100201BF00FFF94F893
:101120008E202AE70021FF201BF008FF94F88E2074
:1011300020E701201BF002FF94F88E2017E72D4ACC
:10114000137A43F001031372FEF7A7BB294A137AFF
:1011500023F001031372FEF7A0BB452014F0FAFD43
:10116000FF2014F0F7FD244814F0E0FD304614F0A1
:10117000F1FD059B1B78FEF7E3BC002B3FF46FAF3E
:101180001E491F4A09684FF47A7000FB031313606D
:1011900065E700210320A8E700210220A5E717202A
:1011A00011F03AFCD9E40F2011F036FCD9F8D00048
:1011B00014E60021042098E7044A84F8941084F887
:1011C00095000692FEF76FBBE45E0020D846002033
:1011D000163300205060002054600020643300204B
:1011E000B23300206E6F0020184B0020706F00207B
:1011F000EC2C0020B03F0020AC2103087C610020D3
:10120000E05E002030B4034600F12405064C07CC14
:101210000C3343F80C0C43F8081C43F8042CAB4285
:10122000F4D130BC704700BF84FA0208034B33F896
:101230000C2F02809B788370704700BF84FA0208ED
:1012400010B52920F0F7D7F9044630B11122002358
:101250008271C3712021F0F718F80A20F5F744F9DC
:101260002046F0F7AFFE034B00280CBF01220222FC
:101270001A7010BDC4410020614B1B78002B39D07F
:101280002DE9F0415F4B604D9B792C682860013B54
:1012900082B0041B032B00F28280DFE803F03002EF
:1012A000282811F087FB002800F08180574B58490F
:1012B0001B786A8FD1ED037A6A64DB0700F18380C3
:1012C00002FB04F007EE900ADFED526A524BB8EED3
:1012D000E77AD5ED107A5A60E7EE267A1A60BDEE0D
:1012E000E77AC5ED107A85ED0F7A83ED027A02B0C8
:1012F000BDE8F081484A1360536093607047474AE5
:10130000474BD279DFF82C8133F81220B8F902303C
:101310004448B8F9001092B207EE902A40F6E4472C
:1013200007FB02F6C3EB1633B8EE670A4FF47A7682
:1013300006FB03F393FBF1F32B61EFF739F8D5F8D4
:1013400010E0D5ED027ADFED336AB8F90220324BB6
:10135000B8F900C0C3F804E00EFB04F007EE100A71
:10136000B8EEC77ABCEEC06AE7EE267A8DED016A68
:10137000BDF80410C5ED027ABDEEE77A07FB01F770
:10138000C2EB173706FB07F683ED027A96FBFCF6F5
:1013900085ED017AEE601E6002B0BDE8F0811E4B63
:1013A00000221A605A609A6002B0BDE8F0811E4BBC
:1013B0001B68DE067FF57AAF144B6A8F1B786A6470
:1013C000D9070FD47CE7FDEEE77A184E17EE900AA6
:1013D000A0F57A7101FB01F386FB0306D817C0EB79
:1013E00026100844B5F93810114B00FB01F083FBBF
:1013F0000013C017C0EBA31002446A6460E700BF8B
:1014000056560020A0460020C02D0020F266002085
:10141000585600202FE33E319C5500208461002067
:10142000A0610020D42D0020706B00201F85EB519F
:10143000D34D6210084B0020F0B5244B5B79012B93
:1014400083B00ED0224900230B804B80214B1B78A8
:10145000022B04D1204B48880A8818805A8003B098
:10146000F0BD1E4A1E4B92781E4D33F81240A4B2B6
:1014700007EE904A05F14C00B8EE670AEEF798FFC8
:10148000194A1349107896785378FCEEC07A00EB2D
:101490004010CDED017ABDF8042044F6FB77C3EB94
:1014A000033300FB027200FB0474B2FBF3F2B4FBE3
:1014B000F3F3B2FBF6F2B3FBF6F392B29BB2A5F8EC
:1014C0004820A5F84A300A804B80BFE7A04600209C
:1014D000A8550020385600203C560020846100208A
:1014E000A0610020C02D002001330020F8B5244D5C
:1014F000244C25496E79254B254A264F0420087037
:1015000084F8700000216420012EA4F87210A4F861
:10151000741039701970596058701180518020D042
:10152000A9791D4A00230129136084F8763053609D
:10153000936007D0022904D1184AE3635360936093
:10154000F8BDF8BD164A636053609360D3609FEDA9
:10155000150A02F110004CF25031BDE8F840F1F7E5
:1015600079BF282204F148001DF0FFFF4CF25031F2
:101570009FED0D0A04F14C00F1F76CFFD0E700BFBE
:10158000A0460020C02D0020CC460020BC2B00200F
:10159000A8550020565600209C550020FC2D002008
:1015A000C42D0020CDCCCC3ECDCCCC3D2DE9F04F90
:1015B0000C68DFF800E32588BB4EB6FBF2F285B07D
:1015C000013B013A74459EB2ADB292B2BDF838709B
:1015D0009DF83CC062D0B54B9C425FD0B4F1804FC7
:1015E0005CD0A3F598339C4258D003F580639C42AD
:1015F00054D0AF4B9C4257D003F580639C4253D0EC
:1016000025F4407503F58C33ADB29C422580E6622B
:1016100022850FD003F500639C420BD003F5406395
:101620009C4207D003F580639C4203D003F580639E
:101630009C4201D100232386012363614A79CB793F
:10164000BCF1000F01D083F0020313F004052FD08A
:10165000002113F0020F4FF040060CBF4FF00808B6
:1016600088468C46039189468E460B4601914FF47D
:10167000806502964FF0040A0C2A00F2DC80DFE855
:1016800012F0AA00DA00DA00DA008600DA00DA00E6
:10169000DA006100DA00DA00DA002A00844B25F073
:1016A00070059C42ADB2A7D12580E6622285C3E7D2
:1016B0004FF480660396012603F002030295AA46C2
:1016C000A8464FF480414FF4805C4FF010094FF46E
:1016D000807E0196D0E7256ADFF8D8E125F48055B1
:1016E0002562256A6668D4F81C8025F4005545EA11
:1016F0000C0C744528F4E6454CEA033345F4C04528
:1017000000F0E6800EF5006E744500F0E180666042
:10171000E56127642362E36943F40063E361636C7A
:1017200043F400436364238821469BB243F00103E2
:1017300021F8343B00238D18446005608B5005B0C0
:10174000BDE8F08F216ADFF86C9121F4807121628D
:10175000216A6668D4F81CA021F4007141EA0E0EDB
:101760002AF0730A4C454EEA03234AF0600100F068
:10177000A380DFF838E1744500F09E806660E16187
:10178000E7632362E36943F00803E361C7E7216A83
:10179000484E21F010012162216A6568D4F818C012
:1017A00021F0200E2CF080714EEA090921F4E64167
:1017B000B44249EA031341F4C04168D006F500661B
:1017C000B44264D06560A161A7632362A36943F456
:1017D0000063A361A3E7216A019EDFF8D8C021F06E
:1017E00001012162D4F820906568A16921F480315B
:1017F000334321F0730129F00206644543EA0603EE
:1018000041F0600138D0294EB44235D006F540662B
:10181000B44231D006F58066B4422DD006F580661C
:10182000B44229D06560A16167632362A36943F074
:101830000803A36173E70C2A3FF671AF01A353F8C5
:1018400022F000BF2D1801081F1701081F170108FB
:101850001F170108CD1701081F1701081F170108DE
:101860001F170108851701081F1701081F17010816
:101870001F1701081717010823F00C0343EA080398
:1018800025F4407543EA0A0345EA0E05CAE723F04A
:101890008003029E43EA081323F040033343039E70
:1018A00025F4406535438DE700A24A040034014029
:1018B00000100040002C014023F4006343EA082399
:1018C00023F4806326F440562B434CEA060655E782
:1018D00026F480460E431AE770B5084C236AA28CA2
:1018E0001A850E4619F066FA0546304619F062FA76
:1018F000236AA28C9A61284670BD00BF3C6E00200E
:1019000010B5054C236AA28C1A8519F053FA236A84
:10191000A28C9A6110BD00BF3C6E00202DE9F04101
:101920004A4C94F8783073B304282CD8484AB4F859
:101930008E309FED487ADFED486A94F88C5002EBC8
:10194000800007EE903A0269B4F89230F8EEE77A38
:10195000642006EE102A00FB032367EE877AB8EEB8
:10196000C66A07EE103A67EE867AB8EEC77A0E4678
:1019700087EE870A394900270F6020EE260A002DDE
:101980004ED0012D01D0BDE8F081D4F8888007EE5B
:10199000908AF8EE677A27EE800A1BF025FD60B981
:1019A000E06FF0F7E1FAB4F890003044F4F7F6FD98
:1019B000E06FBDE8F041F0F7DCBA2949294A4862F6
:1019C000C1F82C805762C2F82C80EFF311835020AD
:1019D00080F312880D80DBB2158083F31188224BCF
:1019E000CD60D5601A68B4F89010114431441A687B
:1019F0009142FCD81A491B4A0B88E06F23F001037F
:101A00001B041B0C0B80138823F001031B04002410
:101A10001B0C1380CC60D460BDE8F041F0F7A9BA8C
:101A2000D4ED227AD4F88050F8EE677A27EE800A57
:101A30001BF0DAFC0C4B28601B68B4F890101944BA
:101A40003144C4F89810BDE8F08100BFC02D0020DB
:101A500084FA02080AD7233CCA269B3E1C46002073
:101A600000100040001400407C61002008B5044BC9
:101A7000D86FF0F779FA034B00221A6108BD00BF56
:101A8000C02D00200014004008B5044BD86FF0F7BB
:101A900070FA034B00221A6108BD00BFC02D002060
:101AA00000100040012800D970470129FCD8884265
:101AB000FAD030B4084B01EB410103EB810100EB9C
:101AC000400080000D684C688968C550C218546099
:101AD000916030BCE8E700BF443F0020022806497F
:101AE000064B074A28BF0220487000EB400003EB7A
:101AF0008000106010F0AABF54600020443F002016
:101B0000E85E00202DE9F04F2DED088BBE4CBF4B59
:101B1000C4F89C3087B00023C4F8A030F1F786FFEA
:101B2000EFF78EFDFFF78CFBF1F782F808B9F4F7B9
:101B300043F8F3F757FE0522B549B6481DF060FD9E
:101B400008B1F4F739F894F8A430B34D43F0010329
:101B500084F8A430B14B9A78B14B1A70B14B1B6822
:101B60002B600AF0A7FD01210220F0F711FAF0F72F
:101B7000DDFE2B681F070BD5AB4B1A7A0A2A07D854
:101B80000123934040F20342134201D00AF01AFCB1
:101B90006420F4F703FDF4F7FFF8A44B94F8001168
:101BA000187B9E78A24B94F8012103F1040E13F8E0
:101BB000017F17B1874208BF01461F7917B1B742AD
:101BC00008BF32469E45F2D184F8001184F8012105
:101BD000B4F800312BB1974BC4F8FC30964BC4F8E5
:101BE0000C33964E0AF0ACFA954B32781A7007F027
:101BF00079FA07F0ABF82A68924B039612F4805FEB
